:020000040800F2
:1040000000500020B1FB00081DCD000821CD0008A4
:1040100025CD000829CD00082DCD000800000000A6
:1040200000000000000000000000000035CD000886
:1040300031CD00080000000039CD0008319900089A
:104040003DCD000841CD000845CD000849CD000810
:104050004DCD000851CD000855CD000859CD0008C0
:104060005DCD000861CD000865CD000800000000AE
:104070000000000000000000000000000000000040
:10408000000000000000000085CD000889CD000878
:1040900099CD0008A9CD0008B9CD0008C9CD000808
:1040A000CDCD0008D1CD0008D5CD0008D9CD000870
:1040B000DDCD0008E1CD0008E5CD0008E9CD000820
:1040C000EDCD0008F1CD0008F5CD0008F9CD0008D0
:1040D000FDCD000801CE00083590000809CE00088B
:1040E0000DCE000811CE000815CE0008000000001B
:1040F00000000000000000000000000000000000C0
:0C41000000000000000000005FF800005C
:1041100030BF704720BF704740BF7047BFF36F8FFD
:104120007047BFF34F8F7047BFF35F8F704701DF5A
:104130007047EFF31480704780F31488BFF36F8FDC
:104140007047EFF30980704780F309887047EFF3F9
:104150000880704780F30888704772B6704762B66F
:10416000704771B6704761B6704780F31188704729
:10417000EFF31280704740BA704700BA70470000F2
:104180000E4B10B59B680E4813F4004C0D490E4AB7
:104190000E4B09D04FF0010C0D4C80F800C00D48BB
:1041A0001C6010600C6007E080F800C00A480860DE
:1041B0000A4911600A4A1A6010BD00BF0008014098
:1041C000BC0D0020240E0020E00F0020A00E0020D7
:1041D000A9920008199F00083D93000879980008EB
:1041E000C197000837B50AF0B5F96F4B00254FF4B9
:1041F00080301D700AF0CEF90AF032FB0128044627
:1042000027D1102009F090FC28460AF013FA28461E
:104210000AF024FA4FF480600AF016FA4FF44030A6
:104220004FF4E0110AF0E2F920460AF0EBF93920E8
:104230000AF000FB0028FAD0022009F05DFC022001
:104240000AF0E6F90AF0EEF90828FBD1564B0122F4
:104250001A70042001210AF0A3FA03238DF8063016
:10426000153301A951488DF807304FF48073ADF82C
:10427000043009F08DFE06200AF0D6FA012001462E
:104280000AF08EFA4FF480414FF000600AF084F893
:104290004FF4407009F0E2FF00F050FA00F0B4FB78
:1042A000FFF76EFF00F060F905F0A2FB05F072FB6E
:1042B00004F0E2FD00F080F800F072F930B100F097
:1042C0006FF93B4C607000F06BF9A060384C00F067
:1042D000BDF9207804F00EFFE07804F067FE354B5E
:1042E0001B7823B922696079A16805F0C1F8314BC8
:1042F0001B780BB105F0C2FE06F09EFC08F0ACFA8C
:1043000001F096FD05F0D6FE06F0FCFC274B4FF4BD
:1043100000721A61A2F5A07203F580635A6105F07C
:1043200033FB044603F028FF06F000FD05F0D4FE41
:1043300005F02AFB001B0028B8BF4042B0F57A7F89
:1043400025DD1C4C237893B1184B9B6813F4004374
:104350001AD1237005F052FE05F02EFDFFF710FF75
:10436000134B1A695879996805F082F80CE00F4BE5
:104370009B6813F4004F07D005F03EF8012323702B
:10438000FFF7FEFE05F07AFE05F0FEFA044600F0A7
:104390005DF900F04DF90028C4D006F04DFC01F0A5
:1043A00047FD06F0AFFCBDE7C80F00200008014044
:1043B00004000020BC0D0020134B82B01B7803B317
:1043C000124B4FF400625A61A2F580621A61002319
:1043D00001E0019B01330193019A0D4B9A42F8D9F8
:1043E0000A4B4FF400621A61A2F580625A61002301
:1043F00001E0019B01330193019A054B9A42DFD8FA
:10440000F7E702B0704700BF440E0020000C0140E7
:104410003F0D0300072816D8DFE800F00406080A5D
:104420000C0E101201220CE002220AE0042208E025
:10443000082206E0102204E0202202E0402200E0F0
:104440008022014B5A61704700140140072816D89A
:10445000DFE800F00406080A0C0E101201220CE03E
:1044600002220AE0042208E0082206E0102204E00A
:10447000202202E0402200E08022014B1A617047B6
:104480000014014038B50546002455FA04F2E3B2A1
:1044900012F0010F184602D0FFF7D8FF01E0FFF736
:1044A000B9FF0134082CF0D138BD00BF072805D86A
:1044B000DFE800F0060B10151A1F2429002026E063
:1044C000134BD86800F0010021E0114BD868C0F30D
:1044D00040001CE00E4BD868C0F3800017E00C4B86
:1044E000D868C0F3C00012E0094BD868C0F30010D0
:1044F0000DE0074BD868C0F3401008E0044BD868C3
:10450000C0F3801003E0024BD868C0F3C0107047BE
:1045100000140140052804D8DFE800F0050A0F1454
:10452000191E00201CE00F4B986800F0010017E0F6
:104530000C4B9868C0F3400012E00A4B9868C0F337
:1045400080000DE0074B9868C0F3C00008E0054B01
:104550009868C0F3001003E0024B9868C0F3401065
:10456000704700BF0018014062B6704772B67047CE
:1045700010F0010F03D0094B10221A6102E0074B23
:1045800010225A6110F0020F03D0044B20221A614E
:1045900002E0024B20225A61704700BF000C01402C
:1045A0001C4B9A689B6812F4807F14BF0020802007
:1045B00013F4007F03D1002814BFC0204020154B06
:1045C0009B6813F4806F134B08BF40F020009B687A
:1045D00013F4006F0F4B08BF40F010009B6813F4FA
:1045E000805F0C4B08BF40F008009B6813F4005F2D
:1045F000084B08BF40F004009B6813F4804F054B44
:1046000008BF40F002009B6813F4004F08BF40F061
:104610000100704700100140044B18780138C0B207
:1046200001288CBF00200120704700BF2802002015
:10463000044B1878012801D0002001E002221A70F2
:10464000704700BF2802002000207047082008B5EE
:1046500005F0B6F9592804D9064B1A784AB901323F
:1046600006E0082005F0ACF9542802D8014B0022DE
:104670001A7008BD2802002008B5072805D8DFE811
:1046800000F006080D121720252A002027E0002040
:104690000FE0134B9868C0F3400020E0104B98687F
:1046A000C0F380001BE00E4B9868C0F3C00016E01A
:1046B000042005F085F9B0F5006F94BF00200120BB
:1046C0000DE0074B9868C0F3401008E0044B986871
:1046D000C0F3801003E0024B9868C0F3C01008BD1F
:1046E0000010014038B500242546E0B2FFF7C4FFB2
:1046F00020B10123A34043EA0505EDB20134082CA3
:10470000F3D1284638BD00BF08B5C0B206F042F864
:1047100008BD00BF08B5C0B206F02CF808BD00BF48
:1047200008B510B109F042FE01E009F047FE08BDEE
:1047300008B5C90805F0AAFE08BD00BF2DE9F3477A
:10474000644F6548012101AD09F0B2FC042001214C
:1047500003240AF025F81026384642F2026329465F
:10476000ADF804308DF806408DF8076009F010FCB4
:1047700040F202634FF0040838467B6129464CF250
:104780000803DFF868A1ADF804308DF806408DF815
:10479000078009F0FDFB4FF0010338462946482702
:1047A000ADF804308DF807708DF8064009F0F0FB85
:1047B0000820012109F0F4FF41F6FD495046294641
:1047C000ADF804908DF806408DF8076009F0E0FB25
:1047D000CAF810903046012109F0E2FF4FF0FF09BE
:1047E0003E482946ADF804908DF806408DF80780C4
:1047F00009F0CEFB4FF60073384829460AF5006AE7
:10480000ADF804308DF807708DF8064009F0C0FB54
:104810002020012109F0C4FF4FF0FF335046294604
:104820002F4FADF804308DF806408DF8076009F081
:10483000AFFB4FF47F43CAF8103040200121CAF883
:10484000149009F0ADFF40F2FF3338462946ADF829
:1048500004308DF807808DF8064009F099FB4FF67B
:10486000004329463846ADF804308DF806408DF8EF
:10487000076009F08DFB4FF47C4301217B611948EF
:1048800009F016FC00231A461946124C4FF4005545
:1048900065612046A468013314F4804F4FF400543E
:1048A0000461806808BF013110F4804F18BF0132E5
:1048B0000A2BEAD10A2903D10A2A01D1012200E0F8
:1048C0000022094B04481A70012109F0F1FBBDE8F0
:1048D000FC8700BF000801400002300000100140CA
:1048E0000018014000043000440E0020000C01407C
:1048F00070B504460D46164608287AD8DFE800F061
:1049000005101316191C1F0A0D003B4B4FF4805263
:104910005A6119E04FF4007213E04FF4807210E016
:104920004FF480620DE04FF400620AE04FF48052D1
:1049300007E04FF4005204E04FF4804201E04FF4EE
:1049400000422E4B5A6110E02D4802210AF08AF8ED
:104950000028F9D029462A480AF028F828480121D9
:104960000AF080F80028F9D00FE0264802210AF06A
:1049700079F80028F9D0294622480AF017F821488A
:1049800001210AF06FF80028F9D03EB3082C30D886
:10499000DFE804F005101316191E210A0D00164B4E
:1049A0004FF480521A611DE04FF400720DE04FF495
:1049B00080720AE04FF4806207E04FF4006204E086
:1049C0004FF4805201E04FF400520C4B1A610BE09F
:1049D0004FF48042F9E74FF40042F6E714B1082C97
:1049E00007D801E0064800E0064809F0E1FFC0B240
:1049F00000E0002070BD00BF000C01400014014029
:104A000000380040003001402DE9F04F01218BB00B
:104A10004FF4804009F0D2FE494C012009AF014615
:104A200009F0BEFE03264FF0180B204639464AF225
:104A30000003DFF81491ADF824304FF0040A8DF82C
:104A400026608DF827B009F0A3FA204639464FF4C6
:104A500080430DF11008ADF824308DF826608DF8F4
:104A600027A009F095FA4FF48273002402224FF434
:104A7000007C012548464146ADF812304FF008034E
:104A8000ADF81620ADF81AC00392CDF808C0ADF805
:104A90001C30ADF81040ADF81440ADF81850ADF82A
:104AA0001E40ADF8204009F00DFF4846294609F0A8
:104AB00045FF29464FF4805009F072FE09F5504930
:104AC0002846214609F0F4FA484639464FF0A0033B
:104AD000ADF824308DF827B08DF8266009F058FA2B
:104AE000484639464FF04003ADF824308DF8266033
:104AF0008DF827A009F04CFA039ADDF808C04FF4AE
:104B000082734146ADF812300E484FF02803ADF8DD
:104B10001620ADF81AC0ADF82040ADF81040ADF841
:104B20001440ADF81850ADF81C30ADF81E4009F037
:104B3000C9FE0448294609F001FF0BB0BDE8F08F1B
:104B4000000C01400030014000380040014B187853
:104B5000704700BF2C0200202DE9F8450546144699
:104B60000F4600295FD000285DD081425BD0022A29
:104B700094BF0026012601D8510101E0D11E490150
:104B800041F00601C9B2304607F0CEFA022C824647
:104B900001D8610101E0E11E490141F00C01C9B2F7
:104BA000304607F0C1FA804628460DF0A7F80546C2
:104BB00038460DF0A3F8014628460DF0ABF907463C
:104BC00050460DF09BF839460DF0A4F90DF0B4FAFB
:104BD000054640460DF092F839460DF09BF90DF070
:104BE000ABFA1249002814BF80464FF0010838463E
:104BF000002D08BF01250DF077FA18B14146204677
:104C000007F080FD022C01D8610101E0E11E49019D
:104C100041F00601C9B230462A4607F04DFB044B6D
:104C2000E41801232371BDE8F88500BF0000A0410E
:104C30002C02002010B5114B0446C3181B79DBB1C0
:104C4000022801D8410101E0C11E49010C4B41F08D
:104C5000060153F82420022C94BF00200120C9B281
:104C600007F0C4FB074BE0B253F8241007F04AFDED
:104C7000024BE4180023237110BD00BF2C0200205A
:104C8000A40D00208C09002013B59C4CA0780528A9
:104C900000F283836378A32B00F0E4825BD8842B3B
:104CA00000F0D38028D8062B00F0428110D8022BC8
:104CB00000F0CB8006D8002B00F0AB80012B40F039
:104CC0006A83ADE0042B00F0FB8000F21D81EEE072
:104CD000802B00F09E8009D80C2B00F049810D2B11
:104CE00000F06381072B40F0568330E1822B00F007
:104CF000798100F2E58093E0932B00F0568114D87F
:104D0000872B00F0788106D8852B00F0D080862B89
:104D100040F04183F8E08C2B00F09C818D2B00F05B
:104D2000A5818A2B40F037836EE19A2B00F0078231
:104D300008D8952B00F0AF81C0F01A81992B40F074
:104D40002A83D7E1A12B00F0838200F28682A02B78
:104D500040F0218377E2B22B00F0E78227D8AA2B1C
:104D600000F0BA8211D8A62B00F09C8206D8A42BA2
:104D700000F07C82A52B40F00E8385E2A82B00F08A
:104D8000A2825E4B00F2A48299E2AE2B00F0BB82BD
:104D900006D8AC2B00F0A882584B00F2B0829FE2FC
:104DA000B02B00F0B982554B00F2BB82B0E2C22BAF
:104DB00000F0028215D8B72B00F0E28208D8B52B9C
:104DC00000F0BC8200F2C482B32B40F0E482B0E277
:104DD000C02B00F0BC8000F2E881B82B40F0DB82F1
:104DE000D4E2CC2B00F00B8209D8C72B00F0A080B6
:104DF000C82B00F0F381C32B40F0CD82E4E1D52B2A
:104E000000F01082D62B00F01482D42B40F0C38225
:104E1000FEE1022801D841010AE0C11E490107E074
:104E2000022801D8410101E0C11E490141F00201FF
:104E3000324BC9B25A68DB78022894BF00200120A7
:104E400043EA022207F038FAAAE2022801D8410117
:104E500001E0C11E4901294C41F00801E378626874
:104E6000022894BF00200120C9B243EA022207F0C1
:104E7000BDFAA078022801D8410101E0C11E490114
:104E80001E4C022894BF00200120E378626841F0A4
:104E9000060143EA0222002AB8BF5242C9B207F013
:104EA000A5FA174AA378D31801221A7178E20228CA
:104EB00001D8410101E0C11E490141F00A01DDE0D4
:104EC000022801D8410101E0C11E49010B4C41F00B
:104ED0000601E3786268C9B243EA0222022894BF5D
:104EE0000020012007F082FAE2786068A37842EAA5
:104EF0000020034A03499A1815E000BF6407002008
:104F00002C020020A40D0020994CE378616843EA4C
:104F1000012107F0F7FBE2786068A37842EA0020FD
:104F2000944A95499A1841F823000023137137E2F7
:104F30008F4B924AD978924B924C1B5C02EB4012F9
:104F40004FF0010C04F800C0022B517254E1884B61
:104F50008A4AD9788A4B8B4C1B5C02EB40124FF08B
:104F6000010C04F800C09172002B40F0198204E299
:104F7000022801D8410101E0C11E490141F014019C
:104F8000C9B2022894BF0020012001AA07F01EF92F
:104F9000774A9DF805305168D27852EA012114BF52
:104FA00043F0020323F0020391E0022801D84101FB
:104FB00001E0C11E490141F01401C9B2022894BFA9
:104FC0000020012001AA07F001F9694A9DF8053087
:104FD0005168D27852EA012114BF43F0010323F053
:104FE000010374E0022801D8410101E0C11E49011A
:104FF00041F0040142E0022801D8410101E0C11E54
:10500000490141F00E0139E0022801D8410101E0D7
:10501000C11E490141F01401022894BF0020012063
:10502000C9B201AA07F0D2F8514B9878DB78022870
:1050300001D8410101E0C11E490141F01401C9B28A
:10504000022894BF0020012001AA8DF8063007F045
:10505000A3FAA5E1464B494ADB7802EB4012C3F1C3
:105060000801C9B2D37205F065FD99E1022801D8A3
:10507000410101E0C11E490141F01A013C4BC9B296
:105080005A68DB78022894BF0020012043EA0222FC
:1050900007F0ACF984E1022801D8410101E0C11E0A
:1050A000490141F01401C9B2022894BF0020012037
:1050B00001AA07F08BF82E4A9DF805305168D27886
:1050C00052EA012114BF43F0040323F004038DF8D6
:1050D0000530274B9878022801D8410101E0C11E14
:1050E000490141F01401C9B2022894BF00200120F7
:1050F00001AAACE7022801D8410101E0C11E490123
:1051000041F01801022894BF0020012001AAC9B271
:1051100007F05CF8164A9DF805309078D27802289E
:1051200001D8410101E0C11E490141F0180102F01E
:105130000F0223F00F03C9B242EA03032DE0022855
:1051400001D8410101E0C11E490141F018010228C6
:1051500094BF0020012001AAC9B207F037F8044A21
:105160009DF805309078D27802280DD841010DE0E5
:10517000640700202C0200208C090020A40E0020CF
:10518000D80F0020D00F0020C11E490141F01801A6
:1051900003F00F03C9B243EA0213022894BF0020B0
:1051A000012001AA8DF8053051E77E4B7E4ADB785D
:1051B00002EB40100372F3E0E3786268400143EAD7
:1051C0000222794BC250EBE0764B77495A68DB7884
:1051D00001EB401043EA02234360E1E0714B724A65
:1051E000D978724B724C1B5C02EB40124FF0010CF1
:1051F00004F800C0032BD17740F0D280BDE0626894
:10520000E378694943EA022301EB4010C381C7E018
:10521000644B65495A68DB7801EB401043EA02238E
:105220004361BDE05F4B604ADB7802EB401083775F
:10523000B6E05C4B5C495A68DB7801EB401043EA0E
:1052400002238383ACE0574BD97805F065FCA7E0D7
:10525000544BD97805F056FCA2E0524BD97805F0B2
:1052600015FB9DE0E17805F005FB99E004F06CFF8B
:105270004C4B20B9D978987805F0E4FA90E0D978C9
:10528000987805F0AFFA8BE004F05EFF454B20B94B
:10529000D978987805F0CAFA82E0D978987805F03C
:1052A00089FA7DE004F050FFE178A37818B9184638
:1052B00005F0B0FA74E0184605F088FA70E0D97885
:1052C00005F09CFA6CE0374BD97805F08BF967E074
:1052D000D97805F07BF963E0E17805F06BF95FE0E0
:1052E000D97805F05BF95BE02E4CE17805F04AF9DE
:1052F000A178304BE27803EBC1035A7150E0D978C2
:1053000005F0DCF84CE094F9031005F0CBF847E029
:10531000D97805F091FB43E0224BD97805F080FB6A
:105320003EE0D97805F070FB3AE0E17805F060FBEB
:1053300036E01C4BD97805F043FB31E0194B1A4994
:105340005A68DB7801EB401043EA0223836127E0CF
:105350001449184B4C68CA7842EA042243F83020BA
:1053600022B903EBC003597905F00CF90D4B0F4A34
:105370009878125C012A13D1D978FFF7D9F90FE098
:105380000C4AE37802EBC000037109E0054BD978C1
:1053900005F064FA04E0032200E00422064B1A70D0
:1053A0001CBD00BF64070020A40E0020D80F002001
:1053B000D00F0020E40D00208009002013B5814BA0
:1053C0009878052800F2D9825B787F4CD62B00F2C2
:1053D000D182DFE813F0D700DE00EE00FB0004010D
:1053E00006010A010F011401540170015E01280138
:1053F0003D01CF02CF02CF02CF02CF02CF02CF02B8
:10540000CF02CF02CF02CF02CF02CF02CF02CF0214
:10541000CF02CF02CF02CF02CF02CF02CF02CF0204
:10542000CF02CF02CF02CF02CF02CF02CF02CF02F4
:10543000CF02CF02CF02CF02CF02CF02CF02CF02E4
:10544000CF02CF02CF02CF02CF02CF02CF02CF02D4
:10545000CF02CF02CF02CF02CF02CF02CF02CF02C4
:10546000CF02CF02CF02CF02CF02CF02CF02CF02B4
:10547000CF02CF02CF02CF02CF02CF02CF02CF02A4
:10548000CF02CF02CF02CF02CF02CF02CF02CF0294
:10549000CF02CF02CF02CF02CF02CF02CF02CF0284
:1054A000CF02CF02CF02CF02CF02CF02CF02CF0274
:1054B000CF02CF02CF02CF02CF02CF02CF02CF0264
:1054C000CF02CF02CF02CF02CF02CF02CF02CF0254
:1054D000CF02CF02CF02D700DE0085010401EE002B
:1054E000FB0006018E01CF02CF029701CF02AA0175
:1054F000AF01CF02CF02CF02CF02CF023D01280180
:10550000C101CF02CF02CF02D601EB015E017001D3
:105510001401CF02CF025C025F02620265026802E0
:105520007502830290029302960299029C029F02E6
:10553000A402A702AB02AE02B102B402B702BA02E1
:10554000BD02C202C602CC02CF02CF02CF02CF02FE
:10555000CF02CF02CF020F01FF01040208020D02A9
:105560000F02CF020A011102CF02CF02CF021602B0
:10557000CF021B021D023402CF02CF02CF024D0226
:1055800052025702022801D841010AE0C11E490116
:1055900007E0022801D8410101E0C11E490141F0A4
:1055A0000201C9B2022894BF0020012006F0BCFD10
:1055B000CFE0022801D8410101E0C11E490141F0BC
:1055C0000801BFE06407002080090020022801D8FC
:1055D000410101E0C11E490141F00A01B2E0994BCD
:1055E00000E0994B53F82030BFE1984B03EB40109B
:1055F000437ABAE1954B03EB4010837AB5E1022878
:1056000094BF0020012006F061FC914B9B78022B97
:1056100088BF033B5B00012212FA03F303420CBF75
:105620000022012228E0022801D8410101E0C11E28
:10563000490141F0140101AAC9B2022894BF002017
:10564000012006F0C3FD9DF80520C2F3400213E0DF
:10565000022801D8410101E0C11E490141F01401B5
:1056600001AAC9B2022894BF0020012006F0AEFDB5
:105670009DF8052002F00102764B5A6080E1022875
:10568000744C01D8013000E00230C0B2FEF7F4FFE4
:1056900022E17C21022894BF0020012001AA06F00B
:1056A00095FD6B4B9DF806209B78022B88BF033B32
:1056B0005B00022110E07C21022894BF0020012021
:1056C00001AA06F083FD624B9DF806209B78022B11
:1056D00088BF033B5B00012111FA03F313429EE7ED
:1056E000022801D8410101E0C11E490141F0040135
:1056F00028E0022801D8410101E0C11E490141F022
:105700000E011FE0022801D8410101E0C11E49013C
:1057100041F0140101AAC9B2022894BF002001205F
:1057200006F054FD9DF80620A6E704F0EBFCC0F15E
:105730000800D1E0022801D8410101E0C11E490161
:1057400041F01A01C9B2022894BF0020012006F0DE
:1057500025FD404B586013E1022801D8410101E0CA
:10576000C11E490141F0140101AAC9B2022894BF27
:105770000020012006F02AFD9DF80520C2F38002DA
:105780007AE7022801D8410101E0C11E490141F038
:10579000180101AAC9B2022894BF0020012006F016
:1057A00015FD9DF8052002F00F0265E7022801D8DB
:1057B000410101E0C11E490141F0180101AAC9B22D
:1057C000022894BF0020012006F000FD9DF805206E
:1057D000120951E71D4B03EB4010037AC5E01B4B48
:1057E0004001C358C1E0194B03EB40104368BCE0D3
:1057F000194BF7E6194BF5E6144B03EB4010C37F4A
:10580000B3E0124B03EB4010C389AEE0144BE9E662
:10581000144B00221B5C626013B10E4B01325A60C4
:10582000114B104A1B5C0021115423B1094B5A68DB
:1058300042F002025A600C4B00221A54A0E00B4BBB
:1058400084E000BFA40D00208C090020A40E0020DD
:105850006407002080090020C00D0020680F002090
:105860002C0E0020900E00201C0E0020980E002010
:105870004C4B03EB4010436977E04A4B03EB40107D
:10588000837F72E0474B03EB4010838B6DE004F0A5
:1058900041FC21E004F046FC1EE004F04BFC1BE060
:1058A00004F052FC18E004F04FFC3F4C3F4B18B999
:1058B000987804F05DFC0FE0987804F081FC0BE030
:1058C00004F042FC384C394B18B9987804F05AFC73
:1058D00002E0987804F088FC606051E004F034FC49
:1058E000314C324B18B9987804F056FCF4E79878AC
:1058F00004F070FCF0E704F059FCEDE704F07EFCE6
:10590000EAE704F085FCE7E704F08CFCE4E704F048
:1059100093FCE1E7264B03EBC000437925E004F05C
:105920009FFCD9E704F0A6FC40B2D5E704F0B6FC32
:10593000D2E704F0BBFCCFE704F0C0FCCCE704F0F6
:10594000C5FCC9E704F0D2FCC6E71A4B1B5C0CE0AF
:10595000144B03EB4010836907E0154B53F83030CC
:1059600003E0134B03EBC0000379636008E004F02D
:10597000F5FBB1E70323237002E00B4B04221A70FE
:105980000D4B1B786BB1084B0C495A680C4B0A60E5
:105990001AB91A6842F0080202E01A6822F00802F6
:1059A0001A601CBDA40E002080090020640700209E
:1059B000E40D0020DC0D00207A0900206809002099
:1059C0006C07002008B5754B9878052801D904228A
:1059D000E0E05B789A2B20D8992B74D2822B63D08D
:1059E0000BD8062B44D003D8042B3BD0052B0AE060
:1059F000072B4AD00C3B012B0CE08C2B56D005D842
:105A0000832B2FD0862B40F0C4802DE08D2B58D0D7
:105A1000933B022B00F2BD8044E0C72B28D00ED868
:105A2000C12B5DD005D8B52B4FD0C02B40F0B18035
:105A30002BE0C22B65D0C32B40F0AB8067E0D22BAC
:105A40007DD005D8C82B6AD0CC2B40F0A2806BE06B
:105A5000D52B00F08680D62B00F08E80D42B40F022
:105A6000988072E0062100E00C2106F0FBFB93E039
:105A70004B4A43010833D31803EB401102EB4010AB
:105A800001F14102101A597838E0454A43010833C0
:105A9000D31803EB401102EB401001F14202101A3F
:105AA00099782BE01421E0E70421DEE73C4B821CCF
:105AB00003EB40110B3103EB401001EB4213181ABA
:105AC00058E01A21D1E71821CFE74301344A03F106
:105AD000180151180230D31801EB4010C01A3EE0F3
:105AE0002F4B8200013200F1020C03EBC20101EBEB
:105AF0004C1103EB4010081A13F8321003F072F83F
:105B00004AE02749831C01EB4011580127E0244A51
:105B1000831C02EB4010011D01EB43131EE0204AE1
:105B2000430199181F3120E01D4B821C03EB4011EB
:105B30000E3103EB401001EB4213181A25E0184B0D
:105B4000410110315918821C04E0154B821C03EBF3
:105B50004011143103EB401001EB4213181A0422D8
:105B600014E00F4A430199181E310230D31801EB9B
:105B70004010C01A012209E0094A430199181C315A
:105B80000230D31801EB4010C01A022202F0ACFF21
:105B900002E00322034B1A7008BD00BF6407002017
:105BA000A40E00208009002038B59B4DA878052858
:105BB00001D904222CE16B78952B21D8932B80F00E
:105BC000A8800D2B0BD80C2B80F0A380052B5FD069
:105BD00001D8042B0AE0062B7DD0072B23E0862B6F
:105BE00056D006D8822B00F09680832B40F00F8190
:105BF00030E08C2B00F093808D2B40F00881A5E0E5
:105C0000C32B00F0C88011D8B52B00F0A38004D8B6
:105C1000993B012B00F2FB809AE0C12B00F0A5809C
:105C200000F2B380C02B40F0F28063E0CC2B00F098
:105C3000BF8005D8C72B4ED0C82B40F0E880B2E01B
:105C4000D52B00F0CC80D62B00F0D480D42B40F0A4
:105C5000DE80B8E0062106F029FD6F4B9C78022C0F
:105C600001D8610101E0E11E490141F00601C9B21C
:105C7000022C94BF0020012006F090FA664B674A80
:105C80009B78D318664A42F8240000221A71C1E0BA
:105C90000C2106F00BFD604B9C78022C01D86101B1
:105CA00001E0E11E490141F00C01C9B2022C94BF90
:105CB0000020012006F072FA574B5A4A9B78574948
:105CC00042F8240018465B1852F8201000221A717E
:105CD00006F018FD9EE0544B440108341C1904EBF7
:105CE000401203EB401002F14103181A02F0E4FEE7
:105CF00060708FE04C4B440108341C1904EB4012D7
:105D000003EB401002F14203181A02F0D5FEA07016
:105D100080E0142100E0042106F0C8FC7AE0424C47
:105D2000831C04EB40110B3101EB431304EB4010D7
:105D3000181A012202F09CFEA87804EB4014E17AC4
:105D4000C1F10801C9B204F0F5FE63E01A21E3E7EE
:105D50001821E1E74301344A03F1180151180230D8
:105D6000D31801EB4010C01A37E02F4C85000135E5
:105D7000821C04EBC50303EB421304EB4010181A1A
:105D800002F09AFE04F8350044E02749831C01EB39
:105D90004011580121E0244A831C02EB4010011DF0
:105DA00001EB431318E0204A430199181F311AE010
:105DB0001D4B821C03EB40110E3103EB401001EB35
:105DC0004213181A1FE0184B821C03EB40111431C8
:105DD00003EB401001EB4213181A042214E0124A9C
:105DE000430199181E310230D31801EB4010C01A3C
:105DF000012209E00C4A430199181C310230D318E2
:105E000001EB4010C01A022202F032FE02E003222F
:105E1000064B1A7038BD00BF640700202C0200201A
:105E2000A40D00208C090020A40E00208009002071
:105E30004A49F8B500230B6049494A4A0B604A4970
:105E400093750B60D360136113755375474A4FF018
:105E5000FF3142F82310464A0025D55401332F2B39
:105E6000F4D1FD262C46022C94BF0027012701D82F
:105E7000610100E0710141F00601C9B2384606F047
:105E800053F96101022C88BF71013A4B41F00C01BA
:105E9000E850C9B2384606F047F9374B01340136AD
:105EA000E8500435062CF6B2DDD1344D0024E97AF1
:105EB000E0B2C1F10801C9B2013404F03BFE203563
:105EC000062CF4D100232E4A002199500433B3F557
:105ED000806FF8D12B4B9B7EABB14FF4C3640DE0C8
:105EE000384631460422013502F0C2FD043704363B
:105EF000062DF5D11834B4F5FF6F04D0224E274695
:105F000036190025ECE71F4BDB7E5BB94FF4A76425
:105F10001E49204609190422043402F0A9FDB4F5F3
:105F2000C36FF5D1174B1B79012B03D0112B01D077
:105F3000212B01D1012200E000220A4B83F8D4205A
:105F4000104B5B7D23B1FEF767FB08B1012200E037
:105F50000022044B83F8D520F8BD00BF680900205B
:105F6000880900202C0200206C0700204402002039
:105F7000F40F0020A40D00208C090020A40E0020A6
:105F8000A409002004000020700100206C040020FF
:105F900008B50B4B5A7892B9997881B95A68DB7871
:105FA00043EA022240F2D2439A4208D140F2FF7003
:105FB00002F018FE02F0DAFE0120FEF7B1FB08BD88
:105FC0006407002010B5964A9378022B00F05F8199
:105FD000032B00F06581002B40F06E8253784D2B2F
:105FE00000F0B78023D8452B70D00ED8422B56D066
:105FF00005D8402B45D0412B40F05C8246E0432B36
:1060000053D0442B40F0568256E0482B7CD005D824
:10601000462B61D0472B40F04D826AE04B2B00F0BD
:10602000858000F28F80492B40F0448272E0542B2F
:1060300000F0E98011D8512B00F0B68006D84F2B24
:1060400000F08D80502B40F03582A6E0522B00F0FE
:10605000BD80532B40F02E82C2E0832B00F0FA80EB
:1060600006D8552B00F0E280572B40F02382EAE05F
:10607000852B00F0FF80C0F0F580FF2B40F01A82E6
:1060800001E1674B40F2FF70D97805E0644B654A47
:10609000DB7800201946137002F0A4FD0FE2D378DC
:1060A000604A194601205370F6E75D4B5D4ADB7884
:1060B000042019461371EFE7594B5A495A68DB78A7
:1060C0001C2043EA022341F81C3F0EE0D378554AD6
:1060D000194605205371DFE7514B52495A68DB7866
:1060E0000C2043EA022341F80C3F042202F0FCFC9E
:1060F000E5E14B4B4B4C5A68DB78214643EA0223DF
:1061000041F8083F082075E0D3784649262001F879
:10611000263F83E0424A434BD27812B142490122E2
:106120004A60DA753F4B1720D97DB5E73C4B3D4CB3
:10613000DB7803201946E37002F054FDE07802F0AA
:1061400035FFBCE1364B374ADB78022019469370A5
:10615000A2E7D378334A1946152053759CE7304B94
:10616000304CDB7819201946637602F03BFD607EE7
:1061700010F0010002D00020012100E0014606F0ED
:1061800023F9284B597E11F0020102D0012001466B
:1061900000E0012006F018F991E1214B214ADB785B
:1061A00016201946937577E71E4B1B7D13F0010FE0
:1061B00005D0D37813F0010F01D102F0D7FD184BB1
:1061C000184ADB7814201946137565E7144B1549F6
:1061D0005A68DB78202043EA022341F8203F84E715
:1061E0000F4B104C5A68DB78214643EA022341F8F2
:1061F000103F1020042202F077FC22696079A16828
:1062000003F036F95BE15168D37843EA0122012AB1
:1062100000F2528103491A2001F81A3F012265E772
:106220006407002004000020800900208E4B5A687B
:10623000DB7843EA0222012A00F23E818B491B20CF
:1062400001F81B3FEAE7884B8849DB78272001F8F3
:10625000273FE3E7D378516843EA0122844BC3F830
:10626000D8202CE1804B5A68DB7843EA0222814B2C
:106270001A6024E17C4B5A68DB7843EA02227C4BAB
:10628000C3F8DC201BE1784BDA787B4B16E1D3783E
:106290005168527843EA0121784B43F822100EE10D
:1062A00053782E2B00F20681DFE813F02F003C001C
:1062B0004900040104010401040104010401560021
:1062C0005E0066006E0076007E0004010401040199
:1062D0000401040104010401040104010401040196
:1062E0000401860089008C008F00920095009800C0
:1062F0009B009E00A100A400AD00B600BE00C60039
:10630000CE00D600EC00F400FC00574B5A68DB7856
:1063100043EA02225A4B1A6003F036FB544BC3F88F
:10632000E000CCE0504B5A68DB7843EA0222544B41
:106330005A6003F029FB4E4BC3F8E400BFE04A4B20
:106340005A68DB7843EA02224D4B9A6003F01CFB4B
:10635000474BC3F8E800B2E0434B5A68DB7843EAA6
:106360000222474BDA60AAE03F4B5A68DB7843EAE7
:106370000222434B1A61A2E03B4B5A68DB7843EAA6
:1063800002223F4B5A619AE0374B5A68DB7843EA66
:1063900002223B4B9A6192E0334B5A68DB7843EA26
:1063A0000222374BDA618AE02F4B5A68DB7843EAE6
:1063B0000222334B1A6282E02B4B00201CE02A4B56
:1063C000002022E0284B012016E0274B01201CE092
:1063D000254B022010E0244B022016E0224B032024
:1063E0000AE0214B032010E01F4B042004E01E4B69
:1063F00004200AE01C4B05205968DB7843EA0121A0
:1064000006F01AF95BE0184B05205968DB7843EA7F
:10641000012106F0D5F852E0134B5A68DB7843EAC5
:106420000222174B5A624AE00F4B5A68DB7843EA64
:106430000222134B9A6242E00B4B5A68DB7843EA24
:1064400002220F4BDA623AE0074B5A68DB7843EAE4
:1064500002220B4B1A6332E0034B5A68DB7843EAA3
:106460000222074B5A632AE0640700200400002040
:106470002C0200207C09002079090020A4090020BA
:10648000800F00200E4B5A68DB7843EA02220D4B46
:106490009A6314E00A4B5A68DB7843EA0222094BFC
:1064A000DA630CE0064B5A68DB7843EA0222054BBC
:1064B0001A6404E0032200E00422034B1A7010BDAA
:1064C00064070020800F00208009002010B5774B62
:1064D0009A78022A00F0BB80032A00F0BF80002ACD
:1064E00040F042815B78502B71D022D8462B55D09A
:1064F0000ED8422B48D005D8402B3CD0412B40F041
:10650000A4803FE0442B44D0694C6A4B44D83EE021
:106510004B2B50D006D8482B46D042D3492B40F0C5
:10652000948045E04D2B4CD048D34F2B40F08D80CC
:106530004AE0812B61D010D8542B50D006D8522B72
:106540004AD05B4C5B4B00F2C98043E0572B4CD0E8
:10655000802B4ED0552B78D144E0852B5DD004D8CC
:10656000832B54D0524C56D84FE0FE2B64D066D8C3
:10657000F02B6AD160E040F2FF7002F09DFA4C4BC4
:106580005860F4E04B4B58E04A4B5A7863E01B7973
:1065900087E0484BDA695EE05B7982E0454BDA6878
:1065A00059E0444B9A6856E0424B93F8262052E05B
:1065B000404BDA7D45E03F4BDA784CE03D4B9A7832
:1065C00049E03C4B5A7D46E03A4B5A7E43E0394B1A
:1065D0009A7D40E01B7D64E0364B1A6A3BE0354B08
:1065E0009A7E38E0334BDA7E35E0324B93F8272041
:1065F00031E0314B93F8D5202DE02F4B93F8D52087
:10660000042A14BF0022012225E02B4B63E02A4B11
:10661000D3F8D8201FE0294B3FE0274A284BD2F877
:10662000DC104B4303F540533933214923F000403C
:106630004860C2F8DC309AE0224B1A780BE0224B1B
:106640001A78003A18BF012205E003228DE05A783B
:106650001E4B53F82220164B5A6088E05B78144C8E
:106660002E2B7ED8DFE803F0181B1F7D7D7D7D7DFE
:106670007D36393C3F42457D7D7D7D7D7D7D7D7DC7
:106680007D7D7D484A4C50525456585A5C5E606538
:10669000686B6E7174777A000D4B1B6801E00C4BD0
:1066A0005B68636063E00A4B9B68FAE7640700205D
:1066B00080090020040000202C0200207C0900201A
:1066C0006D4EC641C80F002079090020A4090020A2
:1066D000800F00202F4BDB68E3E72E4B1B69E0E7C0
:1066E0002C4B5B69DDE72B4B9B69DAE7294BDB69B8
:1066F000D7E7284B1B6AD4E7002002E0002014E013
:10670000012005F093FD12E001200EE00220F8E7E1
:1067100002200AE00320F4E7032006E00420F0E76B
:10672000042002E00520ECE7052005F065FD60602F
:106730001DE0184B5B6AB4E7164B9B6AB1E7154B3B
:10674000DB6AAEE7134B1B6BABE7124B5B6BA8E747
:10675000104B9B6BA5E70F4BDB6BA2E70D4B1B6C44
:106760009FE70323237002E004220B4B1A700B4BAC
:106770001B786BB1084B0A495A680A4B0A601AB970
:106780001A6842F0080202E01A6822F008021A6051
:1067900010BD00BF800F0020800900207A09002072
:1067A000680900206C07002010B51C4CA078052853
:1067B00030D86378012B23D003D3022B184C26D179
:1067C00021E004F0EBFEA178164A0023994208D09C
:1067D000144C907F04EB411468B194F81EC08445BA
:1067E00009D111484FF0010C00F803C00F480CF11B
:1067F000FF3C03F800C001332032062BE6D10CE049
:1068000004F0D4FE09E004F0D9FE606005E0032343
:10681000237002E0024B04221A7010BD64070020AE
:1068200080090020A40E0020300200201C0E002051
:1068300037B5584B1A7DA2B957494868CA7842EA19
:106840000022B2F1FF3F04BF544A12680A214A43B2
:10685000C3F8EC2003F098F84E4B01221A75C3F8E8
:10686000F0004D4B5B78042B00F29280DFE803F0E0
:1068700003354659130003F087F8464BD3F8F01060
:10688000D3F8EC20411A0029B8BF494291427CD983
:1068900000221A757CE0404B3E4C987804F08EFE46
:1068A00030B93F4A2075136823F0100313606FE07E
:1068B000D4F8EC30002B67D003F066F8D4F8F02061
:1068C000D4F8EC30821A002AB8BF52429A425BD9FF
:1068D000334B00211A68217552E02F4CA078022812
:1068E00094BF0020012005F0F1FAA378022B88BFA5
:1068F000033B5B0001259D40054026E0264C7C21A2
:10690000A07801AA022894BF0020012005F05EFCB7
:10691000A3789DF80620022B88BF033B5B0002256D
:1069200011E01D4C7C21A07801AA022894BF002010
:10693000012005F04BFCA3789DF80620022B88BFB0
:10694000033B5B0001259D401540124C06D0144BC3
:1069500000211A68217522F0100213E0D4F8EC30FF
:1069600093B103F011F8D4F8F020D4F8EC30821A87
:10697000002AB8BF52429A4206D9094B25751A68B7
:1069800042F010021A6003E0024BDA68013ADA6062
:106990003EBD00BF2C0200206407002068090020D3
:1069A0006C07002008B5184B9A7812B1022A26D13C
:1069B00006E05868DB7843EA0020FDF7D9FD21E0C6
:1069C000587807280AD85A68DB7853EA022202D19D
:1069D000FDF720FD16E0FDF739FD13E0FF280CD18F
:1069E0005868DB7843EA0020B0F1FF3F0ABF074B4D
:1069F000C0B21878FDF746FD04E0032200E004224F
:106A0000034B1A7008BD00BF64070020680900200E
:106A10008009002010B51F4B9A78012A1CD003D39F
:106A2000022A1D4C21D11BE05878082802D8FDF716
:106A300023FE0EE00A2803D1174B00225A6016E00D
:106A40000B2802D1FDF700FE03E0FF280FD1FDF770
:106A500049FE114B58600AE0587802F0B1FFF8E7A0
:106A60005878FDF723FD606001E0042323700B4B91
:106A70001B786BB1084B0A495A680A4B0A601AB96D
:106A80001A6842F0080202E01A6822F008021A604E
:106A900010BD00BF64070020800900207A09002093
:106AA000680900206C07002010B5224B5A78812A13
:106AB0003FD19A78922A3CD19A79A32A39D15A792E
:106AC000B42A36D11A79C52A33D1DB78D62B30D106
:106AD000194B4FF400725A61A2F5A07203F580635E
:106AE0001A6103F08BFA02F04FFF044602F04CFFEC
:106AF000001B0028B8BF4042B0F57A7FF6DBFDF7F7
:106B000035FD07F079FB002008F0A6F800210B48BE
:106B100006F028FF094806F085FE094806F040FB0C
:106B200006F070FF4FF0804008F01AFE0020FDF7DD
:106B3000F7FD10BD64070020000801400800024076
:106B4000002401402DE9F047A84CA94DE078626887
:106B50002378642140EA0220222B86B029706B70D2
:106B6000686001F0128057D80F2B00F0898426D876
:106B7000072B00F0388410D8032B00F05F8106D873
:106B8000012B00F0A980022B41F06F82F5E0052B6C
:106B900000F0218400F223848FE10B2B00F033847A
:106BA00006D8092B00F0278400F2298400F01FBCCE
:106BB0000D2B00F05D8400F25F8400F03DBC192BCA
:106BC00000F0088613D8152B00F0048507D8132B86
:106BD00000F05A84142B41F0488200F0CDBC172BF2
:106BE00000F0D685834B00F2E78500F0C9BD1E2B6F
:106BF00000F02D8609D81B2B00F01F86C0F00886F8
:106C00001C2B41F0328200F01CBE202B00F0D786F6
:106C100000F2658700F079BE812B01F07A802ED8D2
:106C2000412B01F04A8015D8252B00F0F48707D8B6
:106C3000232B00F0B687242B41F0178200F0BDBF54
:106C4000272B01F01F80C0F0F187402B41F00D820F
:106C500001F030B8452B01F03C8006D8432B01F001
:106C6000328001F2338001F02BB8472B01F03780DE
:106C7000C1F03280802B41F0F88101F045B8882BBB
:106C800001F0D88012D8842B01F07D8007D8822BA8
:106C900001F05780832B41F0E88101F057B8862B33
:106CA00001F08B8001F2E68001F082B88C2B01F0BC
:106CB0002B8106D88A2B01F00E8101F2208101F090
:106CC00007B9F22B01F0C081FF2B01F0C0818D2BA1
:106CD00041F0CB8101F063B9A378052B48D8464E2B
:106CE000FD250024414B9B789C4208D0424A02EB90
:106CF00043139B7F002B33D0B27F9A4230D13F4A5F
:106D00004FF0010111553E4A0023A354022C3D4A85
:106D100094BF002701278CBF2946E1B2A35438460F
:106D2000022205F0D3F9022C01D8610100E06901CB
:106D300041F00601C9B2384640F2FF7205F056FB39
:106D4000022C01D8610100E06901284B41F00801E3
:106D50005A68DB78C9B2384643EA022205F046FB9E
:106D6000013401352036062CEDB2BBD101F080B9DB
:106D70001F4B04221A7001F07BB91C4B9B78052B2A
:106D800057D81D4EFD250024184B9B789C4208D0F7
:106D9000194A02EB43139B7F002B42D0B27F9A42E9
:106DA0003FD1164A4FF001011155154A0023A35453
:106DB000022C144A94BF002701278CBF2946E1B258
:106DC000A3543846022205F081F9022C01D8610152
:106DD00000E0690141F00601C9B2384640F2FF7295
:106DE00005F004FB022C0FD861010EE064070020BF
:106DF000800900202C020020A40E00203002002078
:106E00001C0E0020900E00206901954B41F00801F6
:106E10005A68DB78C9B243EA02223846524205F08A
:106E2000E5FA013401352036062CEDB2ACD101F083
:106E30001FB98C4B04221A7001F01AB9A378052BE4
:106E400037D8894EFD250024854B9B789C4207D07E
:106E5000854A02EB43139B7F1BB3B27F9A4220D13A
:106E6000824A0023A354824AE7B2A354384604F06E
:106E70009DFB022C94BF4FF000084FF001088CBF1F
:106E8000294639464046022205F020F9022C01D855
:106E9000790100E0690141F00801C9B2404605F0FE
:106EA000B9FA013401352036062CEDB2CCD101F00F
:106EB000DFB804232B7001F0DBB8694B9878052804
:106EC00003D95B78022B40F08182654B5B78032B02
:106ED00000F27782DFE813F004006700F4003F025D
:106EE000FDF7A8FE5E4B624A9878002313545F4A70
:106EF0000228135401D8410101E0C11E4901584C38
:106F0000022894BF00200120E3786268C9B243EAF6
:106F1000022205F0D1F9A078022801D8014601E04B
:106F2000C11EC9B2022894BF00200120002205F032
:106F3000CDF84B4B4C4E9B7806EB43139B7F002BBD
:106F400001F09680FD250024454B474A9B789C42E2
:106F500002EB43121FD0937FB27F9A421BD120468F
:106F6000FDF768FE022C94BF0027012701D86101BC
:106F700000E069013A4BC9B25A68DB78384643EA07
:106F8000022205F099F9022C8CBF2946E1B238465D
:106F9000002205F09BF8013401352036062CEDB2B5
:106FA000D2D101F065B8FDF745FE2D4B304A9878F7
:106FB000002313542D4A0228135401D8410101E043
:106FC000C11E490141F00201022894BF00200120A6
:106FD000C9B205F0A9F8224BDA785C689B7842EADE
:106FE00004240419022B01D8590101E0D91E4901DA
:106FF000022B94BF00200120C9B2224605F05CF9A3
:10700000174B9878022801D8014601E0C11EC9B289
:107010000022022894BF0020012005F057F8104BF1
:10702000114E9B780F4A06EB43139B7F5460002B55
:1070300001F01E80FD250024094B9878844237D04A
:10704000094BB27F03EB40139B7F9A4230D1FDF78F
:10705000F1FD022C94BF002701270BD861010AE043
:107060006407002080090020A40E00201C0E0020D0
:10707000900E0020690141F00201C9B2384605F0C6
:1070800053F88C4B022C5A68DB7843EA022301D870
:10709000610100E06901C218C9B2384605F00CF977
:1070A000022C8CBF2946E1B23846002205F00EF8CA
:1070B000013401352036062CEDB2BDD100F0D8BF29
:1070C00010F0C00539D1052832D87A4EF3787268AD
:1070D00043EA0223142B2BDC062202FB0303764A2D
:1070E00052F82340FDF7A6FDB078744B02281D54DA
:1070F000734B1D5401D8410101E0C11E4901022812
:1071000094BF00200120C9B2224605F0D5F8694B92
:107110009878022801D8014601E0C11EC9B20228B0
:1071200094BF00200120002204F0D0FF00F0A0BF97
:10713000644B04221A7000F09BBF402D40F0C480C5
:107140005C4B5F68DB7843EA0727142F00F3AD80C0
:1071500000231C4600930193029350FA03F10DF1B2
:10716000180C11F0010F0CEB040204D00134032CB5
:1071700002F80C3C02D00133062BEED1002621E0B0
:1071800003AB9D5D2846FDF755FD022D01D8690131
:1071900001E0E91E490141F00201022D94BF0020E7
:1071A0000120C9B204F0C0FF062303FB0755424B80
:1071B0006A4653F82530C31A002BB8BF5B4242F829
:1071C00026300136A642DBDB012C0ADD022C10D171
:1071D000009B01998B4207DD18469DF80D20FDF7B5
:1071E000BBFCFD2500242DE008469DF80C20194627
:1071F000F5E7032CF5D1009E019D029CAE420DDD0A
:10720000A64207DD304629469DF80D20FDF7A4FC77
:1072100030460CE031469DF80C200DE0A5429DF86B
:107220000C2008DD28463146FDF796FC284621460D
:107230009DF80E20D3E731462046FDF78DFC204611
:107240002946CAE71B4A937853FA04F111F0010F5B
:107250004FF0000122D05068D278022C42EA002080
:107260004FF0060202FB0040154A94BF002601269B
:10727000D154114A52F820201048C15401D861015C
:1072800000E06901C9B2304605F016F8022C8CBF47
:107290002946E1B23046002204F018FF01340135DE
:1072A000062CEDB2CED100F0E3BE064B04221A70DC
:1072B00000F0DEBE64070020700700201C0E0020D6
:1072C000900E002080090020802D40F0D1869F4B39
:1072D0005A68DB7843EA0223142B37DC7D3500241F
:1072E0009A4EB378234113F0010F28D0F3787268D7
:1072F000204643EA0222062303FB0242944B53F842
:107300002270FDF797FCB37892494FF00002CA54FF
:107310009149022CCA5494BF0026012601D861016C
:1073200000E06901C9B23A46304604F0C5FF022CBC
:107330008CBF2946E1B23046002204F0C7FE01347A
:107340000135062CEDB2CBD100F092BE834B042266
:107350001A7000F08DBE10F0800F40F089867B4DD2
:10736000EB786A6843EA0222062303FB0202784BA9
:1073700053F82240FDF75EFCA878764A00231354A8
:10738000754A0228135401D8410101E0C11E490188
:10739000022894BF00200120C9B2224604F08CFFCD
:1073A0006A4B9878022801D8014601E0C11EC9B293
:1073B000022894BF00200120002204F087FE00F084
:1073C00057BE664B03221A7000F052BE634B042274
:1073D0001A7000F04DBEFDF757FC00F049BEFDF7F6
:1073E000EDFF00F045BEFEF7EDFA00F041BEFEF7FE
:1073F000DBFB00F03DBEFEF7E5FD00F039BEFFF718
:1074000065F800F035BEA378022B11D16378372BD5
:107410000AD8534903F5A77001EB830180000422C9
:1074200001F062FB00F024BE03232B7000F020BEAD
:1074300004232B7000F01CBE444B9A78022A12D110
:107440005B78372B0AD8464903F5A77001EB830117
:107450008000023201F00CFB00F00ABE3F4B032219
:107460001A7000F005BE3D4B04221A7000F000BEF9
:10747000FFF79AF900F0FCBDFFF794FA00F0F8BDB1
:10748000FFF7C8FA00F0F4BD6278364B092A53D8EA
:10749000DFE802F0050D151D26313941494C2B4A14
:1074A00019685068D27842EA0022521843E0274A0D
:1074B00019685068D27842EA00228A1A3BE0234ACF
:1074C00019685068D27842EA00224A4333E01F4AE2
:1074D00019685068D27842EA002291FBF2F22AE061
:1074E0001A4819684468C27842EA042291FBF2F013
:1074F00002FB10121FE0154A19685068D27842EA60
:1075000000220A4017E0114A19685068D27842EA0E
:1075100000220A430FE00D4A19685068D27842EA07
:1075200000224A4007E01A68D24304E0074A516843
:10753000D27842EA01221A600A4A0B4B1268AAB9B1
:107540001A6842F008021A6000F092BD6407002039
:1075500070070020900E00201C0E002080090020E3
:10756000A4090020680900206C0700201A6822F096
:1075700008021A6000F07CBDA04BA14A5968DB7874
:10758000126843EA01239A4206DD9E4B1A6842F0D4
:10759000040222F003020CE09A4B05D11A6822F093
:1075A000060242F0010204E01A6822F0070242F0EB
:1075B00002021A60924A934B12682AB91A6842F082
:1075C00008021A6000F054BD1A6822F008021A601E
:1075D00000F04EBD63780C2B00F24A85DFE813F013
:1075E0000D001C002B003A0049005800670076008F
:1075F00085009400A300B200C100824B1B6813F009
:10760000080F00F035857D4B5A68DB7843EA02228B
:107610007D4BDA6000F02CBD7A4B1B6813F0080F2D
:1076200040F02685754B5A68DB7843EA0222764B98
:10763000DA6000F01DBD734B1B6813F0010F00F002
:1076400017856E4B5A68DB7843EA02226E4BDA608C
:1076500000F00EBD6B4B1B6813F0010F40F0088566
:10766000664B5A68DB7843EA0222674BDA6000F027
:10767000FFBC644B1B6813F0040F00F0F9845F4BF0
:107680005A68DB7843EA02225F4BDA6000F0F0BC14
:107690005C4B1B6813F0050F00F0EA84574B5A68E7
:1076A000DB7843EA0222584BDA6000F0E1BC554B2C
:1076B0001B6813F0020F00F0DB84504B5A68DB7834
:1076C00043EA0222504BDA6000F0D2BC4D4B1B68FB
:1076D00013F0030F00F0CC84484B5A68DB7843EA80
:1076E0000222494BDA6000F0C3BC464B1B6813F022
:1076F000100F00F0BD84414B5A68DB7843EA022248
:10770000414BDA6000F0B4BC3E4B1B6813F0200F15
:1077100000F0AE84394B5A68DB7843EA02223A4BD8
:10772000DA6000F0A5BC374B1B6813F0400F00F087
:107730009F84324B5A68DB7843EA0222324BDA608C
:1077400000F096BC2F4B1B6813F0800F00F0908464
:107750002A4B5A68DB7843EA02222B4BDA6000F0AE
:1077600087BC284B1B6813F4807F00F08184234B77
:107770005A68DB7843EA0222234BDA6000F078BCD7
:107780001E4A5168D27842EA0122DA6000F070BCE9
:107790001D4B1A69072A00F26B841849DC68486897
:1077A000C97841EA0020511C03EB8202C2F8F44080
:1077B000D860196100F05CBC1A69134B002A00F014
:1077C0005784013A03EB8201D1F8F4101A61D960B1
:1077D00000F04EBC63782E2B04D80C4A0121D15402
:1077E00000F046BCFF2B04D1074B01225A7500F074
:1077F0003FBC03232B7000F03BBC00BF640700209C
:10780000680900206C0700202C020020F40F0020E3
:107810008F4B5B782E2B04D88E4A0021D15400F078
:1078200027BCFF2B04D18C4B00225A7500F020BCE2
:107830008A4B03221A7000F01BBCFEF7F9FF00F020
:1078400017BC854B002283F8D52000F011BC63786B
:10785000142B57D8A278052A20D8062101FB032330
:107860007F4A804C917E44F82300002900F0008478
:10787000774A5378002B00F0FB83917803F1FF3CAB
:10788000062201F5C37002FB031302FB0C0204EB9A
:1078900083019000042201F027F9E9E3FF2A2DD1AA
:1078A000B3B94FF4C3640EE03846314604220135C3
:1078B00001F01AF904370436062DF5D11834B4F561
:1078C000FF6F00F0D583684E274636190025EBE799
:1078D00000245F4B06215B78624A581E01FB004082
:1078E00001FB034100F5C37002EB8101800004221B
:1078F000013401F0F9F8062CEBD1B9E3574B04221F
:107900001A70B5E303232B70B2E36378142B52D8BB
:107910004F4A9278052A1AD8062101FB03235149C0
:1079200051F82320514B4D491B784A60002B00F041
:107930009F834F494F4B0A6022B91A6842F00802F0
:107940001A6095E31A6822F008021A6090E3FF2A91
:107950002DD1B3B94FF4C3640EE03846314604224A
:10796000013501F085F804370436062DF5D11834B9
:10797000B4F5FF6F00F07C833B4E27463619002597
:10798000EBE70024324B06215B78364A581E01FB98
:10799000004001FB034100F5C37002EB8101800050
:1079A0000422013401F064F8062CEBD160E32B4B88
:1079B00004221A705CE3294B03221A7058E365789D
:1079C000142D00F28880224B9C7814F0800F38D060
:1079D000FD2500241E4B987850FA04F212F0010F96
:1079E00014D0022C5E7801D8610100E0690141F0F9
:1079F0000201C9B2022894BF0020012004F094FBC8
:107A0000062303FB0646174B43F82600144B9B7EC8
:107A10008BB10F4B5B7873B10621581E01FB004000
:107A200001FB03410F4A00F5C37002EB81018000A6
:107A3000042201F059F801340135062CEDB2C9D108
:107A400016E3052C43D8022C16D8610116E000BFBE
:107A500064070020F40F00202C0200208009002081
:107A60000400002070070020700100207A09002027
:107A7000680900206C070020E11E490141F0020165
:107A8000C9B2022C94BF0020012004F04DFB062354
:107A900003FB05449349944A897E42F82400002957
:107AA00000F0E68291484178002900F0E182807878
:107AB00001F1FF3E00F5C37C03FB010103FB0EC394
:107AC00002EB81019800042201F00EF8D0E2884B0D
:107AD00004221A70CCE2864B03221A70C8E2627844
:107AE000844B0A2A43D8DFE802F0060B11161C2447
:107AF0002A30363A3D0080491A6809688A1803E03E
:107B00007D4A196812688A1A1A6030E07A4A196840
:107B100012684A43F8E7784A1968126891FBF2F252
:107B2000F2E7754A1968126891FBF2F002FB101235
:107B3000EAE771491A68096801EA0202E4E76E4956
:107B40001A68096841EA0202DEE76B491A680968A7
:107B500081EA0202D8E7684B1A68D243D4E71A6870
:107B6000654BD1E7644A1868116810601960614A72
:107B7000624B126822B91A6842F008021A6077E272
:107B80001A6822F008021A6072E25A4B02F07F4231
:107B900019681B7842EA11226260E370FDF774F8FD
:107BA00066E2544B02F07F4219681B7842EA1122C8
:107BB0006260E370FEF706FA5AE24C4B5B78052BE5
:107BC00000F25682DFE803F003090F151B214B4B2F
:107BD0001A6802F00F021A604AE2484B1A6822F053
:107BE00010021A6044E2454B1A6822F020021A6023
:107BF0003EE2424B1A6822F040021A6038E23F4BE4
:107C00001A6822F080021A6032E23C4B1A6822F4B1
:107C100080721A602CE263782E2B04D8384A02EB6B
:107C20008303986124E203232B7021E2344BDFF8B5
:107C3000C4C0D3F81491334993F83021D3F818A174
:107C4000CCF80090DFF8B0C0D3F81C71D3F82081D5
:107C5000D3F82461D3F82851D3F82C41CCF800A0F4
:107C6000885CDFF898C0DF60CCF800801E75C3F830
:107C7000F050C3F8EC4008B101238B54204B002294
:107C80009A75F5E1A378052B10D8184A5278142A72
:107C900008D8062101FB0233164A1349126841F83D
:107CA0002320E5E1124B03221A70E1E1104B04227C
:107CB0001A70DDE102F000FADAE102F0FFF9D7E133
:107CC00002F0FEF9D4E102F0FDF9D1E102F0FCF995
:107CD000CEE102F0FBF9CBE102F0FAF9C8E102F0E3
:107CE000F9F9C5E1040000207007002064070020B6
:107CF0008009002068090020880900206C07002006
:107D00002C020020F40F0020924B002283F8D52093
:107D1000AEE1637813B1012B10D104E08D4B012249
:107D200083F8D520A4E1B0F5006F04D2894AD06071
:107D300082F8D5309CE104232B7099E103232B704A
:107D400096E1844B022283F8D52091E1814B0021FA
:107D5000997559757F4A4FF0FF3402F1180040F8C9
:107D600021407D480023435401312F29F2D17B4922
:107D700013750B607A4982F8D5300B607949D3606E
:107D80000B60136174E1784B1B7D13F0020F0CD173
:107D9000B0F5006F06D26F4B0422C3F8340183F8AC
:107DA000D52065E104232B7062E108232B705FE18D
:107DB000684B002283F8D5205AE16B4B01219A7859
:107DC0006A4BB0F5006F1970694B1A7028D2664B78
:107DD0001C7D0C4024D103A901F00CF8644B9DF8E4
:107DE0000C709DF80D609DF80E509DF812C09DF826
:107DF00011009DF810109DF80F201C725F709E708E
:107E0000DD7083F804C058719971DA710123584A02
:107E1000985C117A01334118082B1172F7D127E1D0
:107E20000123534A002199540133082BF9D11378C7
:107E300013721DE163788BB94B4A012091784D4A4A
:107E400014684A4A10704A4A11700133E21812F855
:107E5000011C474A082B9954F7D109E1012B40F046
:107E6000078114222A710332EA716FF02102AA718C
:107E70006B71FDE0404B5B78032B00F2F980DFE88B
:107E800003F002101D22334A3C4BD2F8341192F811
:107E9000D5C0107D0A0A197183F807C098715A710C
:107EA000E6E02C4A354BD16892F8D5C0107D0A0A1D
:107EB000197183F807C098715A71D9E0284B1A6874
:107EC0002E4B5A60D4E0274B1A682C4B5A60CFE0F7
:107ED000FEF75EF8CCE06278294B02B101221A70FD
:107EE000254B284AD8781B4B107093F83811264A36
:107EF00000231170254A1370254A1370B8E0154B02
:107F0000012283F83921B3E0667816B1012E43D1FE
:107F100011E0042240F2FB7005A900F0A9FDE3780E
:107F2000626843EA0222059B9A4202D101236B60F8
:107F30009EE06E609CE0A3782A2B06D140F2FB7095
:107F40001449042200F0D0FD92E00C4B03221A7079
:107F50008EE000BF2C020020F40F00206C070020F0
:107F60006809002088090020040000206C09002016
:107F70007009002000000020640700208009002014
:107F8000D80D0020280E0020D70F0020231000203D
:107F9000220E00206707002003232B7068E0364B79
:107FA0005B78032B4CD8DFE803F00C023C47324BE4
:107FB00032495A68DB78D1F83C1143EA022C00239D
:107FC0002BE02E4BD3F83C21092A0CD82A49501C0F
:107FD0004C68C97803EB820241EA0421C2F84011DF
:107FE000C3F83C0144E0264B09221A7040E052F8E5
:107FF0002340581C64450FD102EB8002013904E094
:1080000052F8040C013342F8080C04328B42F7D3C7
:108010001A4BC3F83C112BE003468B42194AE6D3B6
:1080200026E0164A0023C2F83C31164A0021D150FE
:108030000433282BF9D11BE0114B0A225A6017E0B8
:108040000F4B03221A7013E0FEF72EFD10E00A4BCF
:108050005A68DB7843EA022240F2D2439A4207D1BF
:10806000064B012283F8682102E0054B02221A70B8
:1080700006B0BDE8F08700BF640700202C02002096
:10808000800900206C03002073B5204B0246407825
:108090001F4D1870907800265870D078EC46987074
:1080A00010790C4698715079587192F806E095E86D
:1080B000030083F804E0D2798CE80300DA70154BF2
:1080C0001E70FEF73FFD144B1B7873B9637023706D
:1080D0002B78A3706B78E370EB792371AB796371C4
:1080E0006B79A3712B79E37108E0012B06D10B4B5F
:1080F0009B195B78A3550136082EF8D1044B6A46CC
:1081000092E8030083E803007CBD00BF6407002001
:10811000800900207A0900206C09002070090020E5
:10812000F7B5114D114C6F684FF0000C07F07F4709
:1081300047EA13276F600E4F6E4687F800C028701D
:108140006970AA7094E80300EB7086E80300FEF7FC
:10815000F9FC96E803006368227884E80300054987
:1081600018460A70FEBD00BF640700208009002089
:108170007A0900202C0200202DE9F04F984B9BB08B
:108180001B781BB9974B93F869316BB1964B1B78F1
:10819000062B09D00A2B07D00F2B05D01F2B03D09D
:1081A000904B002283F838218E4A92F83831591EBC
:1081B000C9B2012946D892F86A018C498C4ACC6828
:1081C0001278012B0CBF4FF0070C4FF0080C002366
:1081D0000E948DF834C08DF835008DF83630CAB95C
:1081E000844B8E681D7819795C7893F807C098796C
:1081F0005B798DF83C608DF83D508DF83E408DF8F0
:108200003FC08DF840008DF841308DF842108DF858
:1082100043200AE0012A08D1774A0133995C1AA861
:10822000C218082B02F82D1CF6D1744B1B78002BBA
:1082300040F0C2800DA801F039F8002840F0BC8061
:1082400000F00FBC032B25D192F8D440002C40F055
:108250008680674B1B7893B9644D664CA8786E781E
:10826000227863788619B618E279F618A379B618D9
:108270006279F6182379B618F618F6B219E0012BD0
:1082800040F09A805C4BE05C013400F0ABFE092CBE
:10829000F8D191E0042B27D1544D564CAB786E7831
:1082A00018469E1901360023012222706360F6B23F
:1082B000637000F097FE687800F094FE207800F07C
:1082C00091FE607800F08EFEE07900F08BFEA079E0
:1082D00000F088FE607900F085FE207900F082FED3
:1082E000304600F07FFE67E0072B3CD192F8D43097
:1082F000002B34D13E4A127822BB3C4A3D4B557884
:1083000096781C7893F801C0AF19D879E719997954
:1083100067445A79C7191B79CF19D719DF198DF816
:1083200058708DF850608DF851508DF852408DF88E
:1083300053C08DF854008DF855108DF856208DF8E7
:10834000573008E0012A06D12B4A995C14AAD1546F
:108350000133092BF8D1294B1B786BB328E0254852
:1083600004F03EFB28E0082B26D1204B0022597850
:108370009878224B45181C781E4B4FF0010C0135A4
:108380005A608DF852C08DF8532016468DF854204F
:108390008DF855208DF856208DF857208DF85850BF
:1083A0005A7083F800C08DF850008DF851101CB140
:1083B00014A8092101F0EEFC114B1B78002B00F0F2
:1083C0009980104A0D4B12780F4C013A062A00F2A0
:1083D0008C80DFE802F01B1B418A8A8A650000BF9F
:1083E000790900202C0200206407002004000020EE
:1083F0006C0900208009002070090020BC0D0020BD
:1084000023100020D70F0020220E0020AB4A94F842
:1084100000C0D068926819788DF82C206FF07F0228
:108420008DF82D200A3200238DF82E207D328DF814
:1084300032C08DF824208DF826300A908DF82F3028
:108440008DF830308DF831308DF8253000294CD141
:1084500009A800F02BFF48E0984D2278AB786E78A1
:1084600018469E190A36B61800F0BCFD687800F070
:10847000B9FD802000F0B6FD8A2000F0B3FD002099
:1084800000F0B0FD002000F0ADFD002000F0AAFDDE
:10849000F6B2207800F0A6FD304600F0A3FD24E0FF
:1084A00086482278417880786FF07F0500EB010CD8
:1084B0001C780CF10A0C002394448DF846500A35C0
:1084C0008DF847508DF84A308DF84CC08DF8440037
:1084D0008DF845108DF848308DF849308DF84B20D7
:1084E0001CB111A8092101F055FC754A0023137035
:1084F000744A1370744B754893F868110022027027
:1085000083F8692183F8382111B10120FCF708F9BB
:108510006D4B93F8392152B193F8D4200021D2F158
:10852000010238BF002283F8391183F8D420684B48
:108530001B78002B46D10DA800F096FE002841D0F4
:108540009DF83430062B3DD9624B5C4A9DF83C7057
:108550009DF83D609DF83E509DF83F409DF840E0FD
:108560009DF841C09DF84280116983F803801F7017
:108570005E709D709C7183F805E083F804C00E9BCB
:10858000514A9DF835008B4282F86A0102D10123DD
:1085900082F8693101F0F8F99DF834304FF00002AB
:1085A000072B4D4B484C18604C4B1A7001D10123DE
:1085B00000E0022384F83831434B93F8D5305A1E3B
:1085C000D2B2E8E0404C94F8D450002D40F08C80BA
:1085D0000DF1670000F0D4FC002800F0858000F069
:1085E000EBFC08B184F86B51374B9DF8670093F8AA
:1085F0006B114A1CD2B2C918092A81F86C0183F8A0
:108600006B2140F0F1802D4993F86C2148784FF0B0
:10861000000C904283F86BC107D091F82730002BF3
:1086200000F0E2809A4240F0DF80244B93F827303C
:10863000934203D1244B012283F8692100231A4677
:10864000214C04F5B671C95C01335218082BD2B223
:10865000F6D194F8743193422DD11E4B94F87111D8
:1086600094F8722194F8735194F86D6194F86EE166
:1086700094F86FC194F87001DD7059711A711E7011
:1086800083F801E083F802C0987101F07DF9144D80
:1086900094F8D5302860591E12480022C9B20270E1
:1086A0000320012984F8380184F86B2177D9052B40
:1086B00075D0013291E0042373E000BF0400002074
:1086C00023100020220E00202C0200206C09002024
:1086D000BC0D002064070020C40F0020BD0D002049
:1086E000CC0F0020D60F00209B4C94F8D43083B1DF
:1086F0009A4804F0BBF960B101F046F9984994F842
:10870000D530086097495A1E00200870D2B2032164
:108710003FE0914B93F8D440002C45D1924B1B780D
:10872000002B41D017A801F01FFB00283CD02346A6
:10873000224617A9C95C01335218082BD2B2F8D1CE
:108740009DF86410844C91422BD1844B9DF86110AC
:108750009DF862209DF85D609DF85EE09DF85FC029
:108760009DF860009DF8635059711A711E70DD709C
:1087700083F801E083F802C0987101F005F97849A7
:1087800094F8D530086077495A1E00200870D2B29C
:10879000072184F83811012A01D9052B1CD10022A8
:1087A0001BE084F838311FE06B4C94F8D530013B66
:1087B000DBB2012B18D8E368B3F5006F10D2FBF7DA
:1087C0002BFF68B1E368654918460133E36000F0A8
:1087D00011FB092384F838310122644B1A7003E03D
:1087E0005D4B002283F8D5205B4C94F8D530042BE8
:1087F00005D15A4E327812F0800F00F00581564BA9
:1088000093F838313BB1042B05D0082B03D0062B4D
:1088100001D0FEF797F9504C94F83831092B40F00D
:10882000CA8001F0B1F8D4F8E030514AC31A002BE5
:108830001268B8BF5B4293420AD94E4B1A78012A9C
:1088400001D101321A7001F09FF8434BC3F8E000E8
:1088500001F09AF8404BD3F8E420454B821A002AE5
:108860005B68B8BF52429A420AD9424B5A78012AF1
:1088700001D101325A7001F087F8374BC3F8E40098
:1088800001F082F8344BD3F8E820394B821A002AE1
:108890009B68B8BF52429A420AD9364B9A78012A4D
:1088A00001D101329A7001F06FF82B4BC3F8E80048
:1088B000294A537D002B7ED0937D002B7BD19C4693
:1088C0002D4BD2F8F0001B68D2F8EC1007932B4B1D
:1088D00004901B68D2F814810693294BD2F81871C2
:1088E0001B68D2F81C41059392F83031D2F8206110
:1088F0000293107DD368D2F82451D2F828B1D2F86F
:108900002C21039101926246DFF86890194619F80C
:1089100002A0BAF1020F18D11A4951F82210B1F190
:10892000FF3F0ED00546D0B202900398DDF810B09C
:108930000190059E069FDDF81C804FF0010C002081
:1089400004E0002109F802101946234601322F2ABB
:108950001AD01C460B46D7E72C02002064070020E3
:10896000CC0F0020D60F0020BC0D00207A0900207B
:10897000800F0020F40F00206809002088090020E3
:108980006C07002044020020374AD160C2F81C3135
:108990000199029B82F816C0C2F81481C2F81871BE
:1089A000C2F820611075C2F82451C2F828B1C2F88B
:1089B0002C1182F830312C4B93F83821092A06D13A
:1089C00093F8D510022902D1033183F8D510264B34
:1089D000D3F83C11002944D0092A42D193F8D5207C
:1089E000012A3ED1D868002308E054F8234001331F
:1089F000A04203D1052382F8D53032E01A4A8B42D7
:108A000002F5A074F1D32CE094F838314BB3042B69
:108A100027D0082B25D0062B23D0F3787168D4F803
:108A20003401124D43EA0123B0F5006F6A706B60A8
:108A300012D2314600F00EF93146D4F8340100F07C
:108A400031F930B1D4F834310133C4F8343165230D
:108A500000E007232B7004E007232B70002384F829
:108A6000D5301BB0BDE8F08F2C020020800900201B
:108A700070B5044600200E46154603210246FBF75A
:108A800037FF0020C4F307210246FBF731FF002027
:108A9000E1B20246FBF72CFF002407E0944214BF2A
:108AA00000220122FBF724FF3055013400206A1E0A
:108AB000AC420146F2D370BD10B50446002003213C
:108AC0000246FBF715FF0020C4F307210246FBF71F
:108AD0000FFF0020E1B20246FBF70AFF002001462B
:108AE0000122FBF705FF10BD2DE9F04104460F46BA
:108AF0001646002006210122FBF7FAFE0020052180
:108B00000246FBF7F5FE002001220146FBF7F0FECE
:108B100010F0020FF2D0002002210246FBF7E8FE1F
:108B20000020C4F307210246FBF7E2FE0020E1B279
:108B30000246FBF7DDFE002543E0013414F03F0858
:108B4000795D01D1012204E0721E954214BF00221A
:108B500001220020FBF7CCFEB8F1000F30D1731ECC
:108B60009D422DD2002005210246FBF7C1FE0020C8
:108B700001220146FBF7BCFE10F00100F2D10621F4
:108B80000122FBF7B5FE002005210246FBF7B0FEEF
:108B9000002001220146FBF7ABFE10F0020FF2D0DD
:108BA000002002210246FBF7A3FE0020C4F30721A8
:108BB0000246FBF79DFE0020E1B20246FBF798FE5D
:108BC0000135B542B9D3002005210246FBF790FEDE
:108BD000002001220146FBF78BFE10F0010FF2D1BD
:108BE000BDE8F08138B5012204460D46002006217B
:108BF000FBF77EFE002005210246FBF779FE0020F0
:108C000001220146FBF774FE10F0020FF2D00020A3
:108C100002210246FBF76CFE0020C4F30721024646
:108C2000FBF766FE0020E1B20246FBF761FE294633
:108C300000200122FBF75CFE002005210246FBF725
:108C400057FE002001220146FBF752FE10F0010FF3
:108C5000F2D138BD38B50725454305F500650C460A
:108C6000284609780135FFF7BDFF284661780135B0
:108C7000FFF7B8FF2846A1780135FFF7B3FF284674
:108C8000E1780135FFF7AEFF284621790135FFF77E
:108C9000A9FF28466179FFF7A5FF681CA179FFF7B6
:108CA000A1FF38BD2DE9F3470725454300200C46B9
:108CB00002460321FBF71CFE05F500650020C5F305
:108CC00007210246FBF714FE0020E9B20246FBF73B
:108CD0000FFE002001460246FBF70AFE82460020F6
:108CE00001460246FBF704FE80460020014602468C
:108CF000FBF7FEFD0746002001460246FBF7F8FDA4
:108D00008146002001460246FBF7F2FD06460020A0
:108D100001460246FBF7ECFD054600200122014614
:108D2000FBF7E6FD237853451DD1637843451AD1FF
:108D3000A378BB4217D1E37821798DF804608DF8D0
:108D400005508DF80600627943EA012343EA0243A5
:108D5000A079019A43EA006049EA0229814514BFDB
:108D60000020012000E00020BDE8FC8738B54FF46A
:108D70000064002006210122FBF7BAFD0020052136
:108D80000246FBF7B5FD002001220146FBF7B0FDCE
:108D900010F0020FF2D0002002210246FBF7A8FDDE
:108DA0000020C4F307210246FBF7A2FD0020E1B238
:108DB0000246FBF79DFD002500203F2D14BF002239
:108DC000012201460135FBF793FD402DF4D100202F
:108DD00005210246FBF78CFD002001220146FBF72E
:108DE00087FD10F0010FF2D14034B4F5804FC0D1AF
:108DF00038BD00BF38B50725454300200C46024664
:108E00000321FBF775FD05F500650020C5F307217B
:108E10000246FBF76DFD0020E9B20246FBF768FD54
:108E2000002001460246FBF763FD2070002001464A
:108E30000246FBF75DFD6070002001460246FBF72D
:108E400057FDA070002001460246FBF751FDE0707F
:108E5000002001460246FBF74BFD20710020014631
:108E60000246FBF745FD6071002001460122FBF739
:108E70003FFDA07138BD00BF37B500200521024677
:108E8000FBF736FD002001220146FBF731FD10F013
:108E90007104F2D100F078FD054605E0FFF70CFE05
:108EA000422814BF0024012400F06EFD431B002B58
:108EB000B8BF5B42B3F5FA6F40F2FF7002DA002CE4
:108EC000ECD000E01CB1294B1B78002B3CD040F2C9
:108ED000FF700021FFF786FEFFF748FF00202449BE
:108EE0004022FFF701FE40254FF480742046B42253
:108EF0002049FFF7F9FDB434284620221E49FFF728
:108F0000F3FD2035B4F5A76FF0D100230193E034D1
:108F100001AD2046042204342946FFF7E5FDB4F5EF
:108F2000FF6FF5D100230193A4F53074204604228D
:108F300004342946FFF7D8FDB4F5C36FF6D140F2EB
:108F4000FF704221FFF74EFE002009494022FFF743
:108F50008FFD402409492046091920222034FFF7BB
:108F600087FDB4F5807FF5D13EBD00BF440E0020E3
:108F70000400002078210108A8210108640E0020C7
:108F8000094B19685A68914201D100200BE01A6818
:108F9000D118097A013201701A601A68202A01D1A9
:108FA00000221A6001207047A4030020014B986240
:108FB000704700BFA4030020034B1A78104612B17B
:108FC00000221A70012070472C10002008B5FBF712
:108FD000CDFA034B00221A605A60FBF7C5FA08BDB0
:108FE000A403002038B50B4B8446DC6A1A6B0134AD
:108FF000202C08BF002494420AD0DD6A0648ED18F0
:1090000085F834C040F227710122DC6206F040FC92
:1090100038BD00BFA40300200044004038B5054619
:10902000002401E0FFF7DEFF2B5D01341846002B22
:10903000F8D138BD2A4910B50B8813F0200F1CD089
:10904000284BDB6813F0020F01D08B8815E0264B0C
:109050005A6818680132202A08BF0022824205D0CF
:109060005C688888E118C0B208725A601F4B0A22F7
:109070001A601D4B9A6A1E4B1A601948038813F038
:10908000800F1BD01A4B1A68C2B9174BDC6A196BD8
:109090008C420FD0134902240C61196BCC1894F840
:1090A00034C00131A0F804C01963196B202905D11F
:1090B0001A6303E040F2277106F0EAFB08480388D0
:1090C00013F0400F0BD040F2266106F0D9FC064B9E
:1090D0001A6BDB6A9A4202D1024B02225A6110BD1E
:1090E0000044004000080140A40300202810002094
:1090F0002410002030B5054687B0564806F010FD14
:109100004FF40030012105F059FB0420012105F046
:1091100047FB0420002105F05FFB0820002104F03C
:10912000C7FF06AC4FF0040324F8083D03234A4868
:1091300021468DF8123015338DF8133004F028FFD6
:10914000482345488DF8133021464FF00803ADF809
:10915000103004F01DFF684606F064FB0B2D25D887
:10916000DFE805F02406090C0F1215181B1E20223B
:109170004FF461531CE04FF4964319E04FF4E14380
:1091800016E04FF4164313E04FF4614310E04FF440
:1091900096330DE04FF4E1330AE04FF4613307E01A
:1091A0002E4B05E02E4B03E02E4B01E04FF41653FF
:1091B0000093009B06A95B0841F8183D25486946C5
:1091C00006F066FC26230024012505A88DF814303E
:1091D00007238DF815308DF816408DF8175005F0DF
:1091E00047F81C4840F2FF3106F026FC28212246B1
:1091F000184806F04DFB2A46164840F2277106F043
:1092000047FB2A46134840F2266106F041FB2A46F6
:10921000104840F2255106F03BFB22460D4840F233
:10922000244106F035FB22460A4840F6460106F086
:109230002FFB2246074840F66A1106F029FB602101
:109240002246044806F024FB2946024806F012FB99
:1092500007B030BD004400400008014090D003003A
:1092600020A1070040420F0030B50C4B0C4C844647
:1092700022681B689A4201D100200EE02368094A47
:109280005D1C02EB03130FCB8CE80F0025602368F5
:10929000082B01D100232360012030BDBC10002029
:1092A000301000203C100020704700BFF0B543781C
:1092B00087B00646426833B104238DF80C30002392
:1092C0000292019303E0019202938DF80C30B3787F
:1092D00003B102238DF80D30327800238DF80E2073
:1092E000F21801A8117AC2180133082BD172F7D1F4
:1092F00004F090F8042818D10D4D0E4B2C681B6813
:109300000134082C08BF00249C4201D100200DE04C
:1093100096E80F002F68084E06EB071C8CE80F003C
:10932000012001462C6004F067F8012007B0F0BD71
:109330003410002038100020C01000207FB52B4BC7
:109340002B4A19681268914204D10120002104F0CF
:1093500053F848E01968274A02EB0111487850B1E8
:109360001B6802EB0312536804228DF80C200022C4
:109370000192029307E01B68029002EB031253680C
:109380008DF80C000193194B1A681A4B03EB02136A
:109390009B781BB102238DF80D3001E08DF80D3064
:1093A000124B00221968134B0901CB5C8DF80E306B
:1093B0000E4B0DF1180C18680CEB020102EB001CAF
:1093C0000C4801326044007A082A01F8090CEFD1F8
:1093D0001A6801321A601A68082A01D100221A603C
:1093E00001A804F017F807B000BD00BF3810002036
:1093F00034100020C010002073B50220002103F0BB
:10940000FBFF1020002103F0F7FF01AC0021012039
:1094100003F0F2FF00250726142320468DF80430C0
:109420008DF805608DF806508DF8075004F020FF88
:10943000152320468DF804308DF805608DF8065010
:109440008DF8075004F014FF204613238DF80430E4
:109450008DF805608DF806508DF8075004F008FF70
:1094600004F0D4F929464FF0007005F0A7F97CBD4F
:109470002DE9F04101388AB00C46154607285BD823
:10948000DFE800F04C4034281C5A10040C238DF8FF
:109490001C3003238DF81D3000238DF81B304FF056
:1094A000020354E00C238DF81C3003238DF81D308B
:1094B00000238DF81B304FF004023AE00C238DF8A6
:1094C0001C3003238DF81D3000238DF81B304FF026
:1094D00010022EE00C238DF81C3003238DF81D3074
:1094E00000238DF81B304FF0140330E00C238DF86F
:1094F0001C3003238DF81D3000238DF81B304FF0F6
:10950000280216E00C238DF81C3003238DF81D3043
:1095100000238DF81B304FF0640318E00C238DF806
:109520001C3003238DF81D3000238DF81B304FF0C5
:10953000C802ADF81E200CE00C238DF81C3003236C
:109540008DF81D3000238DF81B304FF00803ADF867
:109550001E3004F05BF901214FF0007005F02EF988
:109560000120014605F01CF90820012105F018F939
:109570000820002105F030F901214FF4EA1004F031
:1095800097FD0AAE4FF4007226F8042D03233146EE
:109590008A488DF8263015338DF8273004F0F8FC12
:1095A0000423314685488DF827304FF48073002618
:1095B0000127ADF8243004F0EBFC05A88DF81A6003
:1095C0008DF814608DF815708DF816608DF81760A1
:1095D0008DF818708DF8197003F00CFEB4F5006F5B
:1095E00001A815DA4FF0FF326301ADF80830ADF88D
:1095F00010608DF812708DF804608DF805608DF89C
:109600000670ADF80A60ADF80C20ADF80E2013E03E
:109610004FF0FF338DF80670ADF810608DF81260D2
:109620008DF804608DF80560ADF80860ADF80A604B
:10963000ADF80C30ADF80E3003F04EFEDDB1B5F5EF
:10964000006F18DA002201236901ADF80A208DF8B5
:1096500005204FF0FF3201A8ADF808108DF8123048
:109660008DF804308DF80630ADF80C20ADF80E20E2
:10967000ADF8103016E000230122ADF80A308DF865
:1096800012308DF80530ADF808304FF0FF3301A8E7
:10969000ADF810208DF804208DF80620ADF80C30C0
:1096A000ADF80E3003F018FEE30043F004030DF1B3
:1096B00004080027012602226413ADF80A30404650
:1096C0004FF0FF338DF80420ADF808408DF8057099
:1096D0008DF80660ADF80C30ADF80E30ADF81070B6
:1096E0008DF8126003F0F8FDBD421ADDEB0043F087
:1096F00004036D130322ADF80A304FF0FF334046E8
:109700008DF804208DF80570ADF808508DF81260C2
:109710008DF80660ADF80C30ADF80E30ADF8106085
:1097200017E003238DF804304FF004024FF0FF33AD
:109730004046ADF80870ADF810608DF812708DF8E5
:1097400005708DF80660ADF80A20ADF80C30ADF864
:109750000E3008AF03F0C0FD0124072600251423B6
:1097600038468DF820308DF821608DF822508DF824
:10977000234004F07DFD152338468DF820308DF808
:1097800021608DF822508DF8234004F071FD1323E1
:1097900038468DF820308DF821608DF822508DF8F4
:1097A000234004F065FD0220214603F025FE2146FA
:1097B000102003F021FE0AB0BDE8F081000C01404A
:1097C00030B52A4D2A4B2C681B680134082C08BF81
:1097D00000249C4287B044D0012001A903F0F6FE8A
:1097E0009DF80C20234B042A09D12A68012103EBA0
:1097F000021251702A6803EB0213029A08E02A68E9
:10980000002103EB021251702A6803EB0213019A44
:109810005A609DF80D30154A022B164B04D1126880
:1098200003EB0213012203E0126803EB0213002290
:109830009A700E4B9DF80E101A680E4B1201D154FF
:1098400000230A4A06A9C81811680A4D03EB011142
:1098500010F8090C01334919082B0872F1D1146072
:1098600002E0012003F096FE07B030BDBC100020DE
:10987000301000203C10002030B52A4D2A4B2C68B7
:109880001B680134082C08BF00249C4287B044D0D8
:10989000002001A903F09AFE9DF80C20234B042A16
:1098A00009D12A68012103EB021251702A6803EBE7
:1098B0000213029A08E02A68002103EB0212517099
:1098C0002A6803EB0213019A5A609DF80D30154A7D
:1098D000022B164B04D1126803EB0213012203E0A2
:1098E000126803EB021300229A700E4B9DF80E10C3
:1098F0001A680E4B1201D15400230A4A06A9C8184F
:1099000011680A4D03EB011110F8090C01334919D4
:10991000082B0872F1D1146002E0002003F03AFE37
:1099200007B030BDBC100020301000203C100020DB
:10993000104B1A787AB159680F4A01315960116891
:109940000E4B013111601A6812B11A68013A1A609F
:109950000022084B00E001221A70094B1A683AB144
:109960001A68013A1A601B6813B9064B01221A7073
:10997000704700BFF80300207C090020241000205D
:10998000281000202C100020014B5868704700BFA1
:10999000F803002008B5042005F032F948F6A0408D
:1099A00005F03EF9012005F041F9044803210022A9
:1099B00004F02CFD012005F04FF908BD9AC3020008
:1099C000042807D0082809D008B100200DE0074B73
:1099D000188801E0054B588880B206E0034B988850
:1099E00040F26B1380B2584300137047000400200C
:1099F00070B592B011AE0024032531464FF002033A
:109A00004148ADF844308DF846508DF8474004F099
:109A1000BFFA4FF0110331463C48ADF844308DF8A1
:109A200046508DF8474004F0B3FA0120014604F097
:109A3000A9FE01214FF4007004F0B2FE344803F097
:109A4000F1FE344B32480193334B01A9029380233A
:109A50000693DB18079303F540730893A3F5787317
:109A6000099303F5FF530A930394049505940B940B
:109A700003F048FF2648012103F074FF01264FF44C
:109A8000602326480CA90E930C948DF834608DF851
:109A900035600F948DF8405003F0E0F91F480A211B
:109AA00032462B4603F05CFA1C480E2102222B465C
:109AB00003F056FA2B462A461848092103F050FABB
:109AC000224616484FF4FC6103F00CFA1348314665
:109AD00003F0FEF91148314603F0F0F90F4803F0A6
:109AE0000BFA0E4803F00EFA0028FAD10B4803F0E7
:109AF0000DFA0A4803F010FA0028FAD107480121AC
:109B000003F00EFA12B070BD000C014000100140CD
:109B1000080002404C2401400004002000240140C1
:109B2000014B03221A60704708040020044A054BC9
:109B3000927A0AB1052200E001221A60704700BF44
:109B40004C11002008040020704700BF014B002288
:109B50005A6070470804002008B5074B1A6892B293
:109B600042F008021A601A6892B242F004021A60C7
:109B7000FFF7D6FF08BD00BF405C004010B5064CA3
:109B80004FF6FB73226802EA03032360FFF7CEFF60
:109B90004FF40643236010BD405C0040072818BF07
:109BA0001F4B10B51E4C18BF18702378052B33D8E7
:109BB000DFE803F003060A0E1621FFF7DFFF2BE0B4
:109BC000FFF7DCFF042328E002236370013324E065
:109BD0006378013BDBB263706378FBB9042218E061
:109BE000104B1A6892B242F010021A6005232370DB
:109BF000DB18637012E06378013BDBB2637063785B
:109C000063B9084A4FF6EF73116801EA0303136062
:109C10000622034B1A7001E00623237010BD00BF1B
:109C2000B0110020405C0040034B9B7A13B1034B02
:109C300005221A60704700BF4C1100200804002064
:109C4000014B04221A60704708040020034B1A7A63
:109C5000202A01D100221A72704700BF0804002098
:109C6000704700BF212808B508D1124B1B681B782C
:109C700003F07F03212B1AD10F4B0EE0202816D1C1
:109C80000C4B0E4A1B681B7810720D4A03F07F03C1
:109C9000212B0CBF134600234BB1064A4FF00001A5
:109CA00012680020518293619847002000E0022052
:109CB00008BD00BFAC110020F99C0008080400207A
:109CC000159D0008074B1B681B7803F07F03212BB1
:109CD00005D1022801D0222801D1002000E0022075
:109CE000704700BFAC11002019B9012801D80846FF
:109CF00000E00220704700BF28B9044B4FF0080273
:109D00001B681A8200E00248704700BFAC110020B7
:109D10004400002028B9044B4FF008021B681A8247
:109D200000E00248704700BFAC1100204400002052
:109D30000B4B10B5DA6882B11B68052B01D00022ED
:109D40000BE0002303E00749595CC1540133044987
:109D5000CC68A342F7D30023CB60104610BD00BFF0
:109D600008040020B4110020084BDB68082B01D840
:109D700000200AE00023064A9A5CC2540133092BF2
:109D8000F9D1024B0022DA6001207047080400205C
:109D9000B411002010B5074C0B468AB2C021636095
:109DA00006F09AFC0120A18806F0A4FE012006F02E
:109DB0006FFD10BD0804002007B5142200238DF8A4
:109DC000042001A801228DF806308DF807208DF8B7
:109DD000053004F04DFA0EBD07B5142200238DF8AE
:109DE000042001A801228DF806308DF807208DF897
:109DF000053004F03DFA0EBD08B5064B1B68DB7854
:109E0000042B01D9002004E0034901EBC30106F053
:109E10000BF808BDAC1100204C00002008B5024929
:109E200006F002F808BD00BF6C00002008B502492A
:109E300005F0FAFF08BD00BF74000020334B10B5D9
:109E40001B686FF03F0200245A72DC729C7220463D
:109E500006F096FC20464FF4007106F0AFFC10218E
:109E6000204606F0C1FC4021204606F017FE802166
:109E7000204606F003FE204606F040FD244B204617
:109E800093F8641006F058FE204606F00FFD0120FE
:109E9000214606F093FC0120C02106F0EFFD0120D1
:109EA000202106F0A1FC0120214606F0B5FC02208D
:109EB0004FF4C06106F082FC02204FF4807106F07E
:109EC000DDFD0220214606F0A7FC0220202106F03D
:109ED0008BFC0320214606F071FC03204FF48871AF
:109EE00006F0DCFD0320402106F026FE03204FF49F
:109EF000405106F091FC2146032006F075FC2046F7
:109F000005F0A0FF034B01221A6010BDAC11002028
:109F1000440000200804002008B5174B174A1968B0
:109F200089B2118016491288098801EA020212F4E6
:109F3000806F05D04FF6FF321A60124BDB6B9847EB
:109F40000E4B1A880E4B1B8803EA020212F4007FA4
:109F500008D009490C4A4FF6FF500860117C0131C6
:109F6000C9B21174054A1288134013F4004F01D08E
:109F700006F0EEFA08BD00BF445C0040421100202C
:109F8000F4110020440000200804002010B5032034
:109F900006F002FE064C034602464FF4887105485F
:109FA000E36006F0B1FB032006F080FC10BD00BFAB
:109FB00008040020B411002008B528B105484FF46A
:109FC000806104F04BF804E002484FF4806104F033
:109FD00047F808BD0008014038B5064D01232B6045
:109FE000054B002420461C60FFF7E6FF03232B608F
:109FF000204638BD405C0040445C004008B5FFF797
:10A00000EBFF08BD08B50120FFF7D6FF064B012185
:10A01000196006494FF4E0520A8005490020186093
:10A0200008601A6008BD00BF405C0040F4110020C9
:10A03000445C0040084B10B51B6800249C72FFF77D
:10A04000E1FF064A4FF406431460043A1360044AE1
:10A050001460044A138010BDAC110020445C004021
:10A0600008040020F4110020002008B504F00EFBC5
:10A070004FF40000012104F0A1FB08BD07B5FFF774
:10A08000F3FFFFF7A9FE06F005FA0420012104F012
:10A0900087FB03238DF806300D338DF80730044815
:10A0A0004FF4806301A9ADF8043003F071FF0EBDD9
:10A0B00000080140704700BF704700BF704700BFF5
:10A0C000704700BF704700BF704700BF704700BFB8
:10A0D000704700BF704700BF10B5FFF755FC074C35
:10A0E0002368C31AB3F5FA7F07D9054BDA6882F4FF
:10A0F0000062DA60FFF748FC206010BDF811002014
:10A10000000C0140024B03EBC003D879704700BF3D
:10A110001C040020024B03EBC0035879704700BFBA
:10A120001C040020024B03EBC0039879704700BF6A
:10A130001C040020034B0B2202FB003393F8300079
:10A14000704700BF1C040020034B0B2202FB0033AE
:10A1500093F83100704700BF1C040020034B0B2212
:10A1600002FB003393F83300704700BF1C0400204B
:10A17000034B0B2202FB003393F83200704700BF01
:10A180001C040020034B0B2202FB003393F8340025
:10A19000704700BF1C040020034B0B2202FB00335E
:10A1A00093F83500704700BF1C040020034B0B22BE
:10A1B00002FB003393F83600704700BF1C040020F8
:10A1C000034B0B2202FB003393F83800704700BFAB
:10A1D0001C040020034B0B2202FB003393F83900D0
:10A1E000704700BF1C040020034B0B2202FB00330E
:10A1F00093F83A00704700BF1C040020034B05226F
:10A2000002FB003393F87400704700BF1C04002069
:10A21000034B052202FB003393F87500704700BF23
:10A220001C040020034B052202FB003393F8760048
:10A23000704700BF1C040020034B052202FB0033C3
:10A2400093F87700704700BF1C040020034B0522E1
:10A2500002FB003393F87800704700BF1C04002015
:10A26000034B032202FB003393F89400704700BFB6
:10A270001C040020034B032202FB003393F99500DA
:10A28000704700BF1C040020034B032202FB003375
:10A2900093F89600704700BF1C040020024B03EBAC
:10A2A000C00393F8A80070471C040020024B03EB86
:10A2B000C00393F8A90070471C040020024B03EB75
:10A2C000C00393F8AA0070471C040020024B03EB64
:10A2D000C00393F8AB0070471C040020024B03EB53
:10A2E000C00393F8AC0070471C040020024B03EB42
:10A2F000C00393F8AD0070471C040020024B03EB31
:10A30000C00393F8AE0070471C040020024B03EB1F
:10A31000C00393F8AF0070471C040020062821D822
:10A32000DFE800F004080C1014181C000E4BD3F8E2
:10A33000D83016E00C4BD3F8DC3012E00A4BD3F8DF
:10A34000E0300EE0084BD3F8E4300AE0064BD3F8D7
:10A35000E83006E0044BD3F8EC3002E0024B93F80F
:10A3600037300B60704700BF1C040020F8B5104B5D
:10A370000D461E5CC1F3074100223046FAF7B8FAD9
:10A380000C4C0702C5F3072100223046C4F8D870F0
:10A39000FAF7AEFA07433F023046E9B20122C4F8A9
:10A3A000D870FAF7A5FA07433F09C4F8D870F8BD8A
:10A3B000802201081C040020334B032202FB0033DF
:10A3C00010B5943393F901203F2A01DD3F225A70E2
:10A3D0002D4B032202FB0033943393F9012012F139
:10A3E0003F0FBCBF6FF03E025A70274B032202FBA7
:10A3F000003394339A781F2A01D91F229A70224B76
:10A40000032202FB00324FF44021C3F8F01092F80F
:10A410009420012A04BF4FF45022C3F8F0201A4BB5
:10A4200003EBC00292F8AF204AB9033202FB0032BC
:10A4300092F89520D3F8F01002F07F020CE003218F
:10A4400001FB003191F895C002F003020CF07C0C86
:10A45000D3F8F0104CEA02020B4C41EA0222C3F896
:10A46000F020032303FB004393F89620D4F8F03048
:10A4700042EA03031946C4F8F030FFF777FFD4F837
:10A48000F030C4F8E83010BD1C04002008B5044BBF
:10A49000032202FB003383F89610FFF78DFF08BDFF
:10A4A0001C04002008B5044B032202FB003383F890
:10A4B0009510FFF781FF08BD1C04002008B5044B70
:10A4C000032202FB003383F89410FFF775FF08BDE9
:10A4D0001C0400202A4B052210B502FB003393F820
:10A4E0007420012A02D9012283F87420244B05220A
:10A4F00002FB003374335A78032A01D903225A70BD
:10A500001F4B052202FB003374339A780F2A01D9BE
:10A510000F229A701A4B052202FB00337433DA784B
:10A52000032A01D90322DA70154B052202FB0033FE
:10A5300074331A790F2A01D90F221A71104C05238E
:10A5400003FB004303F1740292F804C093F8741003
:10A550004CF4202392F801C043EAC133917843EAD6
:10A560004C33D27843EA012343EA42131946C4F834
:10A57000F030FFF7FBFED4F8F030C4F8E43010BD43
:10A580001C04002008B5044B052202FB003383F8AD
:10A590007810FFF79FFF08BD1C04002008B5044B8E
:10A5A000052202FB003383F87710FFF793FF08BD05
:10A5B0001C04002008B5044B052202FB003383F87D
:10A5C0007610FFF787FF08BD1C04002008B5044B78
:10A5D000052202FB003383F87510FFF77BFF08BDEF
:10A5E0001C04002008B5044B052202FB003383F84D
:10A5F0007410FFF76FFF08BD1C0400205C4B0B229A
:10A6000010B502FB003393F83020032A02D903224D
:10A6100083F83020564B0B2202FB003330339A78FC
:10A62000032A01D903229A70514B0B2202FB0033FB
:10A6300030331A790F2A01D90F221A714C4B0B2291
:10A6400002FB003330335A79072A01D907225A71A5
:10A65000474B0B2202FB003330339A790F2A01D982
:10A660000F229A71424B0B2202FB003338335A7887
:10A670000F2A01D90F225A703D4B0B2202FB0033E7
:10A6800038339A780F2A01D90F229A70384B0B224F
:10A6900002FB003292F83010C90341F40024C3F8E1
:10A6A000F04092F831201AB141F40421C3F8F010BF
:10A6B0002F4B0B2101FB003191F8331029B1D3F856
:10A6C000F01041F40051C3F8F010294B92B90B324D
:10A6D00002FB0032303292F804C091784FEACC1C71
:10A6E000D3F8F0404CEAC12C51794CEA040242EA1A
:10A6F000011222E00B2202FB003292F838202AB12C
:10A70000D3F8F02042F48052C3F8F020184B0B210C
:10A7100001FB0031383191F801E0D3F8F02089785D
:10A7200042EACE1201F0070C42EA0C1211F0080FB7
:10A73000C3F8F02003D042F40062C3F8F0200C4BC1
:10A740000B2202FB00323032D17931B99179D3F842
:10A75000F02041EA0202C3F8F020054CD4F8F010D2
:10A76000FFF704FED4F8F030C4F8E03010BD00BFAD
:10A770001C04002008B5064B0B2202FB00333033CB
:10A78000DA791AB10022DA71FFF738FF08BD00BF8D
:10A790001C04002008B5064B0B2202FB00333033AB
:10A7A000DA791AB90132DA71FFF728FF08BD00BF64
:10A7B0001C04002008B5044B0B2202FB003383F875
:10A7C0003A10FFF71BFF08BD1C04002008B5044B1E
:10A7D0000B2202FB003383F83910FFF70FFF08BD8F
:10A7E0001C04002008B5044B0B2202FB003383F845
:10A7F0003810FFF703FF08BD1C04002008B5044B08
:10A800000B2202FB003383F83610FFF7F7FE08BD7A
:10A810001C04002008B5044B0B2202FB003383F814
:10A820003510FFF7EBFE08BD1C04002008B5044BF3
:10A830000B2202FB003383F83410FFF7DFFE08BD64
:10A840001C04002008B5044B0B2202FB003383F8E4
:10A850003210FFF7D3FE08BD1C04002008B5044BDE
:10A860000B2202FB003383F83310FFF7C7FE08BD4D
:10A870001C04002008B5044B0B2202FB003383F8B4
:10A880003110FFF7BBFE08BD1C04002008B5044BC7
:10A890000B2202FB003383F83010FFF7AFFE08BD38
:10A8A0001C04002010B52D4A4FF46021C2F8F010AE
:10A8B00002EBC00191F8AF10034619B14FF47021BB
:10A8C000C2F8F010254A02EBC30191F8A90091F8F3
:10A8D000A8C0D2F8F040000340EA8C302043C2F810
:10A8E000F00091F8AA10012904BF40F48060C2F87A
:10A8F000F0001A4A02EBC30090F8ABC0D2F8F01097
:10A9000041EA0C21C2F8F01090F8AC00012804BF15
:10A9100041F08001C2F8F010104A02EBC30191F837
:10A92000AD10012905D1D2F8F01041F04001C2F874
:10A93000F0100A4C184604EBC30393F8AE20D4F889
:10A94000F03043EA02131946C4F8F030FFF70EFD69
:10A95000D4F8F030C4F8EC3010BD00BF1C04002067
:10A9600008B5044B03EBC00383F8AE10FFF79AFF62
:10A9700008BD00BF1C04002070B5104B064603EB59
:10A98000C00393F8AE50032D02D00321FFF7E8FF78
:10A990003046FFF787FF094BD3F8D84014F4002F57
:10A9A0001CBF6FEA04346FEA1434032D03D0304621
:10A9B0002946FFF7D5FF204670BD00BF1C040020CC
:10A9C00008B5044B03EBC00383F8AD10FFF76AFF33
:10A9D00008BD00BF1C04002008B5044B03EBC003F6
:10A9E00083F8AC10FFF75EFF08BD00BF1C04002019
:10A9F00008B5044B03EBC00383F8AB10FFF752FF1D
:10AA000008BD00BF1C04002008B5044B03EBC003C5
:10AA100083F8AA10FFF746FF08BD00BF1C04002002
:10AA200008B5044B03EBC00383F8A910FFF73AFF06
:10AA300008BD00BF1C04002008B5044B03EBC00395
:10AA400083F8A810FFF72EFF08BD00BF1C040020EC
:10AA5000064B10B503EBC003044683F8AF10FFF7B5
:10AA600021FF2046FFF7A8FC10BD00BF1C040020FA
:10AA700010B5194A0021C2F8F01002EBC001497963
:10AA8000034619B14FF40071C2F8F010124A02EBFC
:10AA9000C301897929B1D2F8F01041F48071C2F86C
:10AAA000F0100D4A02EBC302D1790F2901D90F2111
:10AAB000D171094C184604EBC303DA79D4F8F030AD
:10AAC00042EA03031946C4F8F030FFF74FFCD4F80C
:10AAD000F030C4F8DC3010BD1C04002070B5084D07
:10AAE0009DF810E09DF8146005EBC00426716270BB
:10AAF000A37084F803E005F83010FFF7B9FF70BDCC
:10AB00001C04002008B5034B03EBC0039971FFF749
:10AB1000AFFF08BD1C04002008B5054B03EBC003C4
:10AB2000597109B10422DA71FFF7A2FF08BD00BF15
:10AB30001C04002008B5054B042903EBC003D971A0
:10AB400001D000225A71FFF793FF08BD1C040020BA
:10AB50002DE9F047374D0446401990F8F4000E46B1
:10AB600017469846DDF82090DDF824A004281FD869
:10AB7000DFE800F003090F151B002046FFF73EFD3C
:10AB80006519012316E02046FFF78CFE65190223A4
:10AB900010E02046FFF79EFC651903230AE02046DB
:10ABA000FFF70AFC6519042304E02046FFF760FF65
:10ABB0006519002385F8F4301E4B03EBC40494F8A8
:10ABC000AE20012A0FD002D3022A28D114E01EB1F0
:10ABD000D3F8D8309B0C33700FB3164BD3F8D83062
:10ABE0009B0A3B701BE0B8F1000F18D0D3F8D830A7
:10ABF0009B0AC8F8003012E0B8F1000F05D0D3F876
:10AC0000D830DB0B5B01C8F80030B9F1000F06D07B
:10AC1000084BD3F8D830C3F3842389F80030BAF155
:10AC2000000F04D0034BD3F8D8308AF80030BDE8C9
:10AC3000F08700BF1C04002000202F4A2DE9F84FA8
:10AC4000844686462D4B2E4C03F1940B03F1A80A43
:10AC50004FF001090BF80C900AEB0E01251803EBDD
:10AC60000E08032400230527E3444FF002068BF867
:10AC700002708BF8017081F80590CB714C708B706D
:10AC8000CB700B718E711E490CF1030C0AF80E404B
:10AC90000B542B716B70AB70EB70C01988F80730D8
:10ACA00088F8053088F8063016719771947216701E
:10ACB0005370D37093705471D371137253720B32FB
:10ACC000BCF1120F0EF1080EBCD11D46ECB22046AD
:10ACD000FFF700FC2046FFF76FFB2046FFF7E2FD81
:10ACE0002046FFF7C5FE01352046FFF787FC062DFD
:10ACF000ECD1BDE8F88F00BF4C0400201C040020FC
:10AD00009004002038B5074D0024074B0022E25480
:10AD1000E0B2A97A0134F9F70BFD2035062CF4D105
:10AD200038BD00BFA40E0020D80F0020F0B5834B23
:10AD300085B01A784AB96FF00042012119709A6102
:10AD40005A609A60DA601A615A617C4B1C7F5CB968
:10AD5000E0B2F9F791FC794B03F120021055013470
:10AD6000082CF5D101221A7727240025E8B2F9F73B
:10AD700083FC734A535D83421BD0724B05F108017B
:10AD800003EB81035B685055022B05D0032B0AD0DF
:10AD9000012B0ED168B106E058B96B4A115D01294B
:10ADA00007D1135505E0684B1A5D012A01D1013224
:10ADB0001A5501350134082DD8D1644DEB69B3B172
:10ADC000634B1C789CB9FEF7DFFD624AEB691268A1
:10ADD000821A002AB8BF52429A4208D9204601344A
:10ADE00001F036FB062CF9D1594B01221A70574D50
:10ADF0002B6AB3B1584B1C789CB9FEF7C5FD574A76
:10AE00002B6A1268821A002AB8BF52429A4208D9A5
:10AE10002046013401F01CFB062CF9D14E4B0122D7
:10AE20001A70464C4E4A94F82800830002EBC30285
:10AE3000127B62B14B4A4C4D4C4C0021D3182D185B
:10AE400024180A4600950194FFF782FE97E3FEF767
:10AE50009BFDE36AC31A002BB8BF5B420A2B40F389
:10AE60008E8394F82800022801D8410101E0C11E18
:10AE7000490141F00A01C9B2022894BF0020012013
:10AE800001F08CF92D4D044695F8280001F018FBCF
:10AE900095F828304FF00C0C022B98BF194694BF40
:10AEA0000022012288BFD91E242050430CFB01013F
:10AEB0002F480918097A59B1022B94BF1946D91E97
:10AEC000242042430C2000FB012129480D580BE0AF
:10AED000022B94BF1946D91E242042430C2000FBAC
:10AEE0000121234809184D68224AD25C032A00F246
:10AEF0001181DFE802F0029E1E75002C00F00A812D
:10AF0000174A0E4E02EB4311C97F1A4D31B1184654
:10AF1000F9F70EFC96F82830032208E002EB431202
:10AF20001846517AF9F704FC96F828300222EA54C0
:10AF3000F0E07CBB022B1FD859011FE01805002050
:10AF400038050020800F0020F40F002004000020AE
:10AF5000D60F0020CC0F0020BD0D0020C40F002014
:10AF6000A40E00202C0E0020DC0D0020980E0020E6
:10AF7000480E0020D80F0020D91E490141F00801D9
:10AF8000C9B2022B94BF0020012001F007F9064648
:10AF9000002861D0534E544B96F8280003EB401321
:10AFA000D97F002900F0AE80002D84EAE472B8BF9A
:10AFB0006D42A2EBE472AA4202D0002C40F09B80CA
:10AFC0004A4B53F830108A4280F09C8003EBC00358
:10AFD0001979F9F7ADFB434B012193F828308FE045
:10AFE000002D84EAE471B8BF6D42A1EBE471A9427F
:10AFF00002D0002C40F086803C4A3A4E52F8330092
:10B000003B4D814209D202EBC30218461179F9F790
:10B010008FFB96F82830012209E0334A184602EBEC
:10B020004313597AF9F784FB96F828300222EA5440
:10B0300068E0002C32D1022B01D8590101E0D91E61
:10B04000490141F00801C9B2022B94BF0020012040
:10B0500001F0A4F8064608BBFEF796FC214D224AF3
:10B0600095F828304FF00A0E02EB4311B1F81CC0DE
:10B0700099004F197F680EFB0CFCC71B002FB8BF4F
:10B080007F42674546DD02EBC1021846917AF9F727
:10B090004FFB95F82830164AD6543BE0114E124A21
:10B0A00096F8283002EB4312D17F59B3002D84EA81
:10B0B000E472B8BF6D42A2EBE472AA4200D0CCB9F0
:10B0C0000A4951F833108A421CD3074A184602EB4A
:10B0D0004313597AF9F72CFB024B022193F82830DD
:10B0E0000EE000BF18050020A40E0020E40D002093
:10B0F000D80F00201846F9F71BFB96F828300321DB
:10B10000A44AD154A44D95F82860FEF73DFC05EB08
:10B1100086056860A04DA14F95F82830A04E1846CE
:10B12000F618FF189F4B002103EB80030A46019697
:10B1300000979D4EFFF70CFD95F8280006EB401395
:10B140009B69002B38D0F9F7E5F9002834D095F841
:10B15000280084EAE47206EB40139B69A2EBE472D8
:10B160009A4229D901F074F995F828308F4906EBF5
:10B170004312927F0120C854A2B10025864B8A4A0F
:10B1800093F82810B37F02EB4112927F20369A4247
:10B1900005D1284601F05CF9E8B200F007FA013564
:10B1A000062DEBD17C4B824A93F828300F33D15CCB
:10B1B000012901D10131D154774D95F82830022B66
:10B1C00025D8002000F082FE95F8303010F0010FF5
:10B1D00003F0F80385F830301CBF43F0010385F815
:10B1E000303010F0040F8DF80C0006D06A4B93F845
:10B1F000302042F0020283F8302010F0100F06D009
:10B20000654B93F8302042F0040283F83020624D01
:10B2100095F82830033BDBB2022B25D8012000F043
:10B2200055FE95F8303010F0010F03F0C70385F894
:10B2300030301CBF43F0080385F8303010F0040FA5
:10B240008DF80D0006D0544B93F8302042F01002D8
:10B2500083F8302010F0100F06D04F4B93F83020B9
:10B2600042F0200283F83020524A137853B14A4901
:10B2700091F830100B4205D14F49504809780370BE
:10B2800001B911704D4B1B784BB1434A92F83020F5
:10B2900003EA02029A4202D1494B01221A703E4B44
:10B2A00093F8302012F0010F0AD093F8313013F0E8
:10B2B000010F05D13E4BDA78012A01D10132DA7053
:10B2C000354B93F8302012F0020F0AD093F831304A
:10B2D00013F0020F05D1364B1A79012A01D1013240
:10B2E0001A712D4B93F8302012F0040F0AD093F806
:10B2F000313013F0040F05D12D4B5A79012A01D1B9
:10B3000001325A71244B93F8302012F0080F0AD002
:10B3100093F8313013F0080F05D1254B9A79012AA3
:10B3200001D101329A711C4B93F8302012F0100FAA
:10B330000AD093F8313013F0100F05D11C4BDA7995
:10B34000012A01D10132DA71134B93F8302012F047
:10B35000200F0AD093F8313013F0200F05D1144B91
:10B360001A7A012A01D101321A720B4B032293F887
:10B3700028000DF1100CB0FBF2F2624412F9042C1B
:10B3800093F83010002A83F8311076DA022819D8A1
:10B39000410119E0D80F002018050020DC0D002025
:10B3A000980E00202C0E0020A40E0020900E0020ED
:10B3B000F40F0020280E0020D80D0020220E0020BF
:10B3C00023100020C11E490141F01601022894BF3C
:10B3D00000200120C9B202AA00F0F8FE9DF80A3050
:10B3E00013F0400F0AD0674A674992F828205200AC
:10B3F0001B32885C012801D10130885413F0800F82
:10B400000BD06049604A91F828100E3112F81100F3
:10B41000012802D1013002F8110013F0100F0AD0F8
:10B42000584A594992F8282052001B32885C01285A
:10B4300001D10130885413F0200F0BD0514A524BE8
:10B4400092F828200E3213F81210012902D101318E
:10B4500003F812104B4B93F82800022801D8410141
:10B4600001E0C11E490141F01601C9B2022894BF92
:10B470000020012002AA01F08FF894B9414B93F803
:10B480002800022801D8410101E0C11E490141F014
:10B490000801C9B2022894BF0020012000F07EFEFE
:10B4A00028B1384D394B95F828609B5D5BB3354B1F
:10B4B000374A93F8283002EB4312D28912B9334A43
:10B4C000D35C2BB3FEF760FA2E4D314995F8283046
:10B4D0004FF00A0C9A0001EBC201C9895219526B54
:10B4E0000CFB01F1821A002AB8BF52428A420FDDDA
:10B4F000284EF25C62B91846FFF74CF995F82830EF
:10B500000122F25404E0FEF73FFA05EB860568637A
:10B510001C4E214D96F82800002C55F83030B8BF4D
:10B5200064429C420BD2FEF791FE96F8283005EB60
:10B53000C3056A7982420ED11846002109E0FEF760
:10B5400085FE96F8283005EBC3056979884202D05C
:10B550001846FFF717F80B4C94F8280000F034F861
:10B5600094F828300133DBB2052B84F8283002D957
:10B57000002384F82830FEF707FA024BD86205B0A2
:10B58000F0BD00BF18050020F40F0020E40F0020DC
:10B59000A40E0020EC0F0020E40D0020024B1A5CEA
:10B5A0000AB901321A54704764050020024B1A5C34
:10B5B0000AB10F221A54704764050020014B185C31
:10B5C000704700BF6405002002282DE9F7450446B6
:10B5D00094BF0025012501D8410101E0C11E4901A8
:10B5E00041F07C01C9B2284601AA00F0EFFD022C0F
:10B5F00005D863004FF0020808FA03F806E0A4F14A
:10B6000003084FEA4808022303FA08F89DF80630B9
:10B610005FFA88F8022C08EA030805D862004FF0A8
:10B62000010A0AFA02FA06E0A4F1030A4FEA4A0AFA
:10B63000012202FA0AFA5FFA8AFA0AEA030A984B26
:10B64000022C03EB44131E7A274606F07F0601D82E
:10B65000601C00E0A01CC0B2F9F70EF8904B03EBA1
:10B66000441393F90830002B03DAD0F1010038BFFE
:10B670000020731E072B00F2F483DFE813F00800AC
:10B68000080008000800DF01DF01DF01DF01854B52
:10B690001B5D013B0E2B00F2E483DFE813F00F008B
:10B6A00035025D007D0274007D009900BD00190126
:10B6B00076017C01E203AB01BB01B403022C01D88B
:10B6C000610101E0E11E490141F0140101AAC9B282
:10B6D000284600F07BFD734B9DF8052003EB8403A7
:10B6E000022C9A6001D8610101E0E11E490141F09C
:10B6F0000601C9B2284600F051FD6A4B022C03EB4B
:10B700008403186201D8214601E0E11EC9B2022279
:10B71000284600F0DBFC022C01D8610101E0E11EAB
:10B72000490141F00601C9B2284640F2FF7200F01B
:10B730005DFE022C01D9033CE4B2023E03222846FE
:10B740002146F6B200F094FC012E564B01D802229D
:10B7500000E00422DA5584E3BAF1000F00F081839F
:10B76000022C01D8610101E0E11E490141F0020112
:10B77000C9B2284600F0D8FC4A4B04221A554A4B5D
:10B7800043F824006DE3B8F1000F00F06A8320460F
:10B7900000F05EFE062255E3022C01D8214601E0AE
:10B7A000E11EC9B20322284600F062FC022C01D837
:10B7B000610101E0E11E4901394B41F0080103EB51
:10B7C0004413C9B228465A6800F010FE072239E334
:10B7D000B8F1000F40F04583022C01D8610101E06F
:10B7E000E11E490141F008010022C9B2284600F0DB
:10B7F000FDFD022C01D8610101E0E11E4901284B49
:10B8000041F0080103EB44135A68C9B2524228467A
:10B8100000F0ECFD082215E3B8F1000F00F02183E1
:10B82000022C01D8610101E0E11E490141F0020151
:10B83000C9B2284600F078FC022C064601D8610106
:10B8400001E0E11E490141F008010022C9B2284689
:10B8500000F0CCFD144B53F82420921B022C43F82B
:10B86000242001D8214601E0E11EC9B20322284666
:10B8700000F0FEFB022C01D8610101E0E11E49014C
:10B88000074B4FEA4418434441F00601C9B25A68D5
:10B89000284600F0ABFD022C08D85FFA88F108E0DA
:10B8A000A40E002064050020C00D0020E11E490107
:10B8B000C9B23246284600F0FFFC022C01D9033CF5
:10B8C000E4B200222846214600F000FC092247E2AB
:10B8D000284600F0FBFA022C01D8630001E0E31EC9
:10B8E0005B00012212FA03F3034200F0BA82022C39
:10B8F00001D8610101E0E11E490141F00201C9B234
:10B90000284600F011FCA04B022C43F8240001D87B
:10B91000610101E0E11E490141F008010022C9B2C4
:10B92000284600F063FD022C01D8214601E0E11E0B
:10B93000C9B20222284600F0C9FB022C01D86101DD
:10B9400001E0E11E490141F002010022C9B228468E
:10B9500000F0B2FC022C01D8610101E0E11E4901B6
:10B96000033E0022C9B22846F6B200F0A5FC012E23
:10B9700000F26782022C01D8214601E0E11EC9B223
:10B980002846022200F0A2FB83E1B8F1000F00F08C
:10B9900068820B2256E2B8F1000F40F06282022C5E
:10B9A00001D8610101E0E11E490141F00201C9B283
:10B9B000284600F0B9FB022C064601D8610101E0DF
:10B9C000E11E490141F008010022C9B2284600F0F9
:10B9D0000DFD022C01D8610101E0E11E49010222A6
:10B9E000C9B296FBF2F2284600F066FC022C00F287
:10B9F000AF81AFE1284600F069FA022C01D863005C
:10BA000001E0E31E5B00012212FA03F3034200F09F
:10BA1000288216E2022C01D8610101E0E11E4901F1
:10BA20005A4B41F0060103EB8403C9B21A6A284657
:10BA300000F0DCFC022C00F2088208E2534B1B5D94
:10BA4000013B0E2B00F20D8201A252F823F000BF41
:10BA50008DBA000805BB000867BB000895BB00084D
:10BA6000F9BB000863BE00081DBC000863BE0008E7
:10BA700063BE0008B9BC0008E5BC000867BC00084C
:10BA800065BD000835BA000807BE0008022C01D8C1
:10BA9000610101E0E11E490141F0140101AAC9B2AE
:10BAA000284600F093FB394B9DF8052003EB8403F7
:10BAB000022C9A6001D8214601E0E11EC9B202229F
:10BAC000284600F003FB022C01D8610101E0E11ED1
:10BAD000490141F00601C9B2284640F2FF7200F068
:10BAE00085FC022C01D9033CE4B2032228462146FE
:10BAF00000F0BEFA062E01D0082E01D102222FE15D
:10BB000004222DE1062E11D1022C01D8214601E09C
:10BB1000E11EC9B21D4B284603EB84039A6802F06C
:10BB20000402002A14BF0522012209E0082E09D1CF
:10BB3000022C01D8214601E0E11EC9B228460322A9
:10BB400000F096FA022C01D8610101E0E11E4901E2
:10BB50000F4B41F008016201D258C9B2284600F0EB
:10BB600045FC03226EE1731FDBB2012B07D8BAF14B
:10BB7000000F04D0062E054B4AD1042263E10028B1
:10BB800000F06F810C225DE1680F00206405002049
:10BB9000A40E0020052E11D1022C01D8214601E06F
:10BBA000E11EC9B29A4B284603EB84039A6802F05F
:10BBB0000402002A14BF0622022209E0072E09D13E
:10BBC000022C01D8214601E0E11EC9B22846032219
:10BBD00000F04EFA022C01D8610101E0E11E49019A
:10BBE0008C4B6201D25841F008015242C9B228463A
:10BBF00000F0FCFB052225E1731FDBB2012B09D805
:10BC0000B8F1000F06D0052E814B01D102221AE1B6
:10BC10000F2218E1002800F02481D7E5002840F029
:10BC20002081022C01D8214601E0E11EC9B2784BE7
:10BC3000284603EB84039A6802F00402002A14BF2A
:10BC40000522012200F014FA022C01D8610101E062
:10BC5000E11E49016F4B41F0080103EB4413C9B2E7
:10BC600028465A6824E0002840F0FB80022C01D8C6
:10BC7000214601E0E11EC9B2654B284603EB84036F
:10BC80009A6802F00402002A14BF0622022200F081
:10BC9000EFF9022C01D8610101E0E11E49015D4B81
:10BCA00041F0080103EB44135A68C9B228465242D6
:10BCB00000F09CFB0A22C5E0002800F0D280022C94
:10BCC00001D8610101E0E11E490141F00201C9B260
:10BCD000284600F029FA4E4B0B2103EB840219553C
:10BCE0009063BEE0002840F0BC80022C01D86101C6
:10BCF00001E0E11E490141F00201C9B2284600F00D
:10BD000013FA444B002203EB44130833022C804601
:10BD10005A7101D8610101E0E11E49013D4B660104
:10BD2000F31841F00601C9B25A68284600F0C4FA77
:10BD3000022C01D8F1B202E0E11E4901C9B2344B34
:10BD400003EB84039B6B9844022398FBF3F24AE6CF
:10BD5000033CE4B200222846214600F0B7F90D2248
:10BD60002B4BF7E4284600F0B1F8022C01D8630011
:10BD700001E0E31E5B00012212FA03F3034270D0DC
:10BD8000234B0E22022C1A5501D8610101E0E11E5D
:10BD9000490141F00201C9B2284600F0C5F91E4B25
:10BDA000022C43F8240001D8610101E0E11E4901A1
:10BDB00041F008010022C9B2284600F017FB022C0E
:10BDC00001D8214601E0E11EC9B20222284600F056
:10BDD0007DF9022C01D8610101E0E11E490141F029
:10BDE00002010022C9B2284600F066FA022C02D8ED
:10BDF0006401E1B202E0E11E4901C9B22846002215
:10BE000000F05AFA2DE0022C08D8214608E000BFC5
:10BE100064050020A40E0020680F0020E11EC9B2B6
:10BE20000222284600F052F9022C01D8610101E0FB
:10BE3000E11E490141F00801C9B22846002200F084
:10BE4000D5FA0E22084B1A550BE0033CE4B2064E1D
:10BE5000284606EB87031A7A214600F009F90023E9
:10BE6000F355BDE8FE8500BF64050020000000001A
:10BE7000154B10B503EB0012926891420EDD8A1A41
:10BE8000C2F18074A2424FEA001C03DC63445C6888
:10BE900012190EE063445A68141B0FE00FDA521AAD
:10BEA000C2F18074A2424FEA001C04DC63445C6867
:10BEB000A21A5A6003E063445A68A4185C60024BFB
:10BEC00003EB0010816010BDFC11002008B5014695
:10BED00018B1012804D0002006E00121072000E06D
:10BEE00008200A46F8F704FD08BD00BF2DE9F0411F
:10BEF000137814460E46C3F34117054610B10337B5
:10BF0000062F34D0554A02EB4712127B7ABB13F04E
:10BF1000010F2CD15F2B2AD8514AD25D3ABB13F0C6
:10BF20009F0301D0082B22D1DFF83C8118F807309D
:10BF300093B94A4B03EB4712D17F21B13846F8F74A
:10BF4000F7FB032306E003EB4713597A3846F8F76B
:10BF5000EFFB022308F80730DFF8108118F80730EC
:10BF60002BB13846FEF706FC002308F8073015B160
:10BF7000012D2ED115E021782A460720F8F7B8FCCC
:10BF8000307061782A460720F8F7B2FC7070A1780B
:10BF90002A460720F8F7ACFCB070E17807200122B0
:10BFA00014E0217800220820F8F7A2FC30706178B4
:10BFB00000220820F8F79CFC7070A178002208206D
:10BFC000F8F796FCB070E17808202A46F8F790FC64
:10BFD000F070237813F0010F3ED15F2B3CD803F0B3
:10BFE0001E02082A04D0142A2CD0062A34D11BE0C1
:10BFF000242169435B090C2000FB0313A57894F806
:10C0000003C0184A4CEA05259D50A37813F0080F89
:10C0100022D025786D0900FB0515AB586FEA035354
:10C020006FEA1353AB5017E0242255435B090C22EF
:10C03000A17802FB0353E27842EA012209495B1826
:10C040005A6009E0242255435B090C2202FB03538A
:10C050000449E2785B181A72BDE8F081A40E002052
:10C06000E40F0020480E0020D80F0020EC0F002025
:10C07000022973B50C460546164601D84B0101E06E
:10C08000CB1E5B0143F01503DBB22846694601AACB
:10C090008DF80430FFF72AFF022C88BF033C6401AF
:10C0A0009DF801C09DF8033044F01404E4B2284622
:10C0B000694601AA8DF804408DF805C08DF8066028
:10C0C0008DF80730FFF712FF7CBD00BF022973B562
:10C0D0000C460546164601D84B0101E0CB1E5B011C
:10C0E00043F01503DBB22846694601AA8DF80430F7
:10C0F000FFF7FCFE022C88BF033C64019DF801C0E1
:10C100009DF8023044F01404E4B22846694601AABE
:10C110008DF804408DF805C08DF806308DF8076065
:10C12000FFF7E4FE7CBD00BF37B541F001030C46CC
:10C130006A4601A98DF800300546FFF7D7FE9DF845
:10C1400006009DF8052000029DF8073040EA0240F5
:10C15000184310F4000F18BF40F07F405F2C1AD82E
:10C16000C4F3411314F01E0402D0022C13D106E0D4
:10C17000032202FB0535084A2D01A8580BE00322D3
:10C1800002FB053520F07F41E8B2FFF771FE024B5C
:10C1900003EB051568683EBDFC11002007B541F0B2
:10C1A00001036A4601A98DF80030FFF79FFE9DF854
:10C1B00006009DF8073043EA002010F4006F1CBF12
:10C1C0006FEA00506FEA10500EBD00BF13B541F08A
:10C1D0000103144601A96A468DF80030FFF786FE78
:10C1E0009DF805109DF806309DF807202170A2707B
:10C1F00063709DF804001CBD022807B501D84101F9
:10C2000001E0C11E490141F01601C9B2022894BFE4
:10C210000020012001AAFFF7D9FF9DF80530D809B9
:10C2200013F0200F18BF40F002000EBD022807B522
:10C2300001D8410101E0C11E490141F01601C9B216
:10C24000022894BF0020012001AAFFF7BFFF9DF83C
:10C250000530C3F3801013F0100F18BF40F0020038
:10C260000EBD00BF022837B504460D4601D8410176
:10C2700001E0C11E4901C9B2294301AA022C94BFA1
:10C2800000200120FFF7A2FFB4235C436D080323C5
:10C2900004F5807403FB05459DF804102846FCF75F
:10C2A000A1FC681C9DF80510FCF79CFCA81C9DF8DF
:10C2B0000610FCF797FC3EBD5F292DE9F3410D46C2
:10C2C0000646144667D8C1F3411C11F01E0102D086
:10C2D000022960D11EE0032202FB00CC374A4FEA5C
:10C2E0000C1083185B688450E01A0028B8BF4042E5
:10C2F000B0F5000F0ADB9C42CCBF314C314C2F4AC9
:10C300001C1902EB0C120123137344E002EB0C1214
:10C31000117340E0032707FB00C7284B3801C158C1
:10C320007A00C4EB010E0132BEF1000FB8BFCEF1AE
:10C33000000E00EB0308BEF5000F24F07F40C8F8A4
:10C34000044043F8320022DBA142CCBF1C4B1D4B02
:10C350003046E318BCF1030F0CBF4FF0000C4FEA5E
:10C360004C1C4FEA23484FEA232E694601AA8DF858
:10C3700007308DF804C08DF805808DF806E0FFF7D2
:10C38000B5FD0E4B03EB071701233B7303E003EBF3
:10C39000C20300221A714FEA244C23123046694628
:10C3A00001AA8DF804508DF805C08DF806308DF87F
:10C3B0000740FFF79BFDBDE8FC8100BFFC1100209A
:10C3C000FFFF7F00010080FF38B50D46682104465D
:10C3D000FFF7AAFE15B140F0010201E020F00102D2
:10C3E00020466821FFF768FF38BD00BF07B5134638
:10C3F0004FEA222C8DF804104FF0000E694601AA76
:10C400008DF805E08DF806C08DF80730FFF76EFD5A
:10C410000EBD00BF07B50B4611F01E01024601D04C
:10C42000022905D1104619460022FFF745FF0DE00D
:10C430004FF0000C694601AA8DF804308DF807C052
:10C440008DF805C08DF806C0FFF750FD0EBD00BF8A
:10C45000022838B5044694BF0025012501D8C1B291
:10C4600001E0C11EC9B202222846FFF72FFE022CAE
:10C4700001D8610101E0E11E490141F00801C9B2A2
:10C480002846FFF7C7FF022C01D8610101E0E11E39
:10C49000490141F00A01C9B22846FFF7BBFF38BD88
:10C4A00007B59DF810C08DF804108DF80520694679
:10C4B00001AA8DF806308DF807C0FFF717FD0EBDF5
:10C4C00030B5022885B0044601D8430101E0C31EFF
:10C4D0005B0143F00303022C94BF00250125DBB26E
:10C4E000284603A902AA8DF80830FFF7FFFC9DF843
:10C4F0000E109DF80D209DF80F30090241EA02410F
:10C5000019432046FFF7B4FC1F4B03EB04131B7BBE
:10C51000002B37D0022C1D4A94BF2346E31E0C216A
:10C5200001FB0323022C8CBF242200229B181B7AC0
:10C5300043BB15482201111849681258C1EB020C7F
:10C54000BCF1000FB8BFCCF1000CBCF5000F05DB4F
:10C550008A42CCBF0E4A0F4A8A1802E000EB041050
:10C560000373022C02D86401E1B202E0E11E49012A
:10C57000C9B2D4B2C2F307232846C2F307420094DB
:10C58000FFF78EFF05B030BDFC110020480E0020E3
:10C59000FFFF7F00010080FF07B5937892F800E06D
:10C5A00092F801C08DF8041001AA69468DF805E0E3
:10C5B0008DF806C08DF80730FFF798FC0EBD00BF60
:10C5C000022873B504460E4694BF0025012501D804
:10C5D000410101E0C11E490141F01601C9B22846DE
:10C5E00001AAFFF7F3FD9DF8053016F0010F1ABF01
:10C5F0006FEA43636FEA536303F07F038DF80530FE
:10C600009DF8053016F0020F14BF43F0200323F00D
:10C610002003022C8DF8053001D8610101E0E11EF4
:10C62000490141F016010023C9B2284601AA8DF83C
:10C630000630FFF7B1FF7CBD022873B504460E46F5
:10C6400094BF0025012501D8410101E0C11E490127
:10C6500041F01601C9B2284601AAFFF7B7FD9DF8BF
:10C66000053016F0010F14BF43F0400323F04003E0
:10C670008DF805309DF8053016F0020F14BF43F019
:10C68000100323F01003022C8DF8053001D861014E
:10C6900001E0E11E490141F016010023C9B228461C
:10C6A00001AA8DF80630FFF777FF7CBD73B5B4257E
:10C6B00045434B08032205F5807502FB03550446EC
:10C6C00028460E46FCF7F8F98DF80400681CFCF7C4
:10C6D000F3F98DF80500A81CFCF7EEF9022C0346CF
:10C6E00001D8610101E0E11E4901C9B23143022CC8
:10C6F00094BF0020012001AA8DF80630FFF74CFFFF
:10C700007CBD00BF2DE9FF474D05022804464FEAD6
:10C71000555594BF4FF000084FF0010801D8410172
:10C7200001E0C11E490141F01801C9B2404603AA07
:10C73000FFF74CFD9DF80D9009F00F0A4FEA19190B
:10C74000CA4510DB284604F023FFC9EB0A0A064657
:10C75000012000FA0AF00F4604F02AFF00223C4BA9
:10C7600004F08CFF11E0284604F012FFCAEB090A1E
:10C770000646012000FA0AF00F4604F019FF0246AF
:10C780000B460020324905F0A3F802460B4630461E
:10C79000394605F09DF805F0ABF904F01BFF2AA31C
:10C7A000D3E9002304F06AFF05F0A2F904F012FFB8
:10C7B0000022284B04F062FFCDE900014FF0FF3763
:10C7C000BA4600260120B04004F0F2FE02460B46B5
:10C7D000DDE9000104F052FF05F062F9A0F18002EA
:10C7E0007F2A98BF3746034606F1010688BF5346A5
:10C7F0000E2E01D09A46E5E7022C01D8610101E036
:10C80000E11E490141F012014FF0000CC9B240464F
:10C8100003AA8DF80CC08DF80D308DF80E70FFF75F
:10C82000BBFE022C01D8610101E0E11E490141F08B
:10C830000C014046C9B22A46FFF7D8FD002004B0DB
:10C84000BDE8F087AFF3008004560E2DB29DEF3F98
:10C850000000604000002040F7B5304B587E10F0DB
:10C86000010004D00020682140F2231202E0682178
:10C870004FF49172FFF720FD00207E210346022431
:10C8800002460094FFF70CFE244B5B7E13F0020F70
:10C8900004D00120682140F2231203E00120682126
:10C8A0004FF49172FFF708FD0022022401207E213F
:10C8B00013460094FD25FFF7F3FD00242BE0E7B2BB
:10C8C000F1B238460136FFF7F1FE1D2EF7D1022CEA
:10C8D00094BF0026012601D8790100E0690141F0EA
:10C8E0000C01C9B23046FFF71FFC01463846FFF77E
:10C8F00009FF022C01D8790100E0690141F016011D
:10C90000C9B2304643F2FF1201340135FFF76EFD24
:10C91000062CEDB201D00026D1E7FEBD04000020B8
:10C92000084B1868034605E02C2A02D100221A7031
:10C9300003E001331A78002AF6D1024A013313606A
:10C94000704700BFB405002010B50E4B02461B789F
:10C95000ABB10D4B1C7994B19C68601CE4180D2A96
:10C960002273986002D03F2800D851B9064C014686
:10C9700004F10C00FDF70EFA0023A36001E0FCF7C0
:10C9800031FB10BDBC0D0020B405002030B50121E5
:10C99000044687B02020FFF7D7FF002C04DA2D20B3
:10C9A0000121FFF7D1FF644200230A2194FBF1F239
:10C9B00001FB124101AD3031E954591C141E01DD57
:10C9C0000B46F2E7ED181C460121013C15F8010960
:10C9D000FFF7BAFFB4F1FF3FF6D107B030BD00BF9B
:10C9E00038B50C4D0446A87801214030C0B2FFF79D
:10C9F000ABFF687801214030C0B2FFF7A5FF207877
:10CA0000FFF7C4FF6068FFF7C1FF0D200121FFF7AA
:10CA10009BFF38BD0400002070B5124B06461B7802
:10CA2000EBB1FCF7ADFA104C054618B100232371A9
:10CA3000012016E0E36C226D934208D21A1992F895
:10CA40005420013301203270E364207109E004F1C5
:10CA50005400FDF76DF9E5642065284601E0FCF718
:10CA60008FFA70BDBC0D0020B40500202DE9F34104
:10CA700004460DF10700FFF7CFFF002800F0CB8040
:10CA80008B4B8C4A93F8941019BB51789DF8070092
:10CA9000403188420DD1D3F89810002940F0BB8076
:10CAA0001179012231F0010183F8942040F0B38024
:10CAB000AFE00D2801D01B2802D100227C4B05E0FD
:10CAC000D3F898207E2A00F2A6800132C3F898207D
:10CAD000A1E0117931F0010103D19DF80700FFF7C2
:10CAE00033FF9DF807301F2B0BD9714AD2F89810ED
:10CAF0007E297FD8481C891881F89C30C2F898009C
:10CB000078E0082B08D16A4BD3F89820002A71D01E
:10CB1000013AC3F898206DE00D2B6BD1644BD3F82C
:10CB20009830002B66D0634B1A79112A15D15878AA
:10CB300001214030C0B2FFF707FF002503E0585D38
:10CB4000FFF702FF01355A4B0121D3F898209C339F
:10CB50009542F4D30D20FFF7F7FE554A00231568E0
:10CB6000D2F8987019461A4633E001290FD002D343
:10CB700002292DD122E04E4E06F19C00805C202837
:10CB800026D09E1986F81C010133012120E0484877
:10CB900000F19C0C1CF802C0BCF1200F0AD1012B43
:10CBA00004D91818002180F81C110133424D0221CC
:10CBB000ED180DE0181880F81CC108E03C4E06F195
:10CBC0009C00805C202803D09E1986F81C0101334C
:10CBD0000132BA42C9D3364A0021981880F81C1194
:10CBE0000120C2F89810156082F8A001C2F89C31AB
:10CBF00082F894109DF807301B2B0CD12D4A2C4B3A
:10CC000012790021012A83F89410C3F8981002D1F8
:10CC10000D20FFF799FE264B93F8A001002878D04D
:10CC20000022164683F8A0211546DFF8A8800727C2
:10CC300007FB058720483946013504F03BF930B938
:10CC4000BE797B7916F0010F237049D007E018F800
:10CC500006300736002B5ED0FF2DE6D15BE0FFF7F4
:10CC60005FFE23780546042B0CD1144904F022F909
:10CC70000346D8B12846124904F01CF970B1284681
:10CC800010490FE00D2B28D10F4904F013F903468A
:10CC900060B128460D4904F00DF908B9012305E0FB
:10CCA0000B49284604F006F9B0B90223637017E077
:10CCB000B405002004000020D006002091240108C3
:10CCC00095240108992401089F240108A52401083E
:10CCD000AA24010888220108284604F0E5F86070BB
:10CCE00016F0020F04D0FFF71BFE04F0DDF8A07071
:10CCF00016F0040F0CD0FFF713FE04F0D5F8010E68
:10CD0000C0F30722C0F30743A17122716371E07081
:10CD10000120BDE8FC8100232370F9E7704700BFC4
:10CD2000FEE700BFFEE700BFFEE700BFFEE700BF73
:10CD3000704700BF704700BF704700BF704700BF1B
:10CD4000704700BF704700BF704700BF704700BF0B
:10CD5000704700BF704700BF704700BF704700BFFB
:10CD6000704700BF704700BF704700BF704700BFEB
:10CD7000704700BF704700BF704700BF704700BFDB
:10CD8000704700BF704700BF08B5024B1B6898474B
:10CD900008BD00BF240E002008B5024B1B68984751
:10CDA00008BD00BFE00F002008B5024B1B68984784
:10CDB00008BD00BFA00E002008B5024B1B689847B5
:10CDC00008BD00BF640F0020704700BF704700BF60
:10CDD000704700BF704700BF704700BF704700BF7B
:10CDE000704700BF704700BF704700BF704700BF6B
:10CDF000704700BF704700BF704700BF704700BF5B
:10CE0000704700BF704700BF704700BF704700BF4A
:10CE1000704700BF704700BF704700BF704700BF3A
:10CE2000704700BF704700BF704700BF704700BF2A
:10CE3000704700BF704700BF704700BF704700BF1A
:10CE4000704700BF704700BF704700BF704700BF0A
:10CE5000704700BF704700BF704700BF436830B5E0
:10CE600023F470230C680A7923F48073234343EA84
:10CE70000223436082688D68CC680A4B45EA040C43
:10CE800002EA03034A794CEA030343EA420383605C
:10CE90000B7CC26A013B22F47002DBB242EA03530C
:10CEA000C36230BDFDF7F1FF002301220274C360AD
:10CEB0000360037143718360704700BF19B18368D9
:10CEC00043F0010302E0836823F0010383607047AD
:10CED00019B1836843F4807302E0836823F480739C
:10CEE00083607047C9B212B14368194302E04368D6
:10CEF00023EA010141607047836843F008038360BF
:10CF0000704700BF8068C0F3C0007047836843F07B
:10CF100004038360704700BF8068C0F380007047DF
:10CF200019B1836843F4A00302E0836823F4A003EB
:10CF3000836070478068C0F3805070474368013950
:10CF400023F4604343EA41334360704719B14368B7
:10CF500043F4006302E0436823F4006343607047D6
:10CF6000092930B511D94FF0030C0CFB01FC072542
:10CF7000ACF11E0C05FA0CF503FA0CFCC46824EAAB
:10CF8000050343EA0C03C3600EE04FF0030C0CFBF7
:10CF900001FC072505FA0CF503FA0CFC046924EAE8
:10CFA000050343EA0C030361062A0DD80523013A61
:10CFB0005A434FF01F0C0CFA02FC9140436B23EADA
:10CFC0000C020A4342631CE00C2A0DD805235A4385
:10CFD0004FF01F0C233A0CFA02FC9140036B23EA3A
:10CFE0000C020A4302630CE005235A434FF01F0C66
:10CFF000413A0CFA02FC9140C36A23EA0C020A434C
:10D00000C26230BD19B1836843F4801302E08368C3
:10D0100023F4801383607047C06C80B2704700BFF8
:10D02000014B1868704700BF4C24014019B1436898
:10D0300043F4806302E0436823F4806343607047F5
:10D0400019B1436843F4805302E0436823F48053EA
:10D0500043607047836823F4E04341EA030383603D
:10D06000704700BF19B1836843F4004302E083684E
:10D0700023F400438360704719B1836843F40213BB
:10D0800002E0836823F40213836070478068C0F372
:10D0900040507047092930B511D94FF0030C0CFBF3
:10D0A00001FC0725ACF11E0C05FA0CF503FA0CFC8B
:10D0B000C46824EA050343EA0C03C3600EE04FF0A2
:10D0C000030C0CFB01FC072505FA0CF503FA0CFC1C
:10D0D000046924EA050343EA0C030361836BC3F389
:10D0E000015CCCEB020202324FF0050CD2B20CFB19
:10D0F00002F20CF11A0C0CFA02FC914023EA0C0328
:10D100000B43836330BD00BF836B013923F44013AD
:10D1100043EA0153836370470A50704728304058F0
:10D1200080B27047436823F4400323F4007341EA5C
:10D1300003034360704700BF41628262704700BFD3
:10D14000436823F01F0341EA03034360704700BFB5
:10D1500020B1054B9A6842F4000203E0024B9A6842
:10D1600022F400029A6070470024014003681942CB
:10D170000CBF002001207047C9430160704700BF09
:10D180004368006810EA112004D0C9B219420CBFEC
:10D1900000200120704700BF6FEA11210160704735
:10D1A00008B5134B98420FD003F5A053984213D003
:10D1B000A3F5C053984219D14FF40070012101F03A
:10D1C0000BFB4FF400700EE04FF48060012101F082
:10D1D00003FB4FF4806006E04FF40040012101F0B2
:10D1E000FBFA4FF40040002101F0F6FA08BD00BF41
:10D1F00000280140374B01221A605A6812F00102E0
:10D2000001D1104664E00278012A0BBF1A681A683F
:10D2100042F0800222F080021A604378012B04D190
:10D220002C4B1A6842F0400203E02A4B1A6822F0A5
:10D2300040021A608378012B04D1264B1A6842F011
:10D24000200203E0234B1A6822F020021A60C37800
:10D25000012B04D11F4B1A6842F0100203E01D4B52
:10D260001A6822F010021A600379012B04D1194BBD
:10D270001A6842F0080203E0164B1A6822F008020E
:10D280001A604379012B04D1124B1A6842F0040250
:10D2900003E0104B1A6822F004021A608279C37905
:10D2A00090F808C0920742EA03624189437A42EA51
:10D2B0000C4242EA03520139064B0A43DA611A680A
:10D2C00022F001021A60586880F0010000F00100AD
:10D2D000704700BF0064004090F800C0012202FACD
:10D2E0000CF23B4B2DE9F045D3F8004292B244F0EA
:10D2F0000104C3F80042D3F81C42D14301EA0404FC
:10D30000C3F81C428478A4B90CF1480CD3F80C7211
:10D31000B0F80AA0C688B0F8088085884FEACC0427
:10D3200004F1804446EA0A4645EA084501EA07074F
:10D3300015E0012C1AD10CF1480CD3F80C72B0F89E
:10D3400004A0C688B0F8088045894FEACC0404F1EF
:10D35000804446EA0A4645EA084542EA070704F5DA
:10D36000C844C3F80C7243F83C60656043782BB93D
:10D37000174BD3F8044201EA040404E0144BD3F839
:10D38000044242EA0404C3F80442838923B9104BDF
:10D39000D3F81442214006E0012B06D10C4BD3F800
:10D3A000141242EA0101C3F81412837B012B05D148
:10D3B000074BD3F81C120A43C3F81C22044BD3F8C2
:10D3C000002222F00102C3F80022BDE8F08500BF70
:10D3D0000064004003220272013A002342724FF0BF
:10D3E0000102C3714281037043708370C370037183
:10D3F00043718371704700BF19B1054B5A691043DF
:10D4000003E0034B5A6922EA00005861704700BFED
:10D4100000640040364B70B59968024611F0806F89
:10D4200001D000200CE0996811F0006F01D00120BC
:10D4300006E09B6813F0805F01D1042056E00220D3
:10D440002B4B00F118010901CC5804F00104CC5019
:10D45000157A92F809C035B9146864051460CD587E
:10D460004CEA050C07E0546845EA0C0CE4005460F3
:10D47000CE584CEA060C4CEA0404CC50947A00F1E5
:10D48000180C4FEA0C1C04F00F040CF1804394724A
:10D4900003F5C8435D68010125F00F055D605D6817
:10D4A00001F180412C435C60537B947BD57A1B0453
:10D4B00043EA0463147B2B4343EA042301F5C84188
:10D4C000C1F88831557C937CD47B2D0445EA0365F3
:10D4D000137C45EA040242EA0322054BC1F88C2181
:10D4E0005CF8032042F001024CF8032070BD00BF3D
:10D4F00000640040012810D002D302282CD11AE089
:10D50000164A91689368926801F0010103F00203E2
:10D5100043EA8103C2F380621AE0104A936891687B
:10D5200003F48073926801F400719B0943EA1123AC
:10D53000C2F3C0620CE0094A9368916803F4803337
:10D54000926801F400319B0B43EA1143C2F300726D
:10D550001343034AD05C70470023FAE7006400409D
:10D5600068230108012808D002D302280FD109E05E
:10D57000074B9A6842F0800208E0054B9A6842F433
:10D58000004203E0024B9A6842F400029A6070473E
:10D590000064004018B9044B2022DA6002E0024B1C
:10D5A00020221A61704700BF0064004010B9064B8A
:10D5B000D86805E0012801D0002003E0024B18697B
:10D5C00000F00300704700BF00640040254B00F1ED
:10D5D0001B02120110B5D45804F004040C721CB9DB
:10D5E000D3585B0D0B6002E0D358DB084B6000F1B1
:10D5F0001B021C4B1201D35802F1804203F00203BC
:10D600004B7202F5C8425468030104F00F0C81F814
:10D610000AC0526803F18043120ACA7403F5C84372
:10D62000D3F8B821CA72D3F8B821120A0A73D3F812
:10D63000B821120C4A73D3F8B821120E8A73D3F8AA
:10D64000BC21CA73D3F8BC21120A0A74D3F8BC21D6
:10D65000120C4A74D3F8BC311B0E8B74FFF79AFF7F
:10D6600010BD00BF00640040044B1A6842F0020283
:10D670001A601868C0F34000704700BF00640040A3
:10D68000054B1A6822F002021A60186880F0020046
:10D69000C0F34000704700BF00640040034B9B692B
:10D6A00018420CBF00200120704700BF00640040FA
:10D6B000024B9A6922EA00029A61704700640040B6
:10D6C000202831D00CD8062820D004D8042825D012
:10D6D000052844D118E007281DD008283FD11FE0B5
:10D6E000B0F5007F2BD005D840281FD0B0F5807F43
:10D6F00035D11FE0B0F5803F2CD0B0F5003F2BD0E6
:10D70000B0F5806F2BD11FE0012201E04FF4807251
:10D71000134B9A6023E04FF48032F9E7082200E0CF
:10D7200010220F4BDA601AE0082200E010220C4BA6
:10D730001A6114E00A4B9A6922F0010208E0084BD2
:10D740009A6922F0020203E0054B9A6922F0040272
:10D750009A6104E0082200E01022014B5A607047F1
:10D760000064004001420CBF00200120704700BF50
:10D77000202808B532D00CD8062821D004D8042897
:10D7800026D0052818D119E007281ED0082813D163
:10D7900020E0B0F5007F29D005D8402820D0B0F592
:10D7A000807F09D120E0B0F5803F27D0B0F5003F61
:10D7B00022D0B0F5806F1BD0002024E0012101E0D1
:10D7C0004FF48071104B98681BE04FF48031F9E7FB
:10D7D000082100E010210C4BD86812E0082100E07D
:10D7E0001021094B18690CE0012102E0022100E040
:10D7F0000421054B986904E0102100E00821024B48
:10D800005868FFF7AFFF08BD00640040012108B56C
:10D810004FF0007000F0EEFF4FF00070002100F0BC
:10D82000E9FF08BD0268002322F0010202600360E4
:10D8300043608360C3602D4B984233D011D83C3B8A
:10D84000984229D006D8283B984221D014339842D8
:10D850004BD11FE0264B984220D01433984244D13C
:10D860001EE0244B98422CD008D8A3F56773984249
:10D870001DD003F56273984237D11DE01E4B9842CC
:10D8800029D0143398422BD0283B98422DD11DE04B
:10D890001A4B12E0194B15E0184B18E0174B1BE020
:10D8A000164B1EE0154B5A6842F470021CE0134BF5
:10D8B0005A6842F0706217E0114B5A6842F00F024A
:10D8C00012E00F4B5A6842F0F0020DE00C4B5A6820
:10D8D00042F4706208E00A4B5A6842F4704203E076
:10D8E000074B5A6842F470225A6070476C0002403D
:10D8F000440002401C040240440402400000024074
:10D90000000402408A6870B50C6A0B6944EA02029E
:10D910004C691A438B692243CC6905684E6A42EA16
:10D92000030323438C6A334325F4FE4C23432CF03A
:10D93000F00C43EA0C030360CB6843600B68836020
:10D940004B68C36070BD00BF002383620360436007
:10D950008360C360036143618361C36103624362A7
:10D96000704700BF19B1036843F0010302E0036888
:10D9700023F001030360704712B10368194302E00A
:10D98000036823EA01010160704700BF406880B26C
:10D99000704700BF10F0805F14BF044B044B1B683E
:10D9A00003420CBF00200120704700BF000402406A
:10D9B0000000024010F0805F14BF024B024B586021
:10D9C000704700BF000402400000024010F0805F7A
:10D9D00014BF044B044B1B6803420CBF0020012002
:10D9E000704700BF000402400000024010F0805F5A
:10D9F00014BF024B024B5860704700BF0004024046
:10DA000000000240044B00221A605A609A60DA60FB
:10DA1000024A5A61704700BF00040140FFFF07003F
:10DA2000837930B5016802794BB3184BCC431D683C
:10DA300090F805C004EA05051D605D682C405C6037
:10DA4000D45844EA0101D15002689868D14301EAF0
:10DA500000009860D8680140BCF1100FD96007D170
:10DA6000996811439960D96841EA0202DA600BE0D3
:10DA70005CF8031041EA02024CF8032004E0034B77
:10DA8000D05820EA0101D15030BD00BF0004014050
:10DA900000230C228371427103600371704700BF41
:10DAA000024B1A6940EA02021A6170470004014001
:10DAB000034B5B6918420CBF00200120704700BF78
:10DAC00000040140014B5861704700BF0004014051
:10DAD000054B1A685B69034001D1184603E0104208
:10DAE0000CBF00200120704700040140014B586129
:10DAF000704700BF00040140044B1A6802F038026E
:10DB00001A601A6840EA02021A6070470020024058
:10DB1000044B1A6822F008021A601A6840EA0202EE
:10DB20001A60704700200240044B1A6822F010026D
:10DB30001A601A6840EA02021A6070470020024028
:10DB4000034B044A5A6002F188325A60704700BFA2
:10DB50000020024023016745024B1A6942F080020F
:10DB60001A61704700200240014BD8698008704755
:10DB700000200240014B186A704700BF002002409D
:10DB8000024BD869C0F34000704700BF002002403C
:10DB9000024B1868C0F34010704700BF00200240DD
:10DBA00019B1054B1A69104303E0034B1A6922EAC5
:10DBB00000001861704700BF00200240012804D116
:10DBC000054BD86900F0010005E0034BDB68184203
:10DBD0000CBF00200120704700200240014BD8609C
:10DBE000704700BF00200240094BDA6812F0010FB5
:10DBF00001D001200BE0DA6812F0040F01D00220FE
:10DC000005E0DB6813F0100F14BF032004207047F9
:10DC10000020024013B504460AE000230193FF33BD
:10DC200001E0019B013B0193019B002BF9D1013CD9
:10DC3000FFF7DAFF012802D1002CEED100E004B991
:10DC400005201CBDF8B5124C124B0546A36003F12C
:10DC500088330F20A3600E461746FFF7DBFF04282A
:10DC600014D1236945F0F80543F0100323612E43D6
:10DC7000094B37430B305F80FFF7CCFF012805D0FD
:10DC8000226941F6EF7302EA03032361F8BD00BF86
:10DC9000002002402301674500F8FF1F38B5054604
:10DCA00040F6FF70FFF7B6FF04283CD11E4C1F4B17
:10DCB00040F6FF70A36003F18833A360236943F04B
:10DCC00020032361236943F040032361FFF7A2FF90
:10DCD000042820D1226941F6DF7302EA030323619D
:10DCE000236943F0100323611DB1114B4FF0000273
:10DCF00002E00F4B4FF0A5021A8040F6FF70FFF7CD
:10DD000089FF01280FD0084A41F6EF73116901EA33
:10DD10000303136107E0012805D0226941F6DF7390
:10DD200002EA0303236138BD002002402301674556
:10DD300000F8FF1F10B504460F20FFF76BFF042803
:10DD40003DD11F4A1F4BE443936003F18833936036
:10DD50001169E3B241F01001FF2B116106D01A4A9C
:10DD60000B301381FFF756FF04281FD1C4F307239C
:10DD7000FF2B06D0144A0F205381FFF74BFF0428D6
:10DD800014D1C4F30743FF2B06D00F4A0F20938111
:10DD9000FFF740FF042809D1240EFF2C01D10420F5
:10DDA00006E0094B0F20DC81FFF734FF012806D085
:10DDB000034A41F6EF73116901EA0303136110BDD1
:10DDC000002002402301674500F8FF1F70B504469C
:10DDD0000F200E46FFF71EFF042815D10B4D0C4BEC
:10DDE0000B30AB6003F18833AB602B6943F0100359
:10DDF0002B612680FFF70EFF012805D02A6941F626
:10DE0000EF7302EA03032B6170BD00BF00200240E4
:10DE10002301674570B504460F200E46FFF7FAFE52
:10DE2000042810D1084D0B302B6943F001032B61FE
:10DE30002680FFF7EFFE012805D02A6941F6FE7320
:10DE400002EA03032B6170BD0020024070B5044656
:10DE50000F200E46FFF7DEFE042818D10C4DB3B29A
:10DE60002A690B3042F001022A612380FFF7D2FEBB
:10DE7000042804D1360C66800B30FFF7CBFE012856
:10DE800005D02A6941F6FE7302EA03032B6170BDD7
:10DE90000020024010B540F6FF70FFF7BBFE0428DB
:10DEA0002CD1174C174B40F6FF70A36003F1883359
:10DEB000A360236943F020032361236943F04003F7
:10DEC0002361FFF7A7FE042810D1226941F6DF7312
:10DED00002EA0303236123694FF0A50243F0100314
:10DEE0002361094B0B301A80FFF794FE012805D0FF
:10DEF000226941F6EF7302EA0303236110BD00BFFC
:10DF0000002002402301674500F8FF1F10B540F6CE
:10DF1000FF70FFF77FFE042814D10B4C40F6FF7012
:10DF2000236943F004032361236943F04003236121
:10DF3000FFF770FE012805D0226941F6FB7302EA63
:10DF40000303236110BD00BF0020024038B5054621
:10DF500040F6FF70FFF75EFE042815D10B4C40F62B
:10DF6000FF70236943F0020323616561236943F075
:10DF700040032361FFF74EFE012805D0226941F6D8
:10DF8000FD7302EA0303236138BD00BF0020024095
:10DF9000CB78F0B513F0100F18BF8A78098803F01A
:10DFA0000F0C18BF4CEA020C11F0FF0F1AD00468D6
:10DFB00000220126964006EA0105B5420ED19600E0
:10DFC0000F27B7400CFA06F624EA07043443282B3F
:10DFD00001D1456102E0482B08BF05610132082AE2
:10DFE000E7D10460FF291CD94468002202F108052A
:10DFF0000126AE4006EA0105B5420ED196000F2774
:10E00000B7400CFA06F624EA07043443282B01D162
:10E01000456102E0482B08BF05610132082AE5D1BD
:10E020004460F0BD0423C370022383704FF0FF33BC
:10E0300003807047836819420CBF0020012070479D
:10E04000806880B2704700BFC36819420CBF0020CF
:10E0500001207047C06880B2704700BF01617047FF
:10E06000416170470AB1016100E04161704700BF42
:10E07000C160704741F4803383618161836183694A
:10E0800083697047064A10B514684FF6807341EAF9
:10E09000001104EA030341EA0303136010BD00BF4B
:10E0A00000000140014B1860704700BF1C00204277
:10E0B0000304154A00F4401C1B0CBCF5401F30B58E
:10E0C000546806D1556824F0706425F07065556079
:10E0D00011E010F4801F06D0C0F303424FF0030C90
:10E0E0000CFA02F203E0420D120113FA02F224EAE2
:10E0F000020444F0706419B1400D000183401C43D8
:10E10000014B5C6030BD00BF0000014001F0030323
:10E110009B000F229A4010FA03F310B58908074CB0
:10E12000023154F8210020EA020244F8212054F878
:10E130002120134344F8213010BD00BF00000140EE
:10E140000120014608B500F047FB0120002100F046
:10E1500043FB08BD08B5264B98422BD00CD8A3F53D
:10E16000006398421AD003F5806398421CD0A3F54F
:10E17000006398423AD10BE01E4B984226D003F53B
:10E180008063984228D0A3F5006398422ED117E00F
:10E190000420012100F020FB042024E008200121BC
:10E1A00000F01AFB08201EE01020012100F014FBF3
:10E1B000102018E02020012100F00EFB202012E0AA
:10E1C0004020012100F008FB40200CE080200121CC
:10E1D00000F002FB802006E04FF48070012100F087
:10E1E000FBFA4FF48070002100F0F6FA08BD00BF82
:10E1F00000140140001C01400B4B4FF0FF316FF049
:10E200007042C3F88010C3F88420C3F88011C3F8AB
:10E210008421002303F1C001034A013300200F2BA6
:10E2200042F82100F6D1704700E100E0094B4FF0C1
:10E2300020605860084800224FF0FF319A60D86093
:10E240001A615A619A61DA611A625A629962D962F4
:10E250001963704700ED00E00000FA0540F0BE6071
:10E26000024B40F42020D860704700BF00ED00E072
:10E2700030B5C27803787AB31C4A4178D2684FF03F
:10E280000F0CD243C2F302222CFA02FCC2F10402A8
:10E290009140807803F003020CEA000C4CEA010C78
:10E2A000D2004FEA0C1CFF2090400CFA02FC012423
:10E2B00003F01F02944099080D4AC03152F82150D2
:10E2C0000CEA000C25EA00004CEA00005B0942F869
:10E2D000210042F8234008E003F01F020121914091
:10E2E0005B09034A203342F8231030BD00ED00E003
:10E2F00000E100E00023C370037043708370704737
:10E30000024B5868C0F30930704700BF00ED00E0D1
:10E31000012200F01F0312FA03F34009044A4030BF
:10E3200052F820001840984214BF00200120704786
:10E3300000E100E0014B1860704700BF00EF00E013
:10E3400000F01F0301229A404009024B603043F85D
:10E350002020704700E100E0024B58688005800DE6
:10E36000704700BF00ED00E0012200F01F0312FA29
:10E3700003F34009044A803052F8200018409842C4
:10E3800014BF00200120704700E100E0014B186835
:10E39000704700BF00ED00E021F0604121F07F01F7
:10E3A000014B01439960704700ED00E0014A024BC8
:10E3B000DA6070470400FA0500ED00E0014A024B04
:10E3C000DA6070470100FA0500ED00E019B1054B75
:10E3D0001A69104303E0034B1A6922EA000018612E
:10E3E000704700BF00ED00E000F01F00012313FAAA
:10E3F00000F019B1044B5A6A104303E0024B5A6A09
:10E4000022EA00005862704700ED00E0144B70B53E
:10E41000DC684FF0FF0CE443C4F302242CFA04F54B
:10E42000C4F1040411FA04F4C0F30126F6000CFA56
:10E4300006FC02EA050545EA0404240114FA06F67E
:10E44000C0F38110063053F8202022EA0C0243F872
:10E45000202053F82020164343F8206070BD00BFF1
:10E4600000ED00E0C0F3832001238340044A506A9A
:10E4700003EA0000984214BF00200120704700BF4B
:10E4800000ED00E000F01F0001228240024B5968BD
:10E490000A435A60704700BF00ED00E000F01F0221
:10E4A0000123013A13FA02F2024B59680A435A60F7
:10E4B000704700BF00ED00E0C0F3833001238340CC
:10E4C000044A506A03EA0000984214BF0020012069
:10E4D000704700BF00ED00E0C0F3814313B90A4B61
:10E4E000D86A10E0012B0CD1074AC0F30153906A9F
:10E4F000DA00D040022B14BF00F00F0000F0FF0044
:10E5000001E0014B186B704700ED00E010F4800F44
:10E510000BBF024B014B586B986B704700ED00E04E
:10E5200008B5F5F725FE08BD08B50001F5F71DFE95
:10E5300008BD00BF08B5F5F716FE08BD08B5F5F72C
:10E5400010FE08BD08B5F5F70AFE08BD08B5F5F7D9
:10E5500004FE08BD0D4B0E4A196841F00101196017
:10E56000596801EA02025A601A6822F0847222F4A1
:10E5700080321A601A6822F480221A605A6822F4E3
:10E58000FE025A6000229A60704700BF00100240ED
:10E590000000FFF80C4BB0F5803F1A6822F480327F
:10E5A0001A601A6822F480221A6003D0B0F5802F16
:10E5B00008D103E01A6842F4803202E01A6842F49B
:10E5C000A0221A60704700BF00100240034B1A6877
:10E5D00022F0F80242EAC0021A60704700100240BE
:10E5E000014B1860704700BF00004242044B5A685C
:10E5F00022F47C1240EA02020A435A60704700BFCC
:10E6000000100240014B1860704700BF600042429A
:10E61000034B5A6822F0030240EA02025A60704734
:10E6200000100240024B586800F00C00704700BF19
:10E6300000100240034B5A6822F0F00240EA020246
:10E640005A60704700100240034B5A6822F4E0629F
:10E6500040EA02025A60704700100240034B5A68B9
:10E6600022F4605242EAC0025A6070470010024031
:10E6700019B1054B1A78104303E0034B1A7822EACC
:10E6800000001870704700BF09100240014B18606D
:10E69000704700BFD8004242034B5A6822F4404200
:10E6A00040EA02025A60704700100240064B002206
:10E6B00001281A701A7002D0042804D101E01870E1
:10E6C00001E005221A70704720100240014B1860CB
:10E6D000704700BF80044242024B1A6A40EA0202BD
:10E6E0001A62704700100240014B1860704700BF6B
:10E6F0003C0442421F4B10B55A6802F00C02042A37
:10E7000013D0082A11D15A685968C2F383420232E1
:10E7100011F4803F03D05B6813F4003F01D0164B27
:10E7200000E0164B5A43026001E0144B0360114AAB
:10E73000134B51680468C1F30311595C34FA01F1B9
:10E7400041605468C4F3022C13F80C4031FA04F40D
:10E7500084605468C4F3C22C13F80CC021FA0CF185
:10E76000C1605268C2F381329B181B7CB1FBF3F18C
:10E77000016110BD0010024000093D0000127A0046
:10E780007023010819B1054B5A69104303E0034B8C
:10E790005A6922EA00005861704700BF0010024029
:10E7A00019B1054B9A69104303E0034B9A6922EAB9
:10E7B00000009861704700BF0010024019B1054B7E
:10E7C000DA69104303E0034BDA6922EA0000D861FA
:10E7D000704700BF0010024019B1054BDA681043C2
:10E7E00003E0034BDA6822EA0000D860704700BFFC
:10E7F0000010024019B1054B1A69104303E0034BA6
:10E800001A6922EA00001861704700BF0010024038
:10E81000014B1860704700BF40044242014B186032
:10E82000704700BF4C004242014B1870704700BF58
:10E83000071002404309012B02D1084B1B6805E079
:10E84000022B0BBF054B054B1B6A5B6A00F01F00D8
:10E8500033FA00F000F00100704700BF00100240E2
:10E8600008B53120FFF7E6FF094B18705A680132EE
:10E870005A601A7822B95A6840F2FF139A42F0D1CE
:10E880003120FFF7D7FF003818BF012008BD00BFB7
:10E8900058070020024B5A6A42F080725A62704751
:10E8A00000100240034B9B6818420CBF002001205F
:10E8B000704700BF00100240014B1870704700BF46
:10E8C0000A1002400B884A88B1F804C01A43CB886A
:10E8D00042EA0C02B1F808C01A434B8930B542EA4B
:10E8E0000C028D89B0F800C0CC891A432A43224318
:10E8F0000CF4415313439BB20380838B23F40063D6
:10E900001B041B0C83830B8A038230BD00234FF052
:10E910000702C3810282038043808380C380038116
:10E9200043818381704700BF00234381038043807C
:10E930008380C3804FF002030381704721B10388B5
:10E940009BB243F0400304E0038823F040031B0420
:10E950001B0C0380704700BF21B1838B9BB243F433
:10E96000806304E0838B23F480631B041B0C83838C
:10E97000704700BF0909012313FA01F189B21AB1E6
:10E9800083889BB2194303E083889BB223EA010189
:10E99000818070471AB183889BB2194303E0838852
:10E9A0009BB223EA01018180704700BF81817047DB
:10E9B000808980B2704700BF4FF6FF63994205D04F
:10E9C00003889BB243F48073038002E003881940FC
:10E9D0000180704721B183889BB243F0040304E0B7
:10E9E000838823F004031B041B0C8380704700BF43
:10E9F000038823F400631B041B0C038003889BB271
:10EA000041EA03030380704703889BB243F48053B9
:10EA10000380704721B103889BB243F4005304E0A4
:10EA2000038823F400531B041B0C0380704700BFB2
:10EA3000012914BF008B808A80B27047008A80B29F
:10EA4000704700BFB1F5804F04D103889BB243F4F7
:10EA5000804304E0038823F480431B041B0C0380E1
:10EA6000704700BF038919420CBF00200120704786
:10EA7000202906D1038903889BB243F04003038019
:10EA800008E0402901D0082901D1038902E0C943E7
:10EA900089B20181704700BF012301F00F0213FA10
:10EAA00002F2B0F804C000891FFA8CFC80B210405A
:10EAB00006D009098B401CEA030F0CBF002001207F
:10EAC000704700BF552906D1038903889BB243F0E4
:10EAD000400303800DE0562901D0532901D1038959
:10EAE00007E001F00F01012313FA01F1C94389B2D4
:10EAF00001817047838BF0B523F47A6323F01F0301
:10EB00001B041B0C83834FF0020303840B89868B49
:10EB1000022B87B004460D46B6B201D1002225E093
:10EB200001A88F88FFF7E6FDEB88002F0CBF0127B7
:10EB30000227B3F5007F2989019A06D1A3F5FB735B
:10EB400053430902B3FBF1F305E00A2349015A4399
:10EB50004F43B2FBF7F305330A229BB2B3FBF2F348
:10EB600003F001021202C3F34F0392B2991E89B25D
:10EB7000FE2928BF002228BF0223E98842EA0303B6
:10EB80000B439BB223842B886A8846EA0303A98837
:10EB900043F4006313436A890B4313439BB2A3837B
:10EBA00007B0F0BD08B5154B98421BD003F5744370
:10EBB000984204D0A3F5784398421DD10AE0012180
:10EBC0004FF48050FFF708FE4FF480500021FFF70C
:10EBD00003FE11E04FF480400121FFF70BFE4FF4DC
:10EBE000804006E04FF400400121FFF703FE4FF4A0
:10EBF00000400021FFF7FEFD08BD00BF003C0040C3
:10EC0000042804D1054B1A6842F0040203E0034BC8
:10EC10001A6822F004021A60704700BF10E000E09A
:10EC2000014B5860704700BF10E000E0012804D19C
:10EC3000084B1A6842F0010206E010F1020F05D1FC
:10EC4000044B1A6822F001021A6002E0014B002214
:10EC50009A60704710E000E020B1054B1A6842F05E
:10EC6000020203E0024B1A6822F002021A607047A7
:10EC700010E000E0014B9868704700BF10E000E032
:10EC8000C308022B0BBF044B034B1B68DB6833FA32
:10EC900000F000F00100704710E000E0038803F08E
:10ECA0008F0303800388B1F806C04A889BB243EA09
:10ECB0000C0313439BB203808B8883850B880385E9
:10ECC000064B984203D003F50063984201D10B7ABA
:10ECD00003864FF001038382704700BF002C014080
:10ECE000038C2DE9F04123F001031B041B0C03846A
:10ECF000038C0A894C8823F002031C4E14431B0426
:10ED00008288B1F806C0058B1B0CA4B2B04244EA5D
:10ED1000030392B20C88ADB2A0F834C003D006F55C
:10ED20000066B04218D18E894F89B1F80E804FF637
:10ED3000F77C03EA0C0C4CEA070748EA06064FF694
:10ED4000FB73898847F6FF4C02EA0C0C07EA0303C1
:10ED5000B2B20B4342EA0C024FF68F7105EA010191
:10ED60002143828001830384BDE8F081002C0140AF
:10ED7000038C2DE9F04123F010031B041B0C0384CA
:10ED8000028CB1F808C022F0200212048488120C10
:10ED90004B8842EA0C1242EA0313A2B21B4C068BC8
:10EDA000B1F806C0A0420D88B6B29BB2A0F838C038
:10EDB00003D004F50064A0421BD1B1F80A804FF6DD
:10EDC0007F748F8903EA040447F2FF3C02EA0C0CCB
:10EDD00044EA0814CA894FF6BF73898804EA03031A
:10EDE0004CEA870C43EA01134CEA82023C469BB290
:10EDF00092B248F6FF7106EA010141EA052189B2A3
:10EE0000828001830384BDE8F08100BF002C0140B3
:10EE1000038C2DE9F04123F480731B041B0C038445
:10EE2000028CB1F808C022F4007212048488120C1B
:10EE30004B8842EA0C2242EA0323A2B21A4C868B88
:10EE4000B1F806C0A0420D88B6B29BB2A0F83CC093
:10EE500003D004F50064A0421BD1B1F80A804FF240
:10EE6000FF748F8903EA040444F6FF7C02EA0C0C69
:10EE700044EA0824CA894FF6FF33898804EA030369
:10EE80004CEA071C43EA01234CEA02123C469BB2BF
:10EE900092B24FF68F7106EA010129438280818385
:10EEA0000384BDE8F08100BF002C0140038CF0B565
:10EEB00023F480531B041B0C0384B1F806C0078C99
:10EEC0000C8882880D89868B4B88A0F840C0DFF8BB
:10EED00048C0BFB2604592B2B6B203D00CF5006C28
:10EEE000604505D192048989920C42EA811292B25E
:10EEF0004DF6FF7C07EA0C0C48F6FF7106EA0101AB
:10EF00004CEA053C41EA04214CEA033389B29BB246
:10EF1000828081830384F0BD002C0140B1F802C0DF
:10EF20000B888A884CEA0303B1F806C013430A89A8
:10EF300043EA0C03B1F80AC013438A8943EA0C037D
:10EF400013439BB2A0F84430704700BF00234FF03A
:10EF5000FF320372438082800380C380704700BF0A
:10EF60000023C381038043808380C3800381438166
:10EF70008381704700234FF00102038103804380A7
:10EF80008280C380704700BF002383810380438059
:10EF90008380C38003814381704700BF21B1038810
:10EFA0009BB243F0010304E0038823F001039B05B7
:10EFB0009B0D0380704700BF39B1B0F844306FEA51
:10EFC00043436FEA53439BB203E0B0F844305B0421
:10EFD0005B0CA0F8443070471AB183899BB2194387
:10EFE00003E083899BB223EA01018181704700BF5E
:10EFF000818270470A43A0F8482070471AB183897C
:10F000009BB2194303E083899BB223EA010181810A
:10F01000704700BF038923F007031B041B0C038107
:10F02000704700BFB0F808C05FFA8CFC41EA0C0CD6
:10F0300042EA0C0C4CEA032C1FFA8CFCA0F808C026
:10F04000704700BF10B50446FFF7ECFF23899BB261
:10F0500043F48043238110BD10B50446FFF7E2FF5F
:10F06000238923F077031B041B0C43F077032381D0
:10F0700010BD00BF01858282704700BF038823F066
:10F0800070039B059B0D41EA03030380704700BF9B
:10F09000038923F070031B041B0C41EA0303038163
:10F0A000704700BF10B50446FFF7F2FF23899BB2FB
:10F0B00043F00703238110BD30B50489B0F818C0B0
:10F0C000058C2CF4407CADB22CF0030C24F007042A
:10F0D0004FEA0C4C25F0220542EA050524044FEACC
:10F0E0001C4C45EA0315240C4CF4807C21434CF065
:10F0F000010CADB20181A0F818C0058430BD00BF7D
:10F10000038B23F070031B041B0C41EA03030383EE
:10F11000704700BF038B23F4E0431B041B0C43EA3E
:10F1200001239BB203837047838B23F070031B047E
:10F130001B0C41EA03038383704700BF838B23F4D6
:10F14000E0431B041B0C43EA01239BB283837047FB
:10F1500021B103889BB243F0800304E0038823F0CD
:10F1600080039B059B0D0380704700BF21B18388FE
:10F170009BB243F0040304E0838823F004031B04E0
:10F180001B0C8380704700BF21B183889BB243F082
:10F19000080304E0838823F008031B041B0C83800E
:10F1A000704700BF21B183889BB243F0010304E0A4
:10F1B000838823F001031B041B0C8380704700BF6E
:10F1C000038B23F008031B041B0C41EA0303038396
:10F1D000704700BF038B23F400631B041B0C43EA3E
:10F1E00001239BB203837047838B23F008031B0426
:10F1F0001B0C41EA03038383704700BF838B23F416
:10F2000000631B041B0C43EA01239BB283837047FA
:10F21000038B23F004031B041B0C41EA0303038349
:10F22000704700BF038B23F480631B041B0C43EA6D
:10F2300001239BB203837047838B23F004031B04D9
:10F240001B0C41EA03038383704700BF838B23F4C5
:10F2500080631B041B0C43EA01239BB2838370472A
:10F26000038B23F080031B041B0C41EA030303837D
:10F27000704700BF038B5B045B0C43EA01239BB226
:10F2800003837047838B23F080031B041B0C41EA2C
:10F2900003038383704700BF838B5B045B0C43EAEB
:10F2A00001239BB283837047038C23F002031B046A
:10F2B0001B0C41EA03030384704700BF038C23F057
:10F2C00008031B041B0C41EA03030384704700BFBF
:10F2D000038C23F020031B041B0C43EA01139BB295
:10F2E00003847047038C23F080031B041B0C43EA48
:10F2F00001139BB203847047038C23F400731B0437
:10F300001B0C43EA01239BB203847047038C23F454
:10F3100000631B041B0C43EA01239BB20384704768
:10F32000038C23F400531B041B0C43EA01339BB2F0
:10F330000384704701238B408A40018C89B221EA03
:10F3400003030384018C0A4392B20284704700BF16
:10F3500004238B408A40018C89B221EA0303038491
:10F36000018C0A4392B20284704700BF01238B4094
:10F37000B0F820C010B51FFA8CFC2CEA03030384FC
:10F3800009B1082909D11830490844584FF68F733C
:10F3900004EA0303435043580CE004391830C1F326
:10F3A0004E01445848F6FF7304EA03034350120227
:10F3B000435892B243EA0202425010BD21B1038881
:10F3C0009BB243F0020304E0038823F002039B0591
:10F3D0009B0D0380704700BF21B103889BB243F0AF
:10F3E000040304E0038823F004039B059B0D0380C2
:10F3F000704700BF21B183889BB243F0800304E0D3
:10F40000838823F080031B041B0C8380704700BF9C
:10F41000038823F008039B059B0D038003889BB2A0
:10F4200041EA030303807047838823F070031B04C1
:10F430001B0C838083889BB241EA0303838070475F
:10F44000038923F007031B041B0C038103899BB270
:10F4500041EA030303817047038923F080031B04FF
:10F460001B0C038103899BB241EA030303817047AC
:10F470008184704781857047818670470187704716
:10F4800081877047A0F84010704700BF038B23F0BE
:10F490000C031B041B0C0383038B9BB241EA030385
:10F4A00003837047038B23F440631B041B0C03830B
:10F4B000038B9BB243EA01239BB20383704700BFD7
:10F4C000838B23F00C031B041B0C8383838B9BB265
:10F4D00041EA030383837047838B23F440631B0457
:10F4E0001B0C8383838B9BB243EA01239BB28383F0
:10F4F000704700BF0388DBB2038003889BB241EAF8
:10F5000003030380704700BF808E80B2704700BF46
:10F51000008F80B2704700BF808F80B2704700BFFD
:10F52000B0F8400080B27047808C80B2704700BF56
:10F53000008D80B2704700BF038A19420CBF0020C3
:10F5400001207047C94389B201827047038A8289CA
:10F5500011EA030092B203D011420CBF0020012037
:10F56000704700BFC94389B201827047B0F820C01C
:10F5700010B52CF0010C4FEA0C4C4FEA1C4CA0F8D3
:10F5800020C0048BB0F820C0A4B21FFA8CFC24F079
:10F59000F30442EA04042CF0020C44EA03144CF095
:10F5A000010C4CEA010CA4B20483A0F820C010BDE9
:10F5B000B0F820C010B52CF0100C4FEA0C4C4FEAFC
:10F5C0001C4CA0F820C0B0F818C0048C2CF4407C6F
:10F5D000A4B24FEA0C5C4FEA1C5C24F020044CEA15
:10F5E000022C44F010044CEA033C44EA01141FFAD4
:10F5F0008CFCA4B2A0F818C0048410BD38B50D4628
:10F60000602D1146044603D10122FFF7D1FF02E02D
:10F610000122FFF7ABFF29462046FFF739FD23897A
:10F620009BB243F00703238138BD00BFF8B50C46F9
:10F63000A2884988B4F800C0054600290CBF0227FB
:10F640000027012A0CBF022601262389BCF1000FE6
:10F6500010D1FFF78BFF2846E188FFF717FF2846F8
:10F66000394632462389FFF7A3FF2846E188FFF792
:10F6700019FF0FE0FFF79CFF2846E188FFF712FF14
:10F680002846394632462389FFF770FF2846E1882D
:10F69000FFF7FCFEF8BD00BF38B50B880C460546E9
:10F6A0004BB94988A2882389FFF760FF2846E18883
:10F6B000FFF7ECFE53E0042B09D14988A288238987
:10F6C000FFF776FF2846E188FFF7ECFE47E0082BBE
:10F6D000B1F802C0B1F804E0098920D1028C22F40B
:10F6E00080721204120C0284838B028C9BB292B241
:10F6F00023F0F30322F4007243EA011142EA0C2CD6
:10F7000089B21FFA8CFC41EA0E0E4CF4807CA0F802
:10F710001CE0A0F820C0E188FFF7D2FE1FE0028CB9
:10F7200022F480521204120C0284838B028C23F484
:10F73000407392B21B051B0D22F4005243EA0E23C4
:10F7400042EA0C3C43EA01331FFA8CFC9BB24CF4B6
:10F75000805C8383A0F820C0E188FFF7BDFE38BD40
:10F7600008B52D4B984237D00BD8A3F500639842CB
:10F7700026D003F58063984228D0B0F1804F4AD15B
:10F7800018E0264B984233D004D8A3F58063984202
:10F7900041D127E0224B984204D003F50063984200
:10F7A00039D12EE04FF400600121FFF715F84FF436
:10F7B00000602DE001200146FFF71CF801201CE04D
:10F7C00002200121FFF716F8022016E00420012193
:10F7D000FFF710F8042010E008200121FFF70AF8D5
:10F7E00008200AE010200121FFF704F8102004E0AF
:10F7F00020200121FEF7FEFF20200021FEF7FAFF66
:10F8000009E04FF400500121FEF7E6FF4FF40050ED
:10F810000021FEF7E1FF08BD000C0040001400408D
:10F82000002C0140002383814FF416528380C38053
:10F8300003814FF00C030260438170470A8810B5C2
:10F840004C88B1F804C0038AC98844EA020242EA3B
:10F850000C0223F470630A431B041B0C92B242EAAD
:10F860000303038210BD00BF0023C38003804380D5
:10F870008380704721B183899BB243F4005304E035
:10F88000838923F400531B041B0C8381704700BF42
:10F8900001F01F034FF0010CC1F3421161450CFA56
:10F8A00003F301D10C3004E0022901D1103000E053
:10F8B00014301AB1026842EA030302E0026822EA45
:10F8C00003030360704700BF1AB1838A9BB21943D8
:10F8D00003E0838A9BB223EA01018182704700BF63
:10F8E000038A23F00F031B041B0C0382038A9BB2C1
:10F8F00041EA030303827047838923F400631B04F6
:10F900001B0C838183899BB241EA03038381704787
:10F9100021B183899BB243F0020304E0838923F081
:10F9200002031B041B0C8381704700BF038A23F072
:10F9300020031B041B0C0382038A9BB241EA0303CE
:10F940000382704721B1038A9BB243F4804304E0F1
:10F95000038A23F480431B041B0C0382704700BFFF
:10F96000C905C90D818070478088C005C00D7047EA
:10F9700083899BB243F0010383817047038BDBB221
:10F980000383038B9BB243EA01230383704700BFC9
:10F99000038B03F47F430383038B9BB241EA03038E
:10F9A0000383704721B1838A9BB243F0200304E0B4
:10F9B000838A23F020031B041B0C8382704700BF43
:10F9C00021B1838A9BB243F0100304E0838A23F0C1
:10F9D00010031B041B0C8382704700BF21B1838A74
:10F9E0009BB243F0080304E0838A23F008031B045E
:10F9F0001B0C8382704700BF838A23F004031B041F
:10FA00001B0C8382838A9BB241EA03038382704783
:10FA100021B1838A9BB243F0020304E0838A23F07E
:10FA200002031B041B0C8382704700BF038819422A
:10FA30000CBF002001207047C94389B20180704784
:10FA40004FF0010CC1F3421201F01F0362450CFAA2
:10FA500003F301D1828903E0022A0CBF028A828A61
:10FA600092B21340028892B20BB9184607E0090A15
:10FA7000012313FA01F111420CBF0020012070474D
:10FA8000090A01238B40DB439BB20380704700BF10
:10FA9000038ACA8823F440531B041B0C13430382BC
:10FAA00083898A8830B5044608890D4623F4B0530B
:10FAB000498940EA020223F00C030A431B041B0C91
:10FAC00092B242EA0303A381A38AAA8923F4407372
:10FAD0001B041B0C134387B0A38201A8FEF70AFE88
:10FAE0000E4B2A689C420CBF049B039B192159436F
:10FAF00092006423B1FBF2F1B1FBF3F212011009A1
:10FB000003FB101109013231B1FBF3F303F00F03D2
:10FB100043EA020292B2228107B030BD00380140B0
:10FB200008B5214B98422BD008D8A3F50063984222
:10FB300016D003F58063984234D119E01B4B9842EC
:10FB400026D003F5684398422CD101214FF4804020
:10FB5000FEF742FE4FF480400021FEF73DFE21E01B
:10FB60004FF400300121FEF745FE4FF4003016E05F
:10FB70004FF480200121FEF73DFE4FF480200EE07F
:10FB80004FF400200121FEF735FE4FF4002006E07F
:10FB90004FF480100121FEF72DFE4FF4801000215C
:10FBA000FEF728FE08BD00BF004C0040005000409A
:10FBB000684620F007018D4601B5002303E00B499C
:10FBC0005958995004330A4A0A4998188842F6D37A
:10FBD000094B02E0002243F8042B084A9342F9D370
:10FBE000F4F700FBBDE8014085467047B8240108E2
:10FBF00000000020280200202802002064120020BB
:10FC000010B5074C20B922684FF00103138205E0BC
:10FC1000044B1B681B68984720680A3010BD00BF62
:10FC2000AC1100206811002010B50A4B0A4A1B686D
:10FC30005178DA7891420AD3997841B99C8834B9DD
:10FC40009A72064B1B685B689847204600E00220CA
:10FC500010BD00BFAC110020000100206811002081
:10FC600010B5074C20B922684FF00103138205E05C
:10FC7000044B1B689B68984720680C3010BD00BF80
:10FC8000AC1100206811002038B50E4C0E4B2268D4
:10FC90001B68D1789B695079984723689A7A7AB122
:10FCA00070B91A7962B99D7855B9084B1B68DB6841
:10FCB0009847236828465979DA78D9721A7300E090
:10FCC000022038BDAC110020441100206811002032
:10FCD00008B50246244B20B91B684FF00201198277
:10FCE00040E0224A4FF000011B681180197811F0A2
:10FCF0007F0113D15B7A13F0200F03D0117841F00C
:10FD00000201117013F0400F184B15BF1A781A78C2
:10FD100022F0010242F001021A701EE0012921D0F6
:10FD2000022901D000221DE0597911F0800F01F065
:10FD30000F0306D00E4951F8233003F03003102B87
:10FD400006E00B4951F8233003F44053B3F5805FCC
:10FD500003D1137843F001031370064B1B681B6932
:10FD60009847024A104608BDAC1100205C120020E2
:10FD7000005C00406811002010B51E4B19684A79DC
:10FD800012F0800F22F0800305D01B4850F82300AA
:10FD900000F0300004E0184850F8230000F4405010
:10FDA000164C94F800C0634522D24C8804BBF8B1CD
:10FDB000897AE9B112F0800F09D00F4948F6BF7275
:10FDC00051F8230000EA020282F0100208E00A491A
:10FDD0004BF68F7251F8230000EA020282F480523F
:10FDE00041F82320064B1B689B699847002000E0E0
:10FDF000022010BDAC110020005C0040000100207A
:10FE00006811002008B5064B1B685A7A42F02002A0
:10FE10005A72044B1B68DB699847002008BD00BF7D
:10FE2000AC11002068110020054B1A68538A18B9DC
:10FE30008988CB1A138201E008681818704700BF40
:10FE4000AC11002030B50E4B1C78002310E05FFA97
:10FE500083FC4FEA8C0202F1804202F5B842156839
:10FE600048F68F7105EA010141EA0C011160013386
:10FE7000A342ECD3034B40F08000186030BD00BFBC
:10FE8000000100204C5C0040704700BF08B50C4BDF
:10FE9000002093F82C1000F04FFE0A4B1B68187AD4
:10FEA000082807D1084B4FF480521A80074B4FF0B7
:10FEB00010021A80092814BF0020012008BD00BFCD
:10FEC0007C000020AC1100205E1200206012002097
:10FED00070B52D4B1C68237A032B01D0052B46D11E
:10FEE000A369228AABB1A2B1A58A954228BF154663
:10FEF00028469847228A638A521BEB1806462282BC
:10FF00006382002000F0E8FD2A460146304600F0FA
:10FF1000FBFB238A5BB11D4B4FF4405200201A803B
:10FF2000014600F0E7FD1A4B4FF030021A80A28A1A
:10FF3000238A9A4203D8144B03221B6803E0124A17
:10FF40001BB1136805221A720DE0126806211172A6
:10FF5000104A1168104A89B28A18520013600C4B7B
:10FF60004FF030021A80084B1B681B7A06E0072B03
:10FF700003D10A4B1B68DB6898470823024A1268C2
:10FF80001372FFF783FF70BDAC1100205E120020DA
:10FF900060120020505C004002300020441100201C
:10FFA000F8B5244B1C68238A267ABBB9042E15D1D8
:10FFB000214822490278012A0BD1214C214A246888
:10FFC0000370A0B28218520013604FF030020A8012
:10FFD0002BE04FF010030B80072626E0A68AA269CB
:10FFE0009E4234BF35461D462846B34294BF042680
:10FFF000022690470746002000F060FD2A46014691
:020000040801F1
:10000000384600F069FB2946002000F073FD638A42
:10001000228AEB186382094B551B4FF03002258270
:100020001A80094B4FF440521A80024B1B681E7213
:10003000F8BD00BFAC110020600700206012002056
:10004000505C0040023000205E12002008B5144BC6
:100050001B681A7A022A01D0042A05D1FFF7A0FFF3
:100060000F4B1B681B7A14E0062A11D15A78052A17
:100070000AD11A7812F07F0F06D1D878FFF7E2FE86
:10008000084B1B681B6A9847074B1B689B6898477F
:100090000823034A12681372FFF7F8FE08BD00BF79
:1000A000AC110020681100204411002038B5324BFB
:1000B0001B68187810F07F0004D15A7A22F02002D1
:1000C0005A7258E0022855D15A88002A52D11A791A
:1000D000002A4FD15A7912F0800F22F0800405D007
:1000E000264951F8241001F0300104E0234951F869
:1000F000241001F440512248007884423AD2002969
:1001000038D09B7A002B35D012F0800F0FD01B4BCC
:1001100053F8243003F03003102B25D1E4B22046ED
:1001200000F082FC2046302100F05EFB1CE0134D05
:1001300055F8243003F44053B3F5805F14D134B93B
:10014000104B204693F82C1000F0F6FC02E02046FD
:1001500000F056FC55F824204BF68F7302EA030397
:1001600083F4405345F82430074B1B685B6998477C
:10017000002000E0022038BDAC110020005C0040EF
:10018000000100207C00002068110020F7B58D4B95
:100190008D4E1A6835688D4B92B2D3182A7A5B005F
:1001A000092A1B681BD09BB203F1005303F540538F
:1001B0005B001C4614F8012B03F10A072A705B78D8
:1001C0006B70B4F8030000F063FE6880B4F80700B9
:1001D000346800F05DFEA08033687F88DF807A4C51
:1001E00001212368DA8819725D78002A62D11A78B1
:1001F00012F07F022ED1092D02D1FFF715FD3BE051
:10020000052D0DD193F90320002A4EDB9A78002AA0
:100210004BD19A88002A48D19B7A002B37D044E0F2
:10022000032D0BD1DA78012A27D19A882ABB5B7A71
:1002300013F0200F21D0FFF7E5FD1DE0012D1CD1AB
:10024000DA78012A19D19A88BAB95B7A13F0200FAB
:1002500013D00AE0012A04D10B2D0ED1FFF714FDB3
:100260000AE0022A09D1012D02D1FFF71FFF03E0A6
:10027000032D02D1FFF780FD48B1554B28461B687E
:100280005B699847032801D109230FE068B94D4AFB
:10029000504B12684FF0300192B2D3185B0000222D
:1002A0001A604D4B1980062300E00823464A126865
:1002B0001372E3E0062D18D11A7812F07F0F40F088
:1002C00097809B78012B03D1414B1B68DB696EE063
:1002D000022B03D13E4B1B681B6A68E0032B40F0E6
:1002E00087803B4B1B685B6A61E0002D3CD15988DD
:1002F00000297DD15A6822F47F42B2F5003F77D1C0
:100300001A7812F07F0203D19B88002B70D129E06C
:10031000012A0BD158792E4B1B689B6998470028FE
:1003200066D123689B7A002B62D01BE0022A5FD142
:100330005B7913F0800F03F00F0205D0274951F8C5
:10034000221001F0300104E0244951F8221001F498
:1003500040512348007882424AD213F0700F47D1AF
:10036000002945D01F4B23E0082D05D11B7813F041
:100370007F0F3DD11C4B1BE00A2D39D11A7802F0BA
:100380007F02012A34D19A7A002A31D05988002973
:100390002ED15A6822F47F42B2F5803F28D1587995
:1003A0000B4B1B689B69984710BB104B00E0FBB1DF
:1003B000054A4FF00001126800209361518298476E
:1003C000002020E0505C0040AC11002004300020F0
:1003D000441100200230002060120020005C004028
:1003E00000010020D1FC000801FC000861FC0008AD
:1003F000244C254B22681B6850781B6998470328BA
:1004000001D1236806E01F4B4FF6FF711B681A8A63
:100410008A4201D1092203E0022800D012B9082241
:100420001A722BE093F90010002921DAD988019182
:100430000198824202D9019A1A8211E08A420FD2AF
:100440001149096891F82C108A4201D2002105E077
:1004500092FBF1F001FB102212B901210B4A11703D
:10046000094A126892F82C209A82FFF799FD05E05C
:1004700003221A72064B4FF440521A80FFF706FD12
:10048000FEBD00BFAC110020441100206007002019
:100490005E120020074A022108B507481172074979
:1004A000074B086007490A60074A13601B689847B2
:1004B00008BD00BF4C11002004010020681100207D
:1004C0007C000020AC1100204411002008B529E078
:1004D00047F6FF700860198801F00F018B0003F1E7
:1004E0008043117003F5B843196889B211F4004FC5
:1004F00009D0186840F68F7100EA0101196012787E
:100500000E4B013A0BE011F0800F0BD0186848F643
:100510000F7100EA010119601278094B013A53F892
:10052000223098470749084B0868084A80B218806B
:10053000188800B20028CBDB08BD00BFE400002013
:10054000C8000020445C00404211002048110020F7
:10055000F8B59AE047F6FF761E601688564F06F00B
:100560000F06B30003F1804303F5B8433E70002E3D
:1005700064D127682668236807F4405C03EA00001A
:1005800080F400502060236806F0300003EA010187
:1005900081F0200121601388484A13F0100F108069
:1005A000A5F800C004D023689BB213F0800F08D0D8
:1005B000226848F60F7302EA03032360FFF746FD43
:1005C00016E013F4006F08D0226840F68F7302EA39
:1005D00003032360FFF7DAFD0AE013F4004F54D061
:1005E000226840F68F7302EA03032360FFF770FC72
:1005F00021682A884BF68F7301EA030312F4805FA7
:1006000018BF83F4805312F4005F2D4A18BF83F49F
:1006100000531360294B11681A8848F6BF7301EA2A
:10062000030312F0100F18BF83F0100312F0200F15
:10063000234A18BF83F0200313603BE01C68A4B278
:1006400014F4004F0BD0196840F68F7201EA0202D1
:100650001A603A781B4B013A53F82230984714F04D
:10066000800F12D0144948F60F720B789B0003F1EB
:10067000804303F5B843186800EA02021A600A785A
:10068000114B013A53F822309847104B104A1D681D
:100690000B4C1FFA85FCA2F800C0B2F800C04BF664
:1006A0008F700FFA8CFCBCF1000F48F6BF71094D3A
:1006B000FFF650AFF8BD00BF4811002060120020C7
:1006C000005C0040E4000020C8000020445C0040C2
:1006D000421100205E12002001F10051013201F5AB
:1006E000405110B549005208002308E010F803C03B
:1006F0006478013A4CEA042C21F813C00233C41880
:10070000002AF3D110BD00BF01F10051013201F503
:10071000405110B549005208002304E031F813405D
:10072000013AC4520233002AF8D110BD014B1860BF
:10073000704700BF405C0040014B186880B27047B2
:10074000405C0040014B1860704700BF445C0040B3
:10075000014B186880B27047445C0040014B186838
:1007600080B27047485C0040014B1860704700BF82
:100770004C5C0040014B186880B270474C5C0040F4
:100780004FF6F873024A00EA03031360704700BF94
:10079000505C0040014B186880B27047505C0040CC
:1007A000014B43F820107047005C0040024B53F8A7
:1007B000200080B2704700BF005C0040054B10B5C0
:1007C00053F8204048F68F1204EA02020A4343F825
:1007D000202010BD005C0040024B53F8200000F4C4
:1007E000C0607047005C00400A4B10B553F82020F1
:1007F00048F6BF7402EA040411F0100F18BF84F029
:10080000100411F0200F18BF84F0200443F820409A
:1008100010BD00BF005C00400A4B10B553F820200B
:100820004BF68F7402EA040411F4805F18BF84F45D
:10083000805411F4005F18BF84F4005443F8204042
:1008400010BD00BF005C004038B50D460446FFF700
:10085000ADFF012D02D120F4805003E0022D04D120
:1008600020F01000014B43F8240038BD005C00402C
:10087000024B53F8200000F030007047005C00404D
:10088000024B53F8200000F440507047005C0040D9
:10089000054B48F6BF7253F8201001EA020282F0BD
:1008A000300243F820207047005C0040054B4BF6B7
:1008B0008F7253F8201001EA020282F4405243F88A
:1008C00020207047005C0040054B48F68F6253F8CB
:1008D000201001EA020242F4807243F8202070479F
:1008E000005C0040044B48F68F6253F8201001EA88
:1008F000020243F820207047005C0040044B48F699
:100900008F6253F8201001EA020243F8202070475A
:10091000005C0040054B48F68F6253F8201001EA56
:10092000020242F4807243F820207047005C0040CD
:10093000054B48F68F6253F8201001EA020242F498
:10094000807243F820207047005C0040044B48F65A
:100950008F6253F8201001EA020243F8202070470A
:10096000005C0040044B53F8200000F030001028D9
:1009700014BF002001207047005C0040054B53F875
:10098000200000F44050B0F5805F14BF002001202B
:10099000704700BF005C0040044B40F68F7253F874
:1009A000201001EA020243F820207047005C00405A
:1009B000044B48F60F7253F8201001EA020243F884
:1009C00020207047005C0040054B48F68F7253F8BA
:1009D000201001EA020242F4804243F820207047CE
:1009E000005C0040054B48F68F7253F8201001EA76
:1009F000020242F0400243F820207047005C0040B1
:100A0000084B53F8202012F4804F09D053F82010DF
:100A100048F68F7201EA020242F4804243F8202035
:100A2000704700BF005C0040084B53F8202012F0D4
:100A3000400F09D053F8201048F68F7201EA0202E5
:100A400042F0400243F82020704700BF005C0040A5
:100A5000054B10B553F8204048F68F7204EA0202A5
:100A60000A4343F8202010BD005C0040024B53F8BD
:100A7000200000F00F007047005C0040064B490862
:100A80001B6849009BB203EBC00303F1005303F55D
:100A900040535B0019607047505C0040054A064BAC
:100AA0001268490892B202EBC002D3185B004900F9
:100AB00019607047505C004004300020054B1B68F3
:100AC0009BB203EBC00303F1005303F540535B00FB
:100AD00018887047505C0040044A054B126892B277
:100AE00002EBC002D3185B0018887047505C0040CE
:100AF00004300020044A054B126892B202EBC00297
:100B0000D3185B0019607047505C00400230002031
:100B10003E2909D94B0911F01F0F01D1013B9BB2AE
:100B20009B0243F4004305E04B0811F0010F18BF8E
:100B300001339B02036070470D4A0E4B126892B25C
:100B4000D31803EBC0035B003E2909D94A0911F011
:100B50001F0F01D1013A92B2920242F4004205E025
:100B60004A0811F0010F18BF013292021A60704753
:100B7000505C004006300020054A064B126892B2D5
:100B800002EBC002D3185B0018688005800D704727
:100B9000505C004002300020054A064B126892B2B9
:100BA00002EBC002D3185B0018688005800D704707
:100BB000505C0040063000200C4B30B51D681C68AE
:100BC000C0001FFA85FC8444A4B2094B00190CF143
:100BD000005CC3180CF5405C490852084FEA4C0011
:100BE00049005B00520001601A6030BD505C00405B
:100BF00004300020064B49081B6849009BB203EBF8
:100C0000C00303F1005303F540535B0019607047C4
:100C1000505C0040054A064B1268490892B202EB4C
:100C2000C002D3185B00490019607047505C004057
:100C300004300020054B1B689BB203EBC00303F19B
:100C4000005303F540535B0018887047505C004028
:100C5000044A054B126892B202EBC002D3185B0043
:100C600018887047505C004004300020012910B5FE
:100C700024D1254B25491B68C0009BB2591809187F
:100C80004B003E2A09D9510912F01F0F01D1013939
:100C900089B2890241F4004105E0510812F0010FC8
:100CA00018BF0131890219601749194B096889B2C7
:100CB000CB18181840003E2A1ED913E0022922D171
:100CC000114BC0001C681B68A4B21FFA83FC0F49BB
:100CD0000F4B844400194118634449005B000A60CB
:100CE0001A6010E0530912F01F0F01D1013B9BB2B3
:100CF0009B0243F4004305E0530812F0010F18BFB4
:100D000001339B02036010BD505C004002300020A4
:100D10000630002001291BD11349144B096889B200
:100D2000CB1803EBC00040003E2A09D9530912F04A
:100D30001F0F01D1013B9BB29B0243F4004305E02E
:100D4000530812F0010F18BF01339B0203600AE041
:100D5000022908D10449054B096889B201EBC0009A
:100D6000C3185B001A607047505C004002300020DE
:100D700001291BD11349144B096889B2CB1803EB25
:100D8000C00040003E2A09D9530912F01F0F01D1BB
:100D9000013B9BB29B0243F4004305E0530812F071
:100DA000010F18BF01339B0203600AE0022908D13A
:100DB0000449054B096889B201EBC000C3185B0008
:100DC0001A607047505C004006300020054A064B10
:100DD000126892B202EBC002D3185B00186880055B
:100DE000800D7047505C004002300020054A064BE1
:100DF000126892B202EBC002D3185B00186880053B
:100E0000800D7047505C0040063000200D4BC00044
:100E100019680D4A89B241188A185200128812F4D2
:100E20007C4F01D001200CE01A68084B92B2801868
:100E3000C3185B0018888005800D002814BF0220AD
:100E400000207047505C0040063000200230002037
:100E5000012909D10B4A48F68F7352F8201001EA94
:100E6000030343F040030AE002290AD1054A48F689
:100E70008F7352F8201001EA030343F4804342F8D1
:100E800020307047005C004041EA0020704700BFFE
:100E9000030AC0B243EA0020704700BF08B5002231
:100EA0000A2300F045F808BD08B500210A2200F029
:100EB000DFF808BDF0B40378002B2DD040F23012DB
:100EC000C2F20002156802E010F8013FEBB15A19B6
:100ED00003F12004527812F001070A7808BF1C467B
:100EE00001F10101561C9446AE5D16F0010F18BFCA
:100EF00002F1200C6445E7D007B1203316F0010F52
:100F000018BF2032981AF0BC70470A786F78561CC8
:100F100007F00107AE5DEFE740F230100A78C2F249
:100F20000000561C05686F78AE5D07F00107E3E727
:100F30002DE9F04F40F23015C2F2000583B00C46A7
:100F40001F46D5F800800E460190009216F8015B0E
:100F500008EB050393F801B01BF0080BF6D12D2D1B
:100F600065D02B2D08BF16F8015BD7F1010338BF00
:100F70000023102F14BF1A4643F0010232B1302D66
:100F800066D01BB1302D0CBF08270A27BBF1000F1C
:100F9000394614BF4FF000496FF00049484600F051
:100FA000A5F948468A46394600F072F800218C4679
:100FB00008EB0502A5F13003527812F0040F08D1B6
:100FC00012F0030F20D012F0010F14BF3723572364
:100FD000EB1A9F4218DD844594BF0022012252EA99
:100FE000D1714FF0FF310CD1844514BF0022012292
:100FF0005345D4BF002202F0010212B907FB0C3C9A
:10100000012116F8015BD3E7B1F1FF3F14D0BBF12A
:10101000000F09D16046009B1BB101B1741E009AFC
:10102000146003B0BDE8F08FCCF10000F3E716F8D0
:10103000015B4FF0010B98E7019ABBF1000F4FF0F5
:10104000220314BF4FF000406FF000401360E2E74E
:101050003278782A14BF00210121582A14BF0A4689
:1010600041F00102002A8CD07578102702368DE7F6
:1010700010B540F23414C2F200048C461346014607
:1010800062462068FFF754FF10BD00BF000000005B
:101090004A1E08BF7047C0F02481884240F2168182
:1010A000114200F01781B0FA80F3B1FA81F2A2EB9D
:1010B0000303C3F11F0304A202EB03134FF000026A
:1010C0009F4600BFAFF30080B0EBC17F00BF42EB93
:1010D000020228BFA0EBC170B0EB817F00BF42EBE2
:1010E000020228BFA0EB8170B0EB417F00BF42EB52
:1010F000020228BFA0EB4170B0EB017F00BF42EBC2
:10110000020228BFA0EB0170B0EBC16F00BF42EB41
:10111000020228BFA0EBC160B0EB816F00BF42EBC1
:10112000020228BFA0EB8160B0EB416F00BF42EB31
:10113000020228BFA0EB4160B0EB016F00BF42EBA1
:10114000020228BFA0EB0160B0EBC15F00BF42EB21
:10115000020228BFA0EBC150B0EB815F00BF42EBA1
:10116000020228BFA0EB8150B0EB415F00BF42EB11
:10117000020228BFA0EB4150B0EB015F00BF42EB81
:10118000020228BFA0EB0150B0EBC14F00BF42EB01
:10119000020228BFA0EBC140B0EB814F00BF42EB81
:1011A000020228BFA0EB8140B0EB414F00BF42EBF1
:1011B000020228BFA0EB4140B0EB014F00BF42EB61
:1011C000020228BFA0EB0140B0EBC13F00BF42EBE1
:1011D000020228BFA0EBC130B0EB813F00BF42EB61
:1011E000020228BFA0EB8130B0EB413F00BF42EBD1
:1011F000020228BFA0EB4130B0EB013F00BF42EB41
:10120000020228BFA0EB0130B0EBC12F00BF42EBC0
:10121000020228BFA0EBC120B0EB812F00BF42EB40
:10122000020228BFA0EB8120B0EB412F00BF42EBB0
:10123000020228BFA0EB4120B0EB012F00BF42EB20
:10124000020228BFA0EB0120B0EBC11F00BF42EBA0
:10125000020228BFA0EBC110B0EB811F00BF42EB20
:10126000020228BFA0EB8110B0EB411F00BF42EB90
:10127000020228BFA0EB4110B0EB011F00BF42EB00
:10128000020228BFA0EB0110B0EBC10F00BF42EB80
:10129000020228BFA0EBC100B0EB810F00BF42EB00
:1012A000020228BFA0EB8100B0EB410F00BF42EB70
:1012B000020228BFA0EB4100B0EB010F00BF42EBE0
:1012C000020228BFA0EB0100104670470CBF0120AE
:1012D00000207047B1FA81F2C2F11F0220FA02F039
:1012E000704708B14FF0FF3000F00EB80029F8D079
:1012F0002DE90340FFF7CCFEBDE8064002FB00F3FA
:10130000A1EB0301704700BF704700BF81F00041AF
:1013100002E000BF83F0004330B54FEA41044FEADA
:10132000430594EA050F08BF90EA020F1FBF54EA75
:10133000000C55EA020C7FEA645C7FEA655C00F011
:10134000E2804FEA5454D4EB5555B8BF6D420CDDE2
:101350002C4480EA020281EA030382EA000083EA65
:10136000010180EA020281EA0303362D88BF30BD05
:1013700011F0004F4FEA01314FF4801C4CEA11315B
:1013800002D0404261EB410113F0004F4FEA0333BA
:101390004CEA133302D0524263EB430394EA050F45
:1013A00000F0A780A4F10104D5F1200E0DDB02FAB4
:1013B0000EFC22FA05F2801841F1000103FA0EF248
:1013C000801843FA05F359410EE0A5F120050EF10E
:1013D000200E012A03FA0EFC28BF4CF0020C43FA3F
:1013E00005F3C01851EBE37101F0004507D54FF04C
:1013F000000EDCF1000C7EEB00006EEB0101B1F59C
:10140000801F1BD3B1F5001F0CD349085FEA3000E1
:101410004FEA3C0C04F101044FEA445212F5800FEC
:1014200080F09A80BCF1004F08BF5FEA500C50F189
:10143000000041EB045141EA050130BD5FEA4C0C6C
:10144000404141EB010111F4801FA4F10104E9D1F5
:1014500091F0000F04BF01460020B1FA81F308BFEC
:101460002033A3F10B03B3F120020CDA0C3208DDB8
:1014700002F1140CC2F10C0201FA0CF021FA02F193
:101480000CE002F11402D8BFC2F1200C01FA02F103
:1014900020FA0CFCDCBF41EA0C019040E41AA2BF28
:1014A00001EB0451294330BD6FEA04041F3C1CDAF0
:1014B0000C340EDC04F11404C4F1200220FA04F010
:1014C00001FA02F340EA030021FA04F345EA0301BA
:1014D00030BDC4F10C04C4F1200220FA02F001FA7C
:1014E00004F340EA0300294630BD21FA04F02946FE
:1014F00030BD94F0000F83F4801306BF81F4801197
:101500000134013D4EE77FEA645C18BF7FEA655C09
:1015100029D094EA050F08BF90EA020F05D054EADB
:10152000000C04BF1946104630BD91EA030F1EBFE0
:101530000021002030BD5FEA545C05D140004941E4
:1015400028BF41F0004130BD14F580043CBF01F5D7
:10155000801130BD01F0004545F0FE4141F47001BD
:101560004FF0000030BD7FEA645C1ABF1946104698
:101570007FEA655C1CBF0B46024650EA013406BF99
:1015800052EA033591EA030F41F4002130BD00BF58
:1015900090F0000F04BF0021704730B54FF4806415
:1015A00004F132044FF000054FF0000150E700BF96
:1015B00090F0000F04BF0021704730B54FF48064F5
:1015C00004F1320410F0004548BF40424FF00001E2
:1015D0003EE700BF42004FEAE2014FEA31014FEA25
:1015E00002701FBF12F07F4393F07F4F81F0605174
:1015F000704792F0000F14BF93F07F4F704730B5E3
:101600004FF4607401F0004521F0004120E700BF75
:1016100050EA010208BF704730B54FF000050AE0FC
:1016200050EA010208BF704730B511F0004502D5FD
:10163000404261EB41014FF4806404F132045FEAFF
:10164000915C3FF4DCAE4FF003025FEADC0C18BFA4
:1016500003325FEADC0C18BF033202EBDC02C2F19A
:10166000200300FA03FC20FA02F001FA03FE40EA2C
:101670000E0021FA02F11444C1E600BF70B54FF02C
:10168000FF0C4CF4E06C1CEA11541DBF1CEA13550E
:1016900094EA0C0F95EA0C0F00F0DEF82C4481EA76
:1016A000030621EA4C5123EA4C5350EA013518BF96
:1016B00052EA033541F4801143F4801338D0A0FB83
:1016C00002CE4FF00005E1FB02E506F00042E0FB30
:1016D00003E54FF00006E1FB03569CF0000F18BF36
:1016E0004EF0010EA4F1FF04B6F5007F64F54074DE
:1016F00004D25FEA4E0E6D4146EB060642EAC62171
:1017000041EA55514FEAC52040EA5E504FEACE2EDD
:10171000B4F1FD0C88BFBCF5E06F1ED8BEF1004FE0
:1017200008BF5FEA500E50F1000041EB045170BD5C
:1017300006F0004646EA010140EA020081EA0301A0
:10174000B4EB5C04C2BFD4EB0C0541EA045170BD9C
:1017500041F480114FF0000E013C00F3AB8014F116
:10176000360FDEBF002001F0004170BDC4F100045F
:10177000203C35DA0C341BDC04F11404C4F12005E0
:1017800000FA05F320FA04F001FA05F240EA02003B
:1017900001F0004221F0004110EBD37021FA04F671
:1017A00042EB06015EEA430E08BF20EAD37070BD2B
:1017B000C4F10C04C4F1200500FA04F320FA05F08A
:1017C00001FA04F240EA020001F0004110EBD3708C
:1017D00041F100015EEA430E08BF20EAD37070BDFC
:1017E000C4F1200500FA05F24EEA020E20FA04F3D5
:1017F00001FA05F243EA020321FA04F001F0004184
:1018000021FA04F220EA020000EBD3705EEA430EF4
:1018100008BF20EAD37070BD94F0000F0FD101F023
:101820000046400041EB010111F4801F08BF013C5C
:10183000F7D041EA060195F0000F18BF704703F09A
:101840000046520043EB030313F4801F08BF013D21
:10185000F7D043EA0603704794EA0C0F0CEA1355DD
:1018600018BF95EA0C0F0CD050EA410618BF52EA97
:101870004306D1D181EA030101F000414FF000009D
:1018800070BD50EA410606BF1046194652EA4306AB
:1018900019D094EA0C0F02D150EA013613D195EA1F
:1018A0000C0F05D152EA03361CBF104619460AD167
:1018B00081EA030101F0004141F0FE4141F4700171
:1018C0004FF0000070BD41F0FE4141F4780170BD61
:1018D00070B54FF0FF0C4CF4E06C1CEA11541DBFC6
:1018E0001CEA135594EA0C0F95EA0C0F00F0A7F8C8
:1018F000A4EB050481EA030E52EA03354FEA0131F5
:1019000000F088804FEA03334FF0805545EA131307
:1019100043EA12634FEA022245EA111545EA1065CF
:101920004FEA00260EF000419D4208BF964244F166
:10193000FD0404F5407402D25B084FEA3202B61A85
:1019400065EB03055B084FEA32024FF480104FF459
:10195000002CB6EB020E75EB030E22BFB61A7546CD
:1019600040EA0C005B084FEA3202B6EB020E75EB60
:10197000030E22BFB61A754640EA5C005B084FEAC8
:101980003202B6EB020E75EB030E22BFB61A754695
:1019900040EA9C005B084FEA3202B6EB020E75EBA0
:1019A000030E22BFB61A754640EADC0055EA060E61
:1019B00018D04FEA051545EA16754FEA06164FEAA4
:1019C000C30343EA52734FEAC2025FEA1C1CC0D150
:1019D00011F4801F0BD141EA00014FF000004FF0DD
:1019E000004CB6E711F4801F04BF01430020B4F19E
:1019F000FD0C88BFBCF5E06F3FF6AFAEB5EB030C56
:101A000004BFB6EB020C5FEA500C50F1000041EB52
:101A1000045170BD0EF0004E4EEA113114EB5C041F
:101A2000C2BFD4EB0C0541EA045170BD41F48011F2
:101A30004FF0000E013C90E645EA060E8DE60CEAFA
:101A4000135594EA0C0F08BF95EA0C0F3FF43BAF17
:101A500094EA0C0F0AD150EA01347FF434AF95EACE
:101A60000C0F7FF425AF104619462CE795EA0C0FB2
:101A700006D152EA03353FF4FDAE1046194622E77F
:101A800050EA410618BF52EA43067FF4C5AE50EA59
:101A900041047FF40DAF52EA43057FF4EBAE12E749
:101AA0004FEA410212F5001215D211D56FF4787386
:101AB000B3EB625212D94FEAC12343F0004343EA29
:101AC000505311F0004F23FA02F018BF4042704704
:101AD0004FF00000704750EA013005D111F000408E
:101AE00008BF6FF0004070474FF00000704700BF24
:101AF0004FEA4102B2F1E04324BFB3F5001CDCF130
:101B0000FE5C0DD901F0004C4FEAC0024CEA507067
:101B1000B2F1004F40EB830008BF20F00100704796
:101B200011F0804F21D113F13872BCBF01F0004099
:101B3000704741F480114FEA5252C2F11802C2F1CB
:101B4000200C10FA0CF320FA02F018BF40F001004C
:101B50004FEAC1234FEAD32303FA0CFC40EA0C00FE
:101B600023FA02F34FEA4303CCE77FEA625307D13B
:101B700050EA01331EBF4FF0FE4040F44000704772
:101B800001F0004040F0FE4040F40000704700BF0C
:101B900080F0004002E000BF81F0004142001FBF22
:101BA0005FEA410392EA030F7FEA226C7FEA236C2B
:101BB0006AD04FEA1262D2EB1363C1BFD218414020
:101BC00048404140B8BF5B42192B88BF704710F0B6
:101BD000004F40F4000020F07F4018BF404211F059
:101BE000004F41F4000121F07F4118BF494292EAC1
:101BF000030F3FD0A2F1010241FA03FC10EB0C00ED
:101C0000C3F1200301FA03F100F0004302D5494279
:101C100060EB4000B0F5000F13D3B0F1807F06D326
:101C200040084FEA310102F10102FE2A51D2B1F11E
:101C3000004F40EBC25008BF20F0010040EA030013
:101C40007047490040EB000010F4000FA2F10102C0
:101C5000EDD1B0FA80FCACF1080CB2EB0C0200FA4A
:101C60000CF0AABF00EBC25052421843BCBFD04098
:101C70001843704792F0000F81F4000106BF80F412
:101C800000000132013BB5E74FEA41037FEA226CD5
:101C900018BF7FEA236C21D092EA030F04D092F0A0
:101CA000000F08BF0846704790EA010F1CBF0020D4
:101CB000704712F07F4F04D1400028BF40F0004031
:101CC000704712F100723CBF00F50000704700F051
:101CD000004343F0FE4040F4000070477FEA226278
:101CE00016BF08467FEA23630146420206BF5FEA49
:101CF000412390EA010F40F4800070474FF0000349
:101D000004E000BF10F0004348BF40425FEA000C0F
:101D100008BF704743F0964301464FF000001CE0B7
:101D200050EA010208BF70474FF000030AE000BF0D
:101D300050EA010208BF704711F0004302D540424B
:101D400061EB41015FEA010C02BF844601460020BD
:101D500043F0B64308BFA3F18053A3F50003BCFAD8
:101D60008CF2083AA3EBC25310DB01FA02FC634485
:101D700000FA02FCC2F12002BCF1004F20FA02F28C
:101D800043EB020008BF20F00100704702F120027F
:101D900001FA02FCC2F1200250EA4C0021FA02F2E0
:101DA00043EB020008BF20EADC7070474FF0FF0CE5
:101DB0001CEAD0521EBF1CEAD15392EA0C0F93EAE0
:101DC0000C0F6FD01A4480EA010C400218BF5FEA82
:101DD00041211ED04FF0006343EA501043EA5111F5
:101DE000A0FB01310CF00040B1F5000F3EBF4900EF
:101DF00041EAD3715B0040EA010062F17F02FD2AF3
:101E00001DD8B3F1004F40EBC25008BF20F00100D5
:101E1000704790F0000F0CF0004C08BF49024CEAEC
:101E2000502040EA51207F3AC2BFD2F1FF0340EA7E
:101E3000C250704740F400004FF00003013A5DDCEF
:101E400012F1190FDCBF00F000407047C2F1000230
:101E5000410021FA02F1C2F1200200FA02FC5FEA1D
:101E6000310040F1000053EA4C0308BF20EADC7067
:101E7000704792F0000F00F0004C02BF400010F4D9
:101E8000000F013AF9D040EA0C0093F0000F01F086
:101E9000004C02BF490011F4000F013BF9D041EAA8
:101EA0000C018FE70CEAD15392EA0C0F18BF93EAAA
:101EB0000C0F0AD030F0004C18BF31F0004CD8D1D4
:101EC00080EA010000F00040704790F0000F17BF5B
:101ED00090F0004F084691F0000F91F0004F14D0A1
:101EE00092EA0C0F01D142020FD193EA0C0F03D1F9
:101EF0004B0218BF084608D180EA010000F00040FC
:101F000040F0FE4040F40000704740F0FE4040F4D6
:101F1000400070474FF0FF0C1CEAD0521EBF1CEA75
:101F2000D15392EA0C0F93EA0C0F69D0A2EB030293
:101F300080EA010C49024FEA402037D04FF080532D
:101F400043EA111143EA10130CF000408B4238BFF2
:101F50005B0042F17D024FF4000C8B4224BF5B1A00
:101F600040EA0C00B3EB510F24BFA3EB510340EA4E
:101F70005C00B3EB910F24BFA3EB910340EA9C00FC
:101F8000B3EBD10F24BFA3EBD10340EADC001B016C
:101F900018BF5FEA1C1CE0D1FD2A3FF650AF8B4210
:101FA00040EBC25008BF20F0010070470CF0004C1D
:101FB0004CEA50207F32C2BFD2F1FF0340EAC25048
:101FC000704740F400004FF00003013A37E792F009
:101FD000000F00F0004C02BF400010F4000F013A67
:101FE000F9D040EA0C0093F0000F01F0004C02BF62
:101FF000490011F4000F013BF9D041EA0C0195E7CB
:102000000CEAD15392EA0C0F08D142027FF47DAF63
:1020100093EA0C0F7FF470AF084676E793EA0C0F53
:1020200004D14B023FF44CAF08466EE730F0004C51
:1020300018BF31F0004CCAD130F000427FF45CAFE1
:1020400031F000437FF43CAF5FE700BF4FF0FF3C4F
:1020500006E000BF4FF0010C02E000BF4FF0010CA2
:102060004DF804CD4FEA40024FEA41037FEA226C6B
:1020700018BF7FEA236C11D001B052EA530C18BF8D
:1020800090EA010F58BFB2EB030088BFC81738BFF2
:102090006FEAE17018BF40F0010070477FEA226CE0
:1020A00002D15FEA402C05D17FEA236CE4D15FEADC
:1020B000412CE1D05DF8040B704700BF8446084610
:1020C0006146FFE70FB5FFF7C9FF002848BF10F1D1
:1020D000000F0FBD4DF808EDFFF7F4FF0CBF012016
:1020E00000205DF808FB00BF4DF808EDFFF7EAFFA0
:1020F00034BF012000205DF808FB00BF4DF808ED5B
:10210000FFF7E0FF94BF012000205DF808FB00BF4F
:102110004DF808EDFFF7D2FF94BF012000205DF8D5
:1021200008FB00BF4DF808EDFFF7C8FF34BF0120E2
:1021300000205DF808FB00BF42000ED2B2F1FE4F56
:102140000BD34FF09E03B3EB126209D44FEA002386
:1021500043F0004323FA02F070474FF0000070474D
:1021600012F1610F01D1420202D14FF0FF307047EE
:102170004FF00000704700BF0000000000000000AA
:10218000010003E80000000000000003E800000078
:1021900000000200FA0600030000000000370600FD
:1021A0000000000000000000F401000064000000D6
:1021B000018008080000000000020000000000008C
:1021C00000000000C80000001201100102000040E1
:1021D000D016500601140102030100000902430059
:1021E000020100C0320904000001020201000524BE
:1021F0000010010524010001042402020524060048
:1022000001070582030800FF09040100020A00001B
:10221000000705030240000007058102400000009E
:102220000403090426035400720069006E00610073
:102230006D00690063004D006F00740069006F005D
:102240006E002000430074006C0000003203540054
:102250004D0043004D002D003600310031003000AC
:10226000200028007600690072007400750061008B
:102270006C00200043004F004D00290020000000AA
:102280000102030405060000524F520000010652ED
:102290004F4C000002064D5354000003024D5650AF
:1022A000000004075341500000050747415000005B
:1022B0000603535441500007035253415000080392
:1022C0005347500000090747475000000A03535482
:1022D0004750000B0352534750000C035246530023
:1022E000000D0353494F00000E0747494F00000FF0
:1022F0000353414300001D0753434F00001E07478F
:10230000434F00001F0343434F0000200341434F4E
:1023100000002703554630000040075546310000B5
:102320004107554632000042075546330000430737
:1023300055463400004407554635000045075546CC
:1023400036000046075546370000470752554E00F5
:1023500000810553544F5000800042494E00008BCD
:10236000000000000000000002000000000000016A
:10237000000000000102030401020304060708092B
:1023800002040608002020202020202020202828C9
:102390002828282020202020202020202020202025
:1023A0002020202020881010101010101010101065
:1023B0001010101010040404040404040404041095
:1023C0001010101010104141414141410101010123
:1023D00001010101010101010101010101010101ED
:1023E00010101010101042424242424202020202F9
:1023F00002020202020202020202020202020202BD
:10240000101010102000000000000000000000006C
:1024100000000000000000000000000000000000BC
:1024200000000000000000000000000000000000AC
:10243000000000000000000000000000000000009C
:10244000000000000000000000000000000000008C
:10245000000000000000000000000000000000007C
:10246000000000000000000000000000000000006C
:10247000000000000000000000000000000000005C
:10248000000000000000000036313130563132309B
:10249000004142530052454C00434F4F52440053B9
:1024A000544152540053544F5000535441545553C7
:0824B0000000000043000000E1
:1024B8008824010800010200000800000100000053
:1024C8000200000000000000000000000000000002
:1024D80000000000000000000000000000000000F4
:1024E80000000000000000000000000000000000E4
:1024F8000000000000C201000000080020220108BE
:102508000400000024220108260000004C220108D3
:1025180032000000AC0000201A000000DC21010895
:1025280043000000C82101081200000035A000087F
:102538003D9E00084D9C0008619C0008659C0008B1
:10254800C59C0008E99C00082D9E00081D9E0008F7
:10255800F99D000800000000400000001A03540024
:102568004D0043003600310031003000000000000B
:1025780000000000000000004D9B000889FE0008D4
:1025880089FE000889FE000889FE000889FE000807
:1025980089FE000889FE000889FE00088D9F000852
:1025A80089FE000889FE000889FE000889FE0008E7
:1025B8000401000089FE0008299C000889FE000823
:1025C80089FE000889FE000889FE000889FE0008C7
:1025D80089FE0008419C00080100000085230108CD
:1025E80084230108380100200000000000000000DA
:1025F80000000000000000000000000000000000D3
:102608000000000000000000B424010800000000E1
:1026180000000000000000000000000000000000B2
:1026280000000000000000000000000000000000A2
:102638000000000000000000000000000000000092
:102648000000000000000000000000000000000082
:102658000000000000000000000000000000000072
:102668000000000000000000000000000000000062
:102678000000000000000000000000000000000052
:102688000000000000000000000000000000000042
:102698000000000000000000000000000000000032
:1026A8000000000000000000000000000000000022
:1026B8000000000000000000000000000000000012
:1026C8000000000000000000000000000000000002
:0826D8000000000000000000FA
:04000005080041109E
:00000001FF
